:020000040800F2
:10000000F8FF0120C952090865530908393305086A
:100010006553090865530908655309080000000085
:100020000000000000000000000000006553090807
:10003000655309080000000065530908B901050867
:10004000655309086553090865530908655309088C
:1000500065530908655309084D1E0408551E040818
:100060005D1E0408651E04086D1E0408C506000018
:10007000D9060000ED06000001070000150700008A
:10008000290700003D07000065530908655309086A
:10009000655309086553090865530908751E040866
:1000A000655309081D350408655309080D35040812
:1000B0002D3504083D3504084D350408311A04086F
:1000C000251A0408651A0408591A04086553090812
:1000D000655309083110000085110000D912000095
:1000E0007D1E040865530908000000001936040845
:1000F000F135040829360408E135040851070000E9
:1001000065530908655309085D35040865530908F6
:100110002D140000811500006D350408759D080838
:1001200065070000790700008D070000A1070000A7
:10013000B5070000655309086553090865530908A8
:1001400000000000000000000000000000000000AF
:10015000C9070000DD070000F1070000D516000008
:10016000991A04088D1A040865530908655309088B
:100170006553090865530908655309080000000024
:100180006553090865530908291800007D19000006
:10019000655309086553090865530908655309083B
:1001A000655309086553090865530908655309082B
:1001B000655309086553090865530908CD1A0408F1
:1001C000C11A0408655309086553090865530908ED
:1001D00065530908E58B0808655309086553090844
:1001E00065530908655309086553090865530908EB
:1001F00065530908655309086553090865530908DB
:1002000065530908655309086553090865530908CA
:100210003936040849360408593604086553090874
:100220006553090865530908655309080000000073
:100230006553090865530908000000006553090863
:10024000655309086553090865530908655309088A
:10025000655309086553090865530908655309087A
:10026000655309086553090865530908655309086A
:100270006553090865530908D11A00000000000001
:1002800065530908000000006553090800000000DC
:0802900000000000655309089D
:020000040804EE
:100000004368426D30B49A61EFF31182502383F359
:1000100012884168D2B2856C0B68046D23EA05032F
:1000200023430B6082F31188436981681A68096869
:1000300022F00102D0E908541A60826A1D605C61F6
:100040005A60D0E90B429C60DA600023B0F86C2063
:1000500030BCCA620377704730B5FAB18E464FEABA
:10006000014C034600F1C005002419680C3353F815
:10007000042C43F8084C41EA0C0142EA0E02AB4260
:1000800043F80C1C43F8042CEFD1D0F8C03043EAFD
:100090000E03C0E93144C0F8C03030BD4FEA014E14
:1000A0008C46DEE710B40C4C6368002B11DD002099
:1000B00004F1080C0146DCF8AC3003F1C0025960D1
:1000C0000C339342FBD1013063680CF5867C83428C
:1000D000F1DC5DF8044B704704000020F0B5474C9C
:1000E00004EB401292F8543403B9F0BD4FF4B47CE1
:1000F000434B00264FEA401E0CFB004C9CF83A553F
:100100008CF83A6582F83A541D785A7895420DD0A9
:1001100002EB420C560003EBCC0C9CF804C00CF133
:10012000FF37012F5DD9BCF1030F55D004EB0E0052
:10013000A0F83814EFF31183902282F3128890F81C
:100140003A24DBB2B0F8381442EA4102002192B2FC
:1001500080F83A1483F311881309247883EA122370
:1001600083EA0201DCB11301C943D0F85024012411
:10017000D0F83C049BB201F00F01D2F8AC208440CF
:100180000B4302F1C000590013F4004F8BB202D1AF
:100190005168214351600C328242F4D1F0BD130109
:1001A000D0F83C44D0F8502401F00F0104F11000C5
:1001B0009BB20124D2F8AC200B43844002F1C00072
:1001C000590013F4004F8BB202D1516821435160A2
:1001D0000C329042F4D1F0BD571C07F00307AF4238
:1001E000A4D0324403EBC2030344597C00299DD0C0
:1001F00004EB0E03012283F83A2497E70400002061
:10020000181B0024704700BF024B03EB401090F80E
:100210005504704704000020704700BF0A4810F8DA
:100220004C1C81B101EB410100234438490010B45A
:100230001C4650F82320063302B114608B42F8D1DB
:100240005DF8044B70477047FC1000200A4810F816
:100250004C1C81B101EB410100234438490010B42A
:100260001C4650F82320063302B114609942F8D19D
:100270005DF8044B70477047FC1000200120704768
:10028000034B00EB400003EBC00010F8330C704749
:10029000FC1000202DE9F0431D4C14F84C3CABB38E
:1002A0000022A4F144034FF0500E1A4E4FF02C0CD4
:1002B000194F154607E053F8181B01320D6014F86A
:1002C0004C1C914222DD197C0029F4D05968FE2093
:1002D0004FEA9128A8F58018B8F1520F98BF17F887
:1002E0000800EFF311888EF31288D1F824900CFBEC
:1002F00000605FFA88F809F10109C0F88C9048693C
:1003000040F00100486188F31188D4E7BDE8F0832C
:10031000FC100020181B0024A06D090807EE900AAD
:10032000B8EE670A704700BFBCEEC00A10EE103A84
:1003300098B27047B4224FF4A57C4FF4EB710023C0
:1003400082802322A0F802C04FF4E17C02814FF4A6
:100350008772C1809621828144220370A0F80AC06E
:10036000C1814382028270470346012200205A77EE
:10037000704700BF08B5D0E90B2183690B44836146
:100380000AB108469047002008BD00BF436A0246F4
:100390001B681B6A5B685B7813F0010008BF50772D
:1003A000704700BFC2628161704700BF704700BFE5
:1003B00004307047C2628161704700BF436A0246E1
:1003C0001B681B6A5B689B7813F0010008BF5077BD
:1003D000704700BF0346012200205A77704700BFD4
:1003E00008B5D0E90B2183690B4483610AB1084643
:1003F0009047002008BD00BF704700BF0430704721
:100400000C4B93F8FC22D3F8F81202440844D2B201
:10041000C3F8F80283F8FC2293F8FC22120605D5F3
:1004200093F8FC2282F0800283F8FC22024B012226
:100430001A707047181B0024000000242DE9F84FA3
:10044000154FD7F80053ED0A20D00026DFF84CA056
:1004500007F54179B046AC19D7F80413102352467A
:100460006410D1F828B04846C7F83083E102D84775
:100470000F280BDD094B03F1100253F8041B013167
:1004800007D19342F9D12546B542E4DCE802BDE844
:10049000F88F661CF8E700BF181B0024E0DC00247E
:1004A000184BD3F83813D3F83C238A1A322A15D8BC
:1004B000D3F850238A4200D37047D3F84023E2B1E7
:1004C00010683231928810B44469C3F85013224244
:1004D0005DF8044B18BF120482617047D3F84023C3
:1004E0003AB193F84C031168C007928848BF1204D0
:1004F0008A610022C3F8502370473231C3F8501389
:10050000704700BF181B0024064AD2F840333BB1A5
:1005100092F84C131A68C9079B8848BF1B04936163
:1005200000207047181B0024044B4FF4007C00206F
:10053000D3F86033A2F800C00B607047181B00248A
:10054000002070470120704701207047002070474D
:100550002DE9F0411C4D0FF053FE00260746696857
:100560004FF48678002918DD00231C4608FB03524F
:10057000013392F805218B4244EA0204F6D10FF0D0
:100580003FFEC01BB0F5FA6FCCBF002304F001039F
:10059000B3B169681E460029E6DC0FF031FE26B1D2
:1005A0000A4B93F89023542A02D03046BDE8F081DC
:1005B000B3F8982330460132A3F89823BDE8F081C0
:1005C0003443E6B2EBE700BF04000020181B002410
:1005D0002DE9F04FBD4D87B02B781BB9012007B036
:1005E000BDE8F08F6B68BA4A002BD2F8387318DD7B
:1005F00005F108040020B749D4F8F430BFF34F8F59
:1006000003F59072C1F85C3220339342FAD1BFF304
:100610004F8FBFF36F8F01306B6804F5867498427B
:10062000EADBAD4BAD4EA3FB0723AD4FDFF8C8A20D
:100630005B09A7F17C0BA6FB0326F60806EB8606F2
:10064000A3EB4606F3B207EB8606059307F538736E
:10065000029300239946DBF864344B4540F30F8145
:10066000DAF81830DAF80480D3E93D540FF0C8FD09
:100670000122049002FA08F39A4901936118944BFD
:1006800005EB410193F8A40393F890331A460393C2
:1006900005EB4003542A00F04181019A994240F24F
:1006A0004481B3F800C01CEA020F00F04D81B3F89A
:1006B00002C01CEA020F00F04A81B3F804C01CEA31
:1006C000020F00F04781B3F806C008331CEA020F9E
:1006D000E4D10192A3EB050E99424FEA6E0E40F26F
:1006E0002481A4EB0E04452C28BF452403EB4404CD
:1006F000A34280F01F8100259C46019AA846294606
:10070000019618881040884214D1588810408142C0
:1007100040F0D78098881040814240F0D480D8883B
:1007200008331040814206D19C4207D918881040F6
:100730008842EAD002339C4200F2A880B8F1110F3F
:10074000019E40F2F780D8F1150200F1F38066496E
:10075000049C4B689E455E4BD3F8A80338BFC1F894
:1007600004E0231A002B13DB604B03449C4200F28D
:10077000F6805748C0F8A8334B68052B40F2ED804F
:10078000053BDBB2524880F8A4334FF0FF334B6097
:1007900042B105FA02F2C8F11408012505FA08F879
:1007A00048EA0205524BC5F3C43203EB8202506D96
:1007B00005F01F0203EB8202516DC5F34412C5F32D
:1007C000842503EB820203EB850541EA0031536D7A
:1007D00041EA03116B6D41EA032181EA112383EAA7
:1007E000131303F00F030F2B40F08880B1F5803F07
:1007F00080F08480039B0909542B05D1344AB2F858
:1008000094330133A2F89433DBF86433B1F5606FAD
:1008100003F10103CBF8643300F0B380029B9981AC
:1008200097F85830059883420CD0B2683B689B1A01
:100830003B607B68326B9B1A7B600023B360336341
:1008400087F858003B6801333B60B3680133B360FD
:100850004FF6FF73994205D17B6801337B60336BA0
:1008600001333363029B09F101095C375C361433B1
:10087000B9F1080F0AF1200A02937FF4ECAE0123CC
:1008800001208BF8603407B0BDE8F08FA3EB0C0CAF
:10089000184833F8021C4FEA6C0C11400CF1010CA3
:1008A00080FB0C60A0EBEC704FF0010C0128B8BF8E
:1008B00001208540804401380CFA00F09C46054335
:1008C0001FE7043337E7063335E700BF0400002095
:1008D000181B002400ED00E01F85EB51CDCCCCCCE3
:1008E00078110020C7FFFF7F0000002420A107002F
:1008F000A06D0908565555553C040020039B542B08
:1009000033D0DBF864330133CBF86433DBF8603386
:100910004FF6FF710133CBF8603381E7204A9942EB
:10092000A2F89A03019A3FF6BCAE18B101381C4BED
:1009300083F8A403039B542B94D1194AB2F896333D
:100940000133A2F896338DE702330192C2E60433F5
:100950000192BFE606330192BCE6002312E7049839
:100960000F4B0530C3F8A80306E70D4AB2F89433DD
:100970000133A2F89433DBF864330133CBF86433EA
:10098000C4E7074A537803EB430302EBC3034B442A
:100990005B7C0D2B7FF442AF8023029A93773FE775
:1009A000181B002410B5044655F088FA014620466D
:1009B00089B2BDE81040FFF791BB00BF00EB4000DB
:1009C00010B5084C04EBC00414ED0F7A54ED0E7A08
:1009D000E7EE007AB0EE670A55F070FA54F8443C3E
:1009E000186010BDFC100020F8B5264B1A785B7813
:1009F0009A4242D1244E7368002B23DD002506F174
:100A00000800224C2F46D0F8AC30BFF34F8F03F1D3
:100A1000E002C4F8683220339342FAD1BFF34F8F1B
:100A2000BFF36F8F337813B1037F012B20D042695E
:100A30000135716800F586701368A94243F001031F
:100A40001360E0DC0FF0DCFB114BD3F86844002CA2
:100A50000DDD03F26C4303EBC4041968083333F86B
:100A6000042CC8689C4242EA0002CA60F5D1F8BD75
:100A700080F8FC70FFF7C4FAD9E74DF019FF0028A1
:100A8000B8D1F8BD181B00240400002000ED00E0E0
:100A9000FC1000204FF0B042F8B5D2F88030D2F808
:100AA00088502B4003EA0005C2F888507DB1084FFA
:100AB0000126B5FA85F4C4F11F0407EB840306FA96
:100AC00004F4D3F8AC0303689847A543F1D1F8BD0B
:100AD000181B00240269C3682DE9F04712EA0309D4
:100AE0002AD005460E464FF000474FF00008B9FAED
:100AF00089F327FA03F21B3BD24309EA02092A6170
:100B0000042B16D8DFE803F03B30251A0300B36A44
:100B1000002B3FD003F1FF3AC6F828801FFA8AFA6B
:100B2000746A34B123682046514698476468002CA3
:100B3000F8D1B9F1000FDAD1BDE8F087706800286C
:100B4000F7D0696B036889B29847B9F1000FCED12D
:100B5000F2E7B0680028ECD0A96B036889B2984727
:100B6000B9F1000FC3D1E7E7F0680028E1D0E96BE5
:100B7000036889B29847B9F1000FB8D1DCE7306952
:100B80000028D6D0296C036889B29847B9F1000FC4
:100B9000ADD1D1E7E96A1FFA81FAC1E78069B430C3
:100BA00042F018BB38B590F828300446012B04D029
:100BB000407F40B10023637738BD406A03681A7BE9
:100BC0009AB9637F0BB9012038BD0A4D022305F1A4
:100BD000200205F140010EF08FFA95F8213003F064
:100BE000010383F001006377E6E71B6A002BE8D07E
:100BF000002038BDE0DC0024F8B5144E044690F81F
:100C0000281006F12007437F012904D00BB10023EF
:100C100063770120F8BD606A01680D7B85B9002B00
:100C2000F7D002233A460A490EF066FA96F82130C8
:100C300003F001036377002BEBD094F82810E3E76F
:100C40000A6A002AE8D1002BE3D0EAE7E0DC0024BE
:100C500020DD0024F0B511F0010583B00AD190F831
:100C600028600446012E07D0C368B3F1807F01D904
:100C70000123237703B0F0BD0A4B476AD3F83C0445
:100C80000EF02CFBE368B880B3F1807FF2D9B72176
:100C90002A46384633468DF8041001A926770EF00F
:100CA0002BFAE7E7181B002470B5002394B0054623
:100CB000224C069302200B9304F12002109313930D
:100CC000119301921E4E6A6A04960E460094029099
:100CD000CDE90E3301238DF80C3007938DF82030C9
:100CE0008DF834308DF848302B7F002B14BF05234E
:100CF00004230C9304F140030593124B0993A4F1D0
:100D000020030A93106853F01DF82B7FA3B1A4F1C0
:100D10008002330E1E3C82F86130320C6946330A81
:100D2000A67022706370686A0EF0B6F96B6A186874
:100D300053F008F814B070BD1F3CEEE760DD0024EE
:100D40008D0304086903040810B594B004465022CA
:100D50000649684655F030FE6946606A0EF09CF917
:100D6000636A186852F0EEFF14B010BD746E090883
:100D70002DE9F8431F46436A0446884618689146A1
:100D800052F0E0FF237F002B3BD0A0690523264DC6
:100D9000264EAB63030EE23606F8013CB070030C3E
:100DA000000A012F337070704FF00000D8F8003047
:100DB0006B64D9F80030EB642363E86527D0022F19
:100DC0001DD1D9F8042068651344D8F8041085F8BB
:100DD00050002A660122A9652363154B85F864201B
:100DE000AB66144B617F03F11402606A002914BFE3
:100DF000194611460EF050F9E36A7BB1206BBDE84D
:100E0000F883094D0423A0690B4EAB63C6E7084B7A
:100E100085F85070A86528666B65E2E7636A186814
:100E200052F090FFEAE700BF00000024E0DC00245D
:100E30007503040808000024C1DD002400B583B058
:100E40008161019201A9049A00930123C2626A465A
:100E5000FFF78EFF03B05DF804FB00BF2DE9F04300
:100E60009846436A95B0054618680E46344C91463C
:100E700052F068FF0223334A0027029304F590736F
:100E8000049204F58072009304F5A073297F019306
:100E9000012305928DF80C300697002937D08DF884
:100EA000343004F581748DF84830330ECDF82C9031
:100EB00004F8013C05238DF82070CDF8308013979D
:100EC0000793CDE90977CDE90E77CDE91077330C9B
:100ED000A6701D4F360A23706670D7F83C040EF0DA
:100EE000FDF96C6A6B7FA0803BBB05A920460EF024
:100EF000D3F86B6A186852F025FFD7F840040EF05B
:100F0000EDF96B6A9880404615B0BDE8F0838DF826
:100F1000343004F201148DF848300423CDF82C90BD
:100F20008DF82010CDF8308013910793CDE9091189
:100F3000CDE90E11CDE91011C9E76946D6E700BF2A
:100F4000E0DC00248D030408181B002410B590F881
:100F500028300446012B03D000230120637710BD05
:100F6000406A03681A7B3AB950F062F800F0010356
:100F700083F001006377F2E71B6A002BF4D00020B6
:100F800010BD00BF38B5114D044694F82830012B30
:100F900005D00023637700230120236238BD606AF7
:100FA00003681A7B72B950F043F800F001006077D3
:100FB0000028F0D0D5F83833226A9B1A002BE4DBE6
:100FC000002038BD1B6A002BEDD0F3E7181B00246E
:100FD00010B5FF22044690F82810406A53F0D0F96B
:100FE0000E4B2046D3F8383303F5FA732362FFF72C
:100FF000C9FF94F82830012B00D010BD0022A02199
:10100000606A53F097F994F82830012BF5D1606AA3
:101010001822B021BDE8104053F08CB9181B0024F1
:10102000CB0700D5704710B50446FFF7D1FF94F801
:101030002830012B00D010BD02480EF04FF9636A32
:10104000988010BD00E1F50538B504460D46FFF760
:1010500099FF062294F82810606A53F091F9012252
:1010600094F828306277934205D0074BD3F8383391
:101070000F33236238BDE288D821606AB5FBF2F2F3
:1010800053F034F9F1E700BF181B00242DE9F843B1
:10109000838853B304460025DFF85480012707E016
:1010A000D8F838330135A2880F33AA4223621CD9FD
:1010B0002046268AB4F80690FFF764FF062294F8CB
:1010C0002810606A53F05CF994F828306777012B98
:1010D000E6D109FB06F6E288D821606A05FB06F630
:1010E000B6FBF2F253F002F9DAE7BDE8F88300BF8D
:1010F000181B002470B5114D95F8443403B970BD28
:10110000C2880446D5F848640D4BB6FBF2F6C3F826
:101110008060FFF737FF94F82830012B07D0D5F80F
:1011200038330022023385F84424236270BD3246EE
:101130001021606A53F0DAF8F1E700BF181B0024B1
:1011400000000024B0F806C02DE9F047B1FBFCF523
:10115000DFF80CA11F4690B00646DAF880300C4646
:101160009046AB4222D1DFF8FC900CFB154496F878
:101170002830ACEB040CBC4534BF1FFA8CF5BDB273
:10118000012B3ED0D9F83833304602333362FFF7B3
:10119000F9FE38B196F82830012B25D0284610B03A
:1011A000BDE8F087002010B0BDE8F087FFF7EAFE49
:1011B0000028F7D04FF0FF33CAF8803096F8283077
:1011C000012B46D0DFF89C903046D9F838330233F3
:1011D0003362FFF7D7FE0028E4D0B6F806C0CAF89D
:1011E0008050B4FBFCF5C0E7706A4FF021FFC0F3FC
:1011F000011001380228D1D83046FFF7E9FE284611
:10120000CDE78DF80240240A8DF8243000228DF8B5
:10121000383003238DF8014001A9746A8DF800303D
:10122000042320468DF8032002928DF810200F929F
:10123000CDF804D00393CDE90787CDE90522CDE9A8
:101240000A22CDE90C220DF027FF206852F07AFD2A
:1012500098E72A461321706A53F048F8B2E700BFB6
:1012600000000024181B0024436A2DE9F047404E7B
:10127000044618680D46904652F064FD96F84434D2
:10128000002B41D0E288D6F84C34DFF8F0A0DFF82C
:10129000F090B3FBF2F102FB11338AF862311B0AC2
:1012A0008AF861312B684946324F606AC7F82431A9
:1012B00007F59272D8F80030C7F82C310023C7F830
:1012C00034310EF0A7FAD6F84C340120D8F80020BB
:1012D000E188134486F84404B3FBF1F501FB1535AE
:1012E000C6F84C3425B3244BC7F83431637F0BB9AF
:1012F00009F114094946606A22630DF0CDFEE36AE4
:101300007BB3206BBDE8F087A369E288DFF86CA0AF
:10131000C6F84C34C6F84834DFF86890B3FBF2F1F5
:1013200002FB11338AF882311B0A8AF88131B9E74E
:10133000D6F8483407F5A672606AB3FBF1F1C7F836
:10134000801049BAAAF8A21107F592710EF062FA5C
:10135000D6F84C34D8F8002086F84454C6F84834FF
:10136000C4E7636A186852F0EDFC206BBDE8F087B3
:10137000181B002400000024E1030408E0DC002422
:1013800084000024D400002433B910B51C46C36A7D
:1013900020469847204610BD66E700BF10B582B0D2
:1013A0000C46019201A9049A8461C2626A460093C4
:1013B000FFF75AFF02B010BD2DE9F843DDF8208099
:1013C0000F4616460021202204461D4655F068FBB4
:1013D000B8F1000F0CD0D8F80030B8F80A20E3813B
:1013E0001B0C2382D8F804306282E3821B0C238317
:1013F000384653F069F8F30619D4431EB8B107EB29
:10140000000C01E0013B12D31CF801EDBEF12E0FE0
:10141000F8D1C01A03F10109421EB944032AA8BF3A
:101420000322082BA8BF082390461A4606E0082886
:101430000246B9464FF00008A8BF08224FF02033FB
:10144000394620462360636055F0B6FA04F108037C
:101450001748424649462081A072184655F0ACFA1A
:1014600004F1FF3C0346E21D1CF8011FA1F1610ECF
:101470002039BEF1190F98BF8CF800106245F3D1E6
:10148000184604F10B0110F8013BA3F16102203B67
:10149000192A98BF00F8013C8842F4D118236583CB
:1014A0002D0CE6722373099BA582E361BDE8F883E6
:1014B000202020002DE9F04FDFF88C9487B0D9F878
:1014C0003803C9F83C03002B00F0DA8013441546BA
:1014D00001F1200601F5FE77DFF870A403931FE009
:1014E000002D63D0D9F86C23AA4200F0CD80D9F842
:1014F0006823AA4200F00281D9E9DC21AA424CD833
:10150000A94200F2CF81691A18464CF06FF90135F3
:10151000039B06F5007607F500779D4200F0B0804A
:10152000D9F87843A6F12003AC42D9D82C1BD9F8BE
:101530008883E208D8F8301004F0070402328A42A7
:1015400003D3D8F838108A420DD941461046059386
:1015500004924CF01BF98046DDE90423002800F0DA
:10156000C181C9F8880398F80410002940F03F8130
:10157000D8F828B0BBF1000F00F0AD811846D8F8BC
:1015800030304FF40071D21AD8F80C3004EBC2029C
:1015900003EB42224346D847B9E7A942B3D91846DC
:1015A0004FF40072002155F07BFAB0E74FF400725F
:1015B0002946184655F074FA80220346D94886F821
:1015C0009E210C2286F8A221D9F86813D9F860234D
:1015D0008142C3F8C611C3F8CA2100F36881D24B17
:1015E000013AD24C83FB0103C81784FB01C40B44AE
:1015F000C0EB6313C0EB2430CD4C84FB03C4C3EBBE
:10160000831C86F8A1018010A1EB0C011C4420F082
:101610003F000131014386F8A011D917C1EBE41155
:101620000B4486F89F31BF4B9A4200F34C81BE4B6E
:10163000BE4883FB0213D11780FB02401344C1EB69
:101640006313C1EB2031BA4880FB0340C3EB831422
:1016500086F8A5118910121B184421F03F010132B0
:101660000A4386F8A421DA17C2EBE010034486F897
:10167000A331552386F8DE31AA2386F8DF3146E709
:10168000002007B0BDE8F08F4FF0FF320024A6F134
:101690001C00049383F8EC21214683F8ED2183F8A4
:1016A000EE2183F8EF2152221A705A7061229A704B
:1016B00083F8E7214122DA7083F8E621722283F869
:1016C000E42183F8E521D9F88023C3F8E8214FF419
:1016D000F07255F0E5F9049B5522C6F8D041C6F8E2
:1016E000D441C6F8D84183F8FE216FF0550283F843
:1016F000FC4183F8FD4183F8FF2108E78D4C002170
:101700004FF40072184655F0CBF903464FF0000C29
:10171000022203CC46F8191CEB2146F81D0C0820C8
:1017200006F8201C582106F81F1C902106F81E1CE4
:10173000F8211A7383F80BC006F8130C9A7383F818
:101740000FC006F8102C06F80B1C83F82C20D9F8D3
:101750006813D9F8602383F819C0521A83F81BC0A4
:1017600083F81DC01A6283F81EC083F81FC083F877
:101770002DC083F82EC083F82FC0D9E9DC12521A8D
:1017800080215A623F221A764FF0FF329A763E222B
:101790001A77012283F8302083F831C086F82010B0
:1017A0002921654B86F82210942186F8260086F8B8
:1017B00023100E21614A86F824100D2186F8251089
:1017C000552186F8DE11AA2186F8DF1103CBC6F871
:1017D0002B101988C6F827009B78A6F82F1086F8DA
:1017E000313003CAC6F83200C6F836108FE64FF41F
:1017F00000721846002155F053F9D8F840200346EE
:10180000002C76D1002A00F0A380D8F830301122C5
:101810004B49CDE90044FFF7CFFDD8F840301A6CB2
:10182000002A00F0A1801B6BCDE90044112245493C
:1018300030464FF4E07BFFF7BFFD06F12003D8F8F8
:101840004480B8F1000F3FF462AE03F120049B44E2
:10185000049523464446984610E05CF81C1B00257E
:10186000236BCDE900C5FFF7A7FDABEB0803A46C24
:1018700008F12008002C18BF1F2B51D92379A4464A
:1018800004F11C0E1122A8F12000002BE5D1627991
:101890002569236B42F021022168CDE900E5FFF7BD
:1018A0008BFDE2E7A91A18464BF0A0FF2FE6FF23B5
:1018B000013A86F89F3186F8A13186F8A031194B9C
:1018C0009A427FF7B4AEFF2386F8A33186F8A5319C
:1018D00086F8A431CDE6594618464FF4007255F00B
:1018E000DFF814E6A6F1240343F804AF9F42FBD1CE
:1018F0000DE6002AD8F844800CBF01220222C2EB78
:101900000414B8F1000F3FF402AE4246013C926C61
:10191000002C01DD002AF9D190464FF4007B90E7BE
:10192000049DF4E5FF03FB008320088297554541A1
:1019300081808080F8EB090804EC090810EC0908A4
:10194000F0EB0908F4EB0908181B0024DEADBEEF2C
:1019500023460822D9F864134FF4F07BCDE9004404
:10196000FFF72AFD33466AE72346CDE900445DE7E9
:1019700010B4294C94F88C346BB3D4F8942490426E
:1019800035D0012B27D0D4F87025824237D0022BD6
:1019900021D0D4F84C26904233D0032B1BD0D4F85E
:1019A000282790422FD0042B15D0D4F80428904239
:1019B0002BD0052B0FD0D4F8E028904227D0062B4F
:1019C00009D0D4F8BC29904223D0072B03D0D4F8F7
:1019D000982A824211D0DC22591C02FB034284F86F
:1019E0008C14C2F8940418465DF8044B7047002329
:1019F000DBB25DF8044B184670470723F8E7012374
:101A0000F6E70223F4E70323F2E70423F0E70523D4
:101A1000EEE70623ECE700BFFC1000200020704733
:101A2000704700BF014845F085BD00BF801F0024FE
:101A3000084810B4D0F86834D0F89C4499691A6802
:101A40002CB1234600F58D605DF8044B18475DF816
:101A5000044B7047181B0024014845F06BBD00BFC4
:101A6000E41F0024084810B4D0F8CC34D0F8004566
:101A700099691A682CB1234600F2CC405DF8044BFA
:101A800018475DF8044B7047181B0024014845F0C7
:101A900051BD00BF48200024084810B4D0F83035AC
:101AA000D0F8644599691A682CB1234600F5A66000
:101AB0005DF8044B18475DF8044B7047181B002471
:101AC000014845F037BD00BFAC200024084810B4E1
:101AD000D0F89435D0F8C84599691A682CB12346D6
:101AE00000F294505DF8044B18475DF8044B7047C2
:101AF000181B0024114A037A0168D35C10B4CC5837
:101B0000CA1824F00104CC501368DB07FCD4037D11
:101B10001F2B09D9203B20225DF8044B02FA03F366
:101B200043F01803CB60704720225DF8044B02FAA3
:101B300003F343F018038B60704700BFC0EC090843
:101B4000F8B507680646D7E90454A0612B7D1F2B22
:101B500049D9203B2022286802FA03F343F01803F6
:101B6000C360237D1F2B48D92022203B02FA03F3B8
:101B7000226843F01803D3606368002269680A6032
:101B80001A601A6842F010021A60BA69297A50F095
:101B9000ABFEFA69217A206850F0A6FE33682E6801
:101BA0001A6A5B6891685868184A024020680A43BC
:101BB00017495A602A7A8D5C725942F001027251BB
:101BC000227A895C425842F0010242509A6842F4FB
:101BD00040429A601A6842F001021A601A6842F4A0
:101BE00000721A60F8BD2022286802FA03F343F05D
:101BF00018038360237D1F2BB6D8202202FA03F33B
:101C0000226843F018039360B6E700BF0000FFFFAF
:101C1000C0EC090810B1036882889A61704700BF60
:101C200018B1838802681B049361704708B51D20B2
:101C30000DF0FAFE08B183794BB11E200DF0F4FED1
:101C400008B1837903B108BD5523C38008BD55236E
:101C5000C380F2E7D3B20F2B2AD84FF0000C10B498
:101C60006346144C04E001332A2B1DD014F803CF33
:101C70006045F8D194F801C08C45F4D10E4C03EBCB
:101C800043030E4902EB420C23445DF8044B01EB85
:101C90008C0201F5CE7093F8263100EB8C00C2F86F
:101CA000A43182F89C31704700205DF8044B7047E6
:101CB00000207047C46E0908A06D090800000024C8
:101CC00010B40C4C002304F5BC6C01E0152B0CD0B7
:101CD00003EB430201331CF802108142F6D1224487
:101CE0005DF8044B92F9E20570474FF0FF305DF864
:101CF000044B7047181B002430B40023114C124DC4
:101D000004E001331A2B1AD054F8085FA842F8D126
:101D100025798D42F5D10D4C02EB42050C4904EBBF
:101D2000C30301EB850201F5CE7093F8A93100EBF6
:101D30008500C2F8A43182F89C3130BC7047002085
:101D400030BC7047446F090800000140A06D0908CD
:101D500000000024F0B1002310B504460E4894F8AA
:101D600004E000F5BC6C01E0152B11D003EB43023D
:101D700001331CF802107145F6D1024461792068E4
:101D800092F9E225D3B20F2B02D8BDE81040B3E799
:101D9000002010BD00207047181B00240138074B9D
:101DA000074A00EBC00003EB8000D0F85C029042D1
:101DB0000CBFA020A1204DF0F5B800BF000000240A
:101DC0000000024001382DE9E84100EBC000134D4E
:101DD0001E46134B05EB800590460F46D5F85C0276
:101DE00098420CBFA020A1204DF0DCF8B5F972029A
:101DF0004FEA9811C5F86C72C5F874624DF050F84E
:101E0000B5F97232002B07DB03F01F0001225B09DA
:101E10000449824041F82320BDE8E8810000002405
:101E20000000024000E100E0800AA0F58010522886
:101E300006D8044B1B5C0D2B02D8034AD0567047C2
:101E400000207047A06D0908B0EC09080120FEF7DA
:101E500021BE00BF0220FEF71DBE00BF0420FEF71A
:101E600019BE00BF0820FEF715BE00BF1020FEF708
:101E700011BE00BF4FF47870FEF70CBE4FF47C40EB
:101E8000FEF708BE30B1036882881B691A4214BF8E
:101E900001200020704700BF70B50C4686B0054693
:101EA000164640B101680E4B0E4A0B449B0A02EBEA
:101EB0004303B3F874024DF075F804F01303AA88D5
:101EC00001A90293C4F341132868C4F38104019269
:101ED0000596CDE9033445F0E7F906B070BD00BFC3
:101EE0000000FEA7A06D090800B1D5E770472DE9F5
:101EF000F84FC34F6423044603FB0073D3F85064C8
:101F0000002E00F06D81D3F858A4BAF1000F04D070
:101F10009AF80630002B40F06381642303FB0473BE
:101F2000D3F85C541DB1AB79002B40F05981631C90
:101F3000DBB2BAF1000F04D015228AF807308AF814
:101F4000062015B11622EB71AA714FF06409308B8F
:101F50004DF028F8294609FB04F9504651F0F6FEE9
:101F6000504607EB090898F8623498F86024002B73
:101F700014BF3E211E21FFF7B7FF98F862342846B0
:101F8000A04D002B98F861244D44DFF8989214BFBF
:101F90003E211E21FFF7A8FF4C220021284654F0C5
:101FA0007FFDD8F85034984A5B689342C8F868348B
:101FB000DFF8748240F0168145F052FED9F82030E7
:101FC000C3F302139FED917A9FED915AB0EE084A48
:101FD0004344F7EE003A4FF0000E40F2145893F8E5
:101FE000883203F01F03D840642307EE900A03FBF6
:101FF0000473F8EE677AB3F86494C7EE275A07EED5
:10200000909A9FED847AF8EEE77AC7EE274ADFEDE3
:10201000827AB0EE007AE5EE877AA5EE875A25EE51
:10202000844A37EE856A74EEE72AB9F5C87F0EF167
:10203000010CD5BF642332234FF49670782007EE4D
:1020400090CAD8BF4FF4167A0344C8BF4FF4827ABF
:10205000B8EEE77AD8BF414607EE903AC8BF4FF4D2
:10206000FA7127EE257A01EB0A03F8EEE76A86EEAD
:10207000873A73EE636AFCEEE67A17EE902A07EE73
:1020800090AAB8EEE73A07EE903AF8EEE77A23EE38
:10209000243AC3EE276A36EEC53A72EEE66AC3EE1C
:1020A000077A77EEE37AFCEEE77A17EE901AC6EE3F
:1020B000877A77EEE37AFCEEE77A17EE903A03F14F
:1020C000020A0AEB010BF0EE466A07EE90BAF8EE50
:1020D000677AE7EE276AF4EEE64AF1EE10FA00F3CB
:1020E00088805FFA82FABAF10F0F00F284803238EA
:1020F00007EE900AF8EEE77A77EEC47AC7EE876AC1
:10210000FCEEE67A17EE900A5FFA80FABAF10F0F4A
:1021100071D81FFA81FABAF1FF0F6CD81FFA83FA4F
:10212000BAF1FF0F67D812054AEA0E7302F07F6218
:102130000004134300F47F00384A034302EA0121FC
:102140000B43642000FB047400272846C4F86C3459
:102150000123C4F87074C4F87434C4F87874C4F8F3
:102160007C74C4F88474C4F8887451F043FA94F809
:10217000A934202BD9B21AD194F8A834012B16D047
:10218000242384F8A934D4F868341A6822F00102B0
:102190001A601A6822F480521A601A681A601A6863
:1021A00042F001021A6084F8A91484F8A87400218E
:1021B000F07E4CF075FEF37E0124194D5A0903F0B0
:1021C0001F03002104FA03F345F82230B07E4CF0DF
:1021D00067FEB37E5A0903F01F039C4045F8224076
:1021E000BDE8F88F45F03CFDD9F81C30E8E6E6463E
:1021F0001BE7013165E7BCF10F0FF8D10023A0E721
:10220000181B0024801F0024001C0058286B6E4EF1
:1022100000001643002474490000704200FFFF00D4
:1022200000E100E000440258A06D09082DE9F843E0
:10223000B14C04EB0017D7F82036002B00F0BF801C
:1022400005460601B7F82A064CF0ACFEB7F82A3668
:10225000012103F01F025B09023B01FA02F2082B85
:102260000FD8DFE813F00801100118012001280140
:102270000900300138014001A04BD96F21EA020268
:10228000DA67A319013593F82406EDB20DF0CCFB03
:10229000074610B11223C5718371A31993F825065F
:1022A0000DF0C2FB814610B11323C5718371A319D0
:1022B00093F826060DF0B8FB804610B11423C571C3
:1022C0008371344448462E2194F82826FFF70CFEEB
:1022D00094F829260E214046FFF706FE94F827269B
:1022E0002E213846FFF700FED4F8203684491A68BC
:1022F0008B4222F001021A6063D0824A934200F0BE
:102300008F8002F58062934279D17C4AD2F8901096
:1023100041F40041C2F89010D2F8901021F400412D
:10232000C2F89010DA6842F00042DA609A6822F44B
:10233000F0729A601A68D60741D473499D68D1F843
:10234000B424D1F8BC4444EA0200D1F8A4241043D8
:102350006E4A2A401043D1F8B0249860DD68D1F865
:10236000A004ED007BD50243D1F8A804DE68B4F5E3
:10237000800F42EA0002D1F8AC04654D42EA000247
:10238000D1F8B80405EA060542EA0002D1F89C0437
:1023900000F4C02600F4006042EA060242EA0502A8
:1023A000DA601A6822F4006242EA00021A6002D17E
:1023B000D1F8C0241A641A6D22F001021A65BDE832
:1023C000F8834E4AD2F8981041F48051C2F8981020
:1023D000D2F8981021F48051C2F898104D4A9342D7
:1023E000A0D1464AD2F89C1041F02001C2F89C10BE
:1023F000D2F89C1021F02001C2F89C1092E7464AC6
:1024000093421BD13D4AD2F8981041F40051C2F8D2
:102410009810D2F8981021F40051C2F8981081E772
:10242000364AD2F8901041F48041C2F89010D2F8A8
:10243000901021F48041C2F89010CFE7374A9342C0
:10244000CCD12E4AD2F8981041F48011C2F89810DD
:10245000D2F8981021F48011C2F8981062E7B2F116
:10246000806F80D1B0F5800F7FF47DAF1D6845F49B
:1024700080551D6077E7214BD3F8981021EA0202BE
:10248000C3F89820FDE61D4BD3F8901021EA020214
:10249000C3F89020F5E6194BD3F8941021EA020214
:1024A000C3F89420EDE6154BD3F8801021EA020220
:1024B000C3F88020E5E6114BD3F8841021EA02022C
:1024C000C3F88420DDE60D4BD3F88C1021EA02021C
:1024D000C3F88C20D5E6094BD3F8881021EA020214
:1024E000C3F88820CDE6054BD3F89C1021EA020200
:1024F000C3F89C20C5E600BF181B00240044025806
:10250000003001400038004000000024E0FFBF8F91
:10251000FFFF39D80014005800340140005001403A
:1025200008B10022B8E470470E4B70B5D3F864646C
:10253000002E14DD0C4C002503E0B54204F120040C
:102540000DD0237F0135002BF7D0E0680022002852
:10255000F3D0217D2034FFF79FFCB542F1D101205B
:1025600070BD00BFFC1000203C040020F8B590F8BE
:10257000EE311C09013C062C0FD81B4E054603F01A
:102580000F0306EB4402B2F8B80240FA03F2D20796
:1025900003D595F8F971012F01D00120F8BD07FA94
:1025A00003F33444013B184052F0BAFC94F8C822BB
:1025B00013180E4A02EBC30152F833208B881069BE
:1025C0001840EBD0002395F8EF210846022185F84A
:1025D000F931FFF761FCD5F850213846136843F014
:1025E00008031360F8BD00BFA06D090898210024FE
:1025F000014B53F82000704750400058014B43F8FE
:10260000201070475040005819481A4B01681A4A68
:1026100041F4807130B4016082B0D3F8F410FF242B
:10262000CA2041F48031C3F8F410D3F8F41001F457
:10263000803101915321019D546250625162D3F85F
:10264000D030DB010CD40D4B00210D4A43F8041BA4
:102650009342FBD1084B0B4A1A6502B030BC70475D
:10266000126D084B9A42EED102B030BC704700BFE9
:102670000048025800440258004000585440005896
:102680006C40005831666542F0B50446D0F85C01F4
:10269000454B83B0A16804F5967204F1E0070E681B
:1026A000C1B220F0FF0001921039A3FB01310909EA
:1026B00050F06AF9D4F81C110023019A012984F81A
:1026C000203118D0042916D0102958D0402912D012
:1026D000B1F5807F56D0B1F5806F53D0B1F5805FF2
:1026E00058D0B1F5803F4FF03C030CBF6FF0080CA1
:1026F0006FF4006C01E06FF0080C06F1180530462D
:10270000E95801EA0C01E950D4F81C114FF0DCFD46
:10271000D4F81C31012B16D0042B14D0102B0FD061
:10272000402B10D0B3F5807F30D0B3F5806F2DD023
:10273000B3F5805F32D0B3F5803F06F1540502D087
:102740004FF4006100E008212B683A46D4F85C01A0
:102750000B4340212B60C4F8E810C1B2124B20F0AB
:10276000FF001039A3FB0131090950F0BDF8D4F87E
:102770005C21136843F01003136003B0F0BD6FF4E5
:10278000006CBAE76FF0080C0423B6E706F11C05ED
:102790000821D9E76FF4006C0423AEE706F11C05AD
:1027A0004FF40061D0E700BFABAAAAAA2DE9F04F11
:1027B000DFF848B185B09BF8004024B901242046D9
:1027C00005B0BDE8F08F474BD3F838530DF018FD36
:1027D000454A92F8B83B002B00F0BC81434B02F114
:1027E0007C070BF5A7640026A3FB0513404D5B098E
:1027F000A5FB0315ED0805EB8505A3EB4505D2F810
:102800007C3BC31A0193EBB207EB8505029302F5FB
:1028100057730093019A002A04DBD4F824319342C1
:1028200000F37C814FF4B47303FB06B393F858367E
:10283000002B00F0C080D4F85C11A3682D481A6802
:10284000CBB221F0FF01103BA0FB03032A481B0978
:10285000C35C19444B68A1891FFA83FED368CEF18B
:10286000160E23EA0103BEF1070FD36040F2A380E6
:102870001D4A0121D2F864338A460133C2F8643319
:102880000022D4F8643190469C4603935CF8049B84
:1028900048461DE0DCF80090B8F1140FA9EB0003E6
:1028A00048462DDC13F1080948BF03F117094FEA28
:1028B000291308EB291803F1FF39013102FA03F358
:1028C0000CF1040C0AFA09F28E4542EA030217D30E
:1028D0008E45DFD8C8F11503DCF800004FF015086D
:1028E000E9E700BF181B0024FC1000201F85EB51F6
:1028F000CDCCCCCCABAAAAAAC0EC0908040000201D
:10290000B8F1150F40F000819649C2F38423C2F359
:10291000441001EB830301EB8000D3F8D032D0F8F0
:10292000D0021B0243EA001302F01F00C2F3C432BC
:1029300001EB800001EB8202D0F8D012D2F8D02255
:102940000B4343EA023383EA132282EA121202F0B3
:102950000F020F2A40F0D880C3F30F134FF6FF7217
:10296000934200F0D180B3F5606F00F0DC80009AF4
:10297000938197F85820029882420CD0A9683A684F
:10298000521A3A607A68296B521A7A600022AA6059
:102990002A6387F858003A6801323A60AA6801321F
:1029A000AA604FF6FF72934205D17B6801337B60CA
:1029B0002B6B01332B63009B204601365C371433AD
:1029C0005C3504F5B4740093FFF75EFE664B93F834
:1029D000B83BB3423FF71EAF63480121002280F8A5
:1029E0006014C0F87C2B002B3FF4E8AE9BF8102657
:1029F000DBF8540612F0020FDBF8402511680A6A72
:102A00000CBF024342EA8002012B0A623FF4D6AEB9
:102A10009BF87827DBF8BC0712F0020FDBF8A8263A
:102A200011680A6A0CBF024342EA8002022B0A6262
:102A30003FF4C4AE9BF8E028DBF8240912F0020F43
:102A4000DBF8102811680A6A0CBF024342EA8002D0
:102A5000032B0A623FF4B2AE9BF8482ADBF88C0ADB
:102A600012F0020FDBF8782911680A6A0CBF0243E2
:102A700042EA8002042B0A623FF4A0AE9BF8B02B1E
:102A8000DBF8F40B12F0020FDBF8E02A11680A6A97
:102A90000CBF024342EA8002052B0A623FF48EAE6D
:102AA0009BF8182DDBF85C0D12F0020FDBF8482CB8
:102AB00011680A6A0CBF024342EA8002062B0A62CE
:102AC0003FF47CAE9BF8802EDBF8C40E12F0020FB0
:102AD000DBF8B02D11680A6A0CBF024342EA80029B
:102AE000082B0A627FF46AAE9BF8E83FDBF8182FE8
:102AF00013F0020F1D4B1268D96A136A14BF43EA20
:102B000081030B43136259E6174AD2F8603301334D
:102B1000C2F86033B6B14FF6FF732AE700242046AF
:102B200005B0BDE8F08F12494A7802EB420201EB92
:102B3000C2023244527C0D2A7FF419AF80220099E0
:102B40008A7716E7039958220A4853F035FF4FF663
:102B5000FF730EE704490122C1F87C3B81F8602431
:102B60002DE600BFA06D0908FC1000200410002015
:102B7000181B002404150020D0F850112422F8B5A9
:102B8000C0F8D02104460A680023806804F5A875BF
:102B900022F001020A600B604B608B6094F805C064
:102BA000C4F8D83184F8CC31C4F8D031C4F86831D5
:102BB000C4F8D431C4F87031C4F864314FEA8C23BE
:102BC000B44A03F48053C4F854019142C4F8583114
:102BD0004FEA0C3303F40053C4F85C314FEA0C2382
:102BE00003F48063C4F8603100F0AE81237913F000
:102BF000010002D00422C4F8642113F0020305D0BE
:102C0000D4F8642142F00802C4F864211CF0010FDA
:102C10000DD048B1D4F8782142F00202C4F87821EE
:102C20004FF48032C4F88021002B40F081819A4B10
:102C300003F12C0053F8042B944200F03F8198429A
:102C4000F8D11CF0080F40F04F81D4F8D031002BA0
:102C500000F09C8124232846C4F8D0310B6823F06F
:102C600001030B6045F072FC012815D0D4F87831CF
:102C7000002B40F09181D4F8503128465A6822F454
:102C800090425A609A6822F02A029A601A6842F0CA
:102C900001021A604FF076FF2379DA076DD5D4F878
:102CA0002C21002A00F05F810023D4F8341104F1B4
:102CB0003C06E2634FF48062C4F8B8103046E26428
:102CC000C4E91133C4E91433C4E91833C4E91A332D
:102CD0004FF48033E3654FF48073A36550F0D8FC64
:102CE000304640F001FFD4F8D431C4F8C861202B3D
:102CF00065673DD1E368626999B2CAB3B1FA81F000
:102D00004009A9B394F8CCC1BCF1010F30D02227FF
:102D1000C4F8D80194F870C0C4F8D4715F4FA4F817
:102D2000AC110121A7675E4F8C45C4F8A821E76765
:102D30005C4FC4F88C0084F8CC11C4F888700ED0B5
:102D400094F8717084F87010012FD4F8501100F0CD
:102D50002B814FF4006384F87000C4F89030102188
:102D600000222023C4F8D81184F8CC21C4F8D03133
:102D7000E26B23795268C4F844219B0740F18880B4
:102D8000D4F83021002A00F0E3800023D4F8381171
:102D900004F1B406C4F8B420C4F8C0304022C4F82A
:102DA000D0303046C4E93233C4E93633C4E938336D
:102DB0004FF48033C4F8D4304FF48063C4E92E124A
:102DC000C4F8C43050F064FC304640F08DFE00285A
:102DD00040F0B980D4F8B420334B344834498242AF
:102DE00018BF9A42C4F8C461C4F8EC5000F1600006
:102DF0000CBF012300232F4C8A4208BF43F001037C
:102E00003031A24208BF43F0010360348A4208BF58
:102E100043F001033031824208BF43F0010300F563
:102E200068708A4208BF43F0010301F55C71A24259
:102E300008BF43F0010304F568748A4208BF43F0F9
:102E400001033031824208BF43F0010360308A42FF
:102E500008BF43F001033031A24208BF43F0010331
:102E60008A4208BF43F001033031824208BF43F079
:102E700001038A4208BF43F001033BB90E4BD31A4A
:102E8000B3FA83F35B09002B00F0A78000235360A3
:102E9000F8BD00BF000C0058BC1C0020614A0808A7
:102EA000954A0808994A0808100002402800024084
:102EB0004000024058000240B8040240002C3FF499
:102EC000C0AE94F8F831002B3FF4BBAED4F87831A3
:102ED0001CF0080F43F00803C4F878314FF40043A6
:102EE000C4F888313FF4B1AED4F8D031002B50D0C3
:102EF00024232846C4F8D0310B6823F001030B606B
:102F000045F024FB01283FF4C7AED4F87831002BFC
:102F100046D1D4F8503128465A6822F490425A607B
:102F20009A6822F022029A609A6842F00802ACE69F
:102F3000D4F8783143F00103C4F878314FF400330A
:102F4000C4F87C3173E6FEE70423C4F874314DE61F
:102F5000D4F8DC311A6842F080021A601A6842F034
:102F600040021A60F8BDD4F8DC21116841F4807188
:102F70001160916841F001019160116841F02001F8
:102F80001160116841F010011160F6E684F8CC314F
:102F900060E684F8CC31ABE7284645F0ADFD6AE643
:102FA000284645F0A9FDB4E79BB22431304643F0F2
:102FB0009DFE00287FF4D3AED4F8503184F8CC01C4
:102FC0001A6842F480721A609A6842F001029A60AC
:102FD0009A6842F040029A60CAE65360F8BD00BFAA
:102FE000F8B50446EFF31185502383F31288D0F827
:102FF00030311B6803F001031BB1EDB285F311887A
:10300000F8BDD0F8D021D0F8D4110A4302F0210243
:10301000212AF2D0D0E909218A424FD04BD8006949
:103020001A46431A9BB2A262002284F8E021D4F827
:10303000D021202AE1D1A2695118DED0B3FA83F25F
:103040005209002BD9D094F8CC010128D5D02120E9
:10305000A4F8A6314FF0010CC4F8D821C4F8D0016F
:10306000D4F8C401C4F8A011A4F8A43184F8CCC1E8
:1030700070B31D4E90F834E0C6631C4EE645026501
:1030800006641B4EC6640CD090F83560D4F85071BD
:10309000664580F834C015D04FF4006380F83420C2
:1030A0004365102100222023C4F8D81184F8CC21D4
:1030B000C4F8D031A1E7531A9BB2B4E7012380F8DA
:1030C000E0319AE707F1280243F010FE0028E8D12A
:1030D000D4F8503100224021196284F8CC219A683A
:1030E00042F080029A6088E7394A08085D4A080879
:1030F000994A08082DE9F8434D4C04EB8004D4F8B4
:10310000C04B002C44D0D4F8E8511F46494B06462A
:10311000A1602046236090466B68C4F8DC31AB6B3D
:1031200063616B6BA361EB8FE360AB8F2361424BF9
:10313000C4F8E4310CF022FE6B68A88DC4F850315D
:10314000002863D194F8EE010CF06EFC022117F018
:103150000802034694F8EC9184F8F9111BD060B38F
:1031600017F0510F4FF00B0206F1010614BF0A21B0
:103170001A2117F0410FC671827114BF402320231A
:1031800094F8EF211943FEF787FED4F82C314BB3A6
:103190002046BDE8F88318F0020F0ED068B14FF05A
:1031A0000B0C3B0680F806C006F1010C80F807C046
:1031B0002FD494F8EF21FEF76FFE48460CF034FC54
:1031C0000028E2D018F0010FDFD00C2201360221D6
:1031D000C671827194F8ED21FEF75EFED4F82C31B1
:1031E000002BD5D195F8321095F8300089094BF0B5
:1031F00057FE95F830300122104903F01F005B099B
:103200008240204641F82320BDE8F8834BF0CAFEF7
:1032100098E7D4F850714FF0010C20213B6823F05F
:1032200008033B6084F8F9C1FEF736FEC5E700BF2E
:10323000FC100020F07009086D25040800E100E092
:10324000BFF34F8F0549064BCA6802F4E06213438F
:10325000CB60BFF34F8F00BFFDE700BF00ED00E084
:103260000400FA0519484FF6FF0C194A84B0C168EA
:10327000184B01EA0C010A43C260D3F8D020D3F8FE
:10328000DC2042F00052C3F8DC20D3F8DC2002F04E
:1032900000520192019AD3F8DC2042F08042C3F838
:1032A000DC20D3F8DC2002F080420292029AD3F8AC
:1032B000DC2042F00042C3F8DC20D3F8DC3003F01D
:1032C00000430393039B04B00CF04EBF00ED00E0FD
:1032D0000005FA050044025808B51D480023C0F84F
:1032E0008430BFF34F8F436923F480334361BFF3CE
:1032F0004F8FD0F8803043F6E074C3F34E3CC3F3F5
:10330000C90E4FEA4C1C0CEA0401734641EA837271
:10331000013BC0F874225A1CF8D1ACF1200C1CF10E
:10332000200FF0D1BFF34F8FBFF36F8FBFF34F8FDD
:10333000BFF36F8F4369002223F400334361C0F869
:103340005022BFF34F8FBFF36F8F72B6FFF778FF36
:1033500000ED00E003689B0AA3F58013522B57D8B9
:1033600070B53E4C14F803C0BCF10D0F4FD8407936
:103370008508002951D04FEA900E4C2438480CEBB8
:103380008C0304FB0C040CEB4303D4F8006A022406
:103390002B4404FA0EFEF46800EB83054EEA0404A5
:1033A000A966AA67F460EFF31184502383F31288AF
:1033B0002C2303FB0CF3C1184A6E52B3131DC1F842
:1033C0008820284A2C21284D01FB0CF105EB010E29
:1033D00014310A4452F8041B19B1196052F8043C24
:1033E00004339645F6D10022E4B21A6084F31188C2
:1033F0002C2303FB0C03D3F888302BB34C2303FBA3
:103400000C00D0F8002AD36843F00103D36070BDEC
:103410007047144A24331344D4E711484C23022440
:1034200003FB0C0304FA05FED3F8006A0CEB8C03D3
:10343000F4680CEB430324EA0E042B44F46000EB25
:103440008304A166A267AEE74C2303FB0C00D0F80F
:10345000002AD36823F00103D36070BDA06D090872
:10346000181B00247C1B0024A01B002403689B0A5B
:10347000A3F58013522B00D97047144AD35C0D2B4F
:10348000FAD84FF04C0C10B4114C79B941790222A2
:103490000CFB03405DF8044B21FA02F3D0F8001A4C
:1034A0009A40CB6823EA0203CB607047417902223D
:1034B0000CFB03405DF8044B21FA02F3D0F8001A2C
:1034C00002FA03F3CA681343CB607047A06D090882
:1034D000181B002403689B0AA3F58013522B10D8F5
:1034E000084AD25C0D2A0CD84079022306494FF0D5
:1034F0004C0CD8400CFB02128340D2F8002ADB436C
:1035000013617047A06D0908181B00240149024887
:10351000FDF7E0BA7C1B002400000140014902488D
:10352000FDF7D8BA7C1B00240000014002494FF08F
:103530008040FDF7CFBA00BFA81B00240149024814
:10354000FDF7C8BAD41B002400040040014902481A
:10355000FDF7C0BA001C00240008004001490248E1
:10356000FDF7B8BA2C1C0024000C00402DE9F843EC
:10357000194E3569F3681D4010D04FF00047DFF851
:103580005C80B5FA85F227FA02F31F2A6FEA03037B
:1035900005EA0305336103D0002DF2D1BDE8F883BD
:1035A000D8F86831A3B103F1FF3900231FFA89F974
:1035B000C8F86831D8F86441002CEDD02368204663
:1035C000494698476468002CF8D1002DD9D1E5E729
:1035D000F16A1FFA81F9EDE700100040181B002482
:1035E00001490248FDF776BAB01C002400040140EE
:1035F00010B5064C064804F5CC71FDF76BFA04F5DE
:10360000F8710448BDE81040FDF764BA181B0024A7
:1036100000040140001C004001490248FDF75ABA6D
:10362000DC1C00240018004001490248FDF752BA92
:10363000341D00240020004001490248FDF74ABA29
:10364000601D00240040014001490248FDF742BAD4
:103650008C1D00240044014001490248FDF73ABA9C
:10366000B81D0024004801402DE9F0414FF42572B7
:103670008EB000217B4853F013FA7B4B7B4E4FF00A
:103680008041D3F8F02006F68415374642F0010257
:10369000DFF8E08106F66814C3F8F020D3F8F020D4
:1036A00002F001020092009AD3F8E82042F00102F1
:1036B000C3F8E820D3F8E82002F001020192019A51
:1036C000D3F8E82042F00202C3F8E820D3F8E8205B
:1036D00002F002020292029AD3F8E82042F00402B9
:1036E000C3F8E820D3F8E82002F004020392039A1A
:1036F000D3F8E82042F00802C3F8E820D3F8E82025
:1037000002F008020492049AD3F8E82042F0100272
:10371000C3F8E820D3F8E82002F010020592059AD9
:10372000D3F8E82042F02002C3F8E820D3F8E820DC
:1037300002F020020692069AD3F8F02042F002022C
:10374000C3F8F020D3F8F02002F002020792079AA3
:10375000D3F8E82042F04002C3F8E820D3F8E8208C
:1037600002F040020892089AD3F8E82042F0800262
:10377000C3F8E820D3F8E82002F080020992099A01
:10378000D3F8E82042F48072C3F8E820D3F8E820A8
:1037900002F480720A920A9AD3F8F02042F480323E
:1037A000C3F8F020D3F8F02002F480320B920B9A89
:1037B000D3F8F02042F40032C3F8F020D3F8F02020
:1037C00002F400320C920C9AD3F8F02042F48022DA
:1037D000C3F8F020D3F8F03003F480230D930D9B51
:1037E0004246002301E054F8332091420BD00133CC
:1037F000112BF8D11C3700204BF0D4FBAF420CD07A
:1038000057F81C1CECE71A4A1C3702EBC303B3F849
:10381000080D4BF0C7FBAF42F2D14FF08041154F7E
:10382000154C3A46002301E054F8332091420BD066
:103830000133112BF8D11C3600204BF0B3FBAE4204
:103840000CD056F81C1CECE7094A1C3602EBC303EB
:10385000B3F8080D4BF0A6FBAE42F2D10EB0BDE8B6
:10386000F08100BF7C1B0024004402583C71090811
:10387000A06D090800000140A47A0908800AA0F59B
:10388000801052280DD8074B1A5C0D2A09D8064B18
:103890004C2101FB0233D3F8002A136843F00103E3
:1038A00013607047A06D0908181B00241F4B984235
:1038B00010B50ED003F5806398420AD01C4A03F578
:1038C0008043984218BF904203D003F5806398422A
:1038D0001BD144F0C5F9174B1749DC69DA69C4F309
:1038E000022CC2F3022201EB0C0393F8883203F09E
:1038F0001F03D8400F4B11491B69C3F3C03342EA81
:10390000C303CB5C03FB00F010BD44F0A9F9094BE5
:103910000949DC69DA69C4F30214C2F302120B1913
:1039200093F8883203F01F03D840E3E7000001401A
:103930000040014000440258A06D09089CEC0908B1
:103940002DE9F04FB34B91B00024DFF8F0820193E2
:10395000B14BA3F68C5BB14E0025DFF8BC92B30AE5
:10396000A3F58013522B57D81BF803300D2B53D8D7
:1039700018F90370AA4B93F8863E012B40F0108192
:10398000012F3FD14FF0000A514638460FF03CFB63
:103990000FF0C2FB90F800C0BCF1000F18BFBCF1E3
:1039A000540F14BF4FF0010C4FF0000C40F0F480A6
:1039B0000AF1040A1FFA8AFABAF1100FE4D1002CB6
:1039C00000F0B580934A00210DE01BF803300D2B69
:1039D00010D818F90330BB420FD0013102F58672BE
:1039E000A14280F2A080906803689B0AA3F580132F
:1039F000522BEAD90023BB42EFD1437999F8050055
:103A00009842EAD10135082D14D059F81C6FB30A39
:103A1000A3F58013522BA7D9814B93F8863E012B37
:103A2000F0D001220027022BACD1002AAAD0013508
:103A3000082DEAD1019B013403F58673042C019310
:103A400089D1784F0026DFF8F8B1774BD3F864348A
:103A5000B34265DDD7F80C80B8F1000F60D0734B2E
:103A6000B8F804105D68D8F800003B7C002DDFF842
:103A7000D4C10193B1FA81F38444C3F11F090293C5
:103A80004FEA9C2C40F3A980624A002405E00134EF
:103A900002F58672AC4200F09D8013686345F6D152
:103AA0004FF486735B4A03FB0424019B0322C7F88F
:103AB000049001363B744FEA4903C7F80C8002FAC0
:103AC00003FCBC6188F80620012288F8076002FA2E
:103AD00003F5A36C43EA0C03A364236D2B43236516
:103AE000524B1B78002B60D0636D02FA09F943EA50
:103AF0000903636581611FFA89F1D4F8AC00FCF712
:103B0000ABFA20462037FCF77BFA0123082E0BF195
:103B1000180B07F8043C07F8033C0BF8073C94D15A
:103B200011B0BDE8F08FBCF1000F7FF46BAFD9F896
:103B3000080000223E4B04E001320C33102A00F052
:103B40002A8359688842F7D152B2304699F8051055
:103B5000FEF7D2F8374A40680023516801338842A3
:103B600017D0102B02F12402F7D14FF0FF3303EBF3
:103B7000C303314A02EB830393F87832002B7FF4BE
:103B800041AF254BC5EBC50503EB8505019B9D604A
:103B900050E7DBB2013BEAE7002C7FF413AF31E7DB
:103BA000B7F1080218BF01223DE7029D4FEA014C20
:103BB00002FA09F1C5F12F0589B202FA05F51A4694
:103BC000636D2B436365C0F818C0D4F8AC00FCF7F4
:103BD00043FA96E7032C00F3E9804FF48673134A07
:103BE00003FB05231869002800F0C1825422C3F8A2
:103BF00008C00CF1010C0E4C83F8102183F811C1A0
:103C00006B1C0A4A53600022054B93F89D3E0393B8
:103C100083681EE00C0000202C7B09080004014092
:103C2000181B00243C040020FC100020040000208D
:103C30009C0100245C02002400000024B0EC090870
:103C4000B81000200000FEA701320C34102A00F04A
:103C5000A28261688B42F7D1417952B20068FEF7C7
:103C60004BF84FF48672B14BDFF804A302FB053228
:103C7000D0E90141C2E90741002251464B680132B7
:103C80009C4217D0102A01F12401F7D1A84BA94674
:103C900093F85422002A00F05C82A648A649A74A5D
:103CA000A74BC0F8101CC0F8082CC0F8183C11B085
:103CB000BDE8F08FD2B24FF48671013A01FB05F3F3
:103CC0009B4902EBC202049301EB8202974919441B
:103CD00092F87832B1F810010593002BDDD1049CE5
:103CE000A2F87802974BA210086903FB02F2964BE8
:103CF0000068C2EBC20C02EBC20203EB4C1C03F5E2
:103D0000607303EB4212D8F80030C1F8B4C0C1F8B8
:103D1000FC203322CB60C1F8B8208C22C1F80021EE
:103D2000FFF7C4FD894B1C19039B062B00F00E8284
:103D3000072B874B874908BF1946874B874A18BF0F
:103D40001A464FF48673B0FBF2F2B0FBF1F1013A80
:103D50007648013903FB050392B2A3F8BC10A3F81F
:103D60007420226600220393A4F858206266E2655C
:103D7000049A02F1580100F1080211441A6910680E
:103D80004EF01EFC039B1A6910680392036843F00F
:103D90008003036053790C2B0DD8DFE803F06F0C20
:103DA0000C0C670C0C0C5E0C0C0C550003236C4ABD
:103DB00082F89C3E71E74FF486735C4A03FB05234F
:103DC00059694FF0600C02680023CDF820C04FF411
:103DD000807C0A9322F00102CDF838C04FF0010C2C
:103DE0000D930F930223CDF824C04FF00A0CCDE9B8
:103DF0000BC3026008AA4EF067FA4C4B4FF4867270
:103E000002FB0532039B526919680023012A3DD049
:103E1000042A3BD0102A00F0AF81402A36D0B2F5F8
:103E2000807F00F0AC81B2F5806F00F0A881B2F520
:103E3000805F00F0A981B2F5803F4FF03C030CBFDA
:103E400008224FF4006222E04FF48673374A4FF4A1
:103E5000805103FB05235961B3E74FF48673334A5E
:103E60004FF4807103FB05235961AAE74FF4867371
:103E70002E4A102103FB05235961A2E74FF48673F4
:103E80002A4A012103FB052359619AE7082201F11F
:103E9000180050F803C042EA0C02C250039B187984
:103EA000002840F03E81214B4FF4867202FB053220
:103EB00000231069D1690068026842F001020260C3
:103EC000DAF804200133914200F02781102B0AF127
:103ED000240AF5D14FF0FF33154A03EBC30302EB7D
:103EE0008303D3F85C021F4B98420CBFA020A12093
:103EF0004BF058F80D4A4FF4867303FB05231A69FB
:103F000051790C2900F20681174B03EB4103B3F8FA
:103F10006CCED2F800E04FF48673044A1349704621
:103F200003FB0523A3F818C000232AE004000020A7
:103F300000000024FC1000209DD8040899D8040833
:103F4000A5D804086B4CA407402401240C000020D1
:103F50001055220044950800D0DD060040771B0074
:103F6000181B002400000240A06D090868150020FD
:103F70005C020024904200F005810133042B00F024
:103F8000078151F83320002AF4D1844A864610462E
:103F9000D2F868240132C0F8682400EBC302DB00C9
:103FA000C2F86CE41944059823469022B1F804E065
:103FB000DFF804A24CEA0E0CA1F804C07849FDF722
:103FC00001FF4FF48673774A4FF4403E40214FF48F
:103FD000805C03FB05250023E869026842F01002BB
:103FE0000260026842F014020260C4E91F33C4E9AF
:103FF0002733C4E929334FF480632A6AC4F898E070
:10400000C4F88430A167C4F89420D5F8B820C4F867
:104010009020C2B220F0FF00103AAAFB0231EA68F9
:10402000049B1832C4F888C04FF4804C09092267F9
:1040300003F170025C4B1A44D5F8B430C4F88CC05C
:1040400063674EF051FCE869049B4FF40031D0F8EF
:1040500000E04FF4006C03F1B802534BC4F820E0C9
:10406000D0F814E01A440023C4F824E0D0F804E0A7
:10407000C4F828E0D0F808E0C4F82CE0D0F80CE050
:10408000C4F8C830C4F830E0C4E93033C4E9393387
:10409000C4E93B332B6AC4F8E01003934FF4806308
:1040A000C4F8CC30039BC4F8DC30D5F80031C4F838
:1040B000D830C3B220F0FF00103BAAFB0331EB68FD
:1040C000C4F8D0C010330909C4F8B830D5F8FC30B2
:1040D00003934FF48043C4F8D430039BC4F8BC303E
:1040E0004EF002FCEB69B8F804101A68D8F800002A
:1040F00062635A69A2635A68E2639A682264DA6862
:1041000062641A6842F010021A601A6842F01402DF
:104110001A60CAE44FF0000CFBE6DBB20593013BEA
:10412000DAE607910BF080FC0799069048B1039BF3
:104130000221DA79FDF7B0FE069B5422DA80039B58
:1041400019684B6C43F400434B64ACE61749184ABA
:10415000F7E5144A4FF4867808FB092898F81111FE
:1041600098F8102183F8551283F8542295E502231C
:10417000104A82F89C3E90E54FF4006287E60822E0
:10418000042384E6DB000DE74FF4006204237EE69F
:1041900000239B88FFDE00235B68FFDEFC1000200D
:1041A00001000000040000200C000020882A1100FB
:1041B000A0BB0D00181B0024ABAAAAAA2DE9F04F42
:1041C00000228FB02F2107460EF0FEFFD0B1B04C79
:1041D00006464379D0F80080A4F83834FDF7BAFDDC
:1041E00080B1456875B1DFF8E0B2002259464B68EE
:1041F000013224319D4210D0102AF8D1A54B93F8FA
:1042000054221AB100200FB0BDE8F08F2F211046C4
:1042100083F8552283F85412F5E7D2B2DFF874A27E
:10422000013A02EBC2020AEB820292F87892B9F1EB
:10423000000FE7D12F2183684046C4F8EC83A2F831
:1042400078120393FFF732FB934A904280F0FF808D
:1042500001234A46029340460192FFF727FB029B47
:10426000019A8E49C4F8F023B0FBF3F2120A002041
:10427000A1FB02328A4BC4F8FC031109C4F8F40311
:104280001209A3FB0131C4F8F8234A08A4F8A02EB0
:104290005200A4F89E2E94F8292402F0FF01002A6F
:1042A00000F0E38002227F49D4F8EC0384F829244B
:1042B00043F0DEFF0122384684F8342484F82A24AF
:1042C00084F82B2484F82C2484F82D2484F82E24BC
:1042D00084F82F2484F8302484F8312484F832249C
:1042E00084F8332484F829240BF09EFBC4F8A40E30
:1042F00028B12F21C1804E21F279FDF7CDFD6A4A08
:104300000021039BC4F8B41EC4F8AC3EC4F8C41E1C
:10431000C4F8CC1EC4F8D41EC4F8D81ED2F8D800F5
:10432000C4F8A85E40F00100C2F8D800D2F8D80066
:1043300000F0010005900598D2F8D80040F0020086
:10434000C2F8D800D2F8D82002F002020692069AEB
:104350004022C4F8B02E4FF48062C4F8B82E4FF457
:104360008052C4F8BC2E4FF48042C4F8C02E4FF4E3
:104370000032C4F8C82E0322C4F8D02E94F8382492
:104380000C2A75D8494901EB4202B2F8887EB8463A
:10439000083747485946002204EB870CCCF8EC0359
:1043A000A0F6BC20C4F8E00E4868013224318542F2
:1043B00064D0102AF8D14FF0FF3202EBC2020AEBB0
:1043C000820A3C4ADAF85C0290420CBFA020A1208D
:1043D0004AF0E8FD0022DBF8041001320BF1240B57
:1043E0008D4248D0102AF6D104EB87074846434651
:1043F00060223149FDF7E6FCD7F8EC033FF074FB8F
:1044000000287FF4FFAE60210C90B379079159002A
:104410000D90DB00089001F002010B9003F00803FF
:10442000B4F838242548CDE9091307A94AF070F8F3
:1044300000287FF4E7AEB379B4F838149B071F481F
:104440001FD544F035F8B0FA80F04009DBE640466D
:10445000FFF72CFA1A4A1B490244A1FB0232920DC3
:10446000013A92B2531C0293F5E684F8281419E736
:1044700088460F468CE75FFA82F9B5E7D2B2013A77
:104480009BE743F06BFEB0FA80F04009BBE600BF4B
:10449000181B002400000024006CDC02598B4F0123
:1044A000ABAAAAAA081F002400440258A06D09085C
:1044B000C0290024000002409D010000041F0024C8
:1044C00000366E01819F5E165C020024830AA3F50C
:1044D0008013522B00D970472DE9F04115460F4A41
:1044E000D65C0D2E17D80E4C4FF04C08013908FB46
:1044F000064789B2C7F80C1AFFF7D8F907F6042166
:10450000B0FBF5F2013AD7F8000AC7F8042ABDE873
:10451000F04143F0ADBEBDE8F08100BFA06D0908D9
:10452000181B0024830AA3F58013522B6BD82DE9A6
:10453000F0411646794A84B0D75C0D2F60D8DFF879
:1045400004824C25044605FB0785D5F8003A8342D2
:1045500056D00139C5F8000A89B2C5F80C1AFFF720
:10456000A5F90023B0FBF6F2C5F8103A013AC5F8F8
:10457000083AC5F8143A95F83D3AC5F8042A03F00C
:10458000FF02002B40D04C23654903FB078503FB4A
:1045900007110223D5F8000A85F83D3A043143F0AB
:1045A00067FE012385F8483A85F83E3A85F83F3A98
:1045B00085F8403A85F8413A85F8423A85F8433A19
:1045C00085F8443A85F8453A85F8463A85F8473AF9
:1045D00085F83D3A534B9C4219D0B4F1804F16D028
:1045E000A3F57C439C4212D003F580639C420ED01D
:1045F00003F580639C426CD003F578439C4268D0FD
:1046000004B0BDE8F081704785F83C2ABBE74C2335
:104610004FF48051002203FB0783009193F83C1A6A
:1046200003920129CDE90122EAD00221D3F8000A40
:10463000012483F83D1A3C4985682940816083F84C
:104640003D4A83F83C2A4C22002302FB0782029356
:10465000CDE9003392F83C3A012BD1D0D2F8003AA0
:104660000221304882F83D1A83425A6899682CD05A
:1046700000F58060834228D022F070022B485A60F7
:104680002B4A934218BFB3F1804F0CBF0122002286
:10469000834208BF42F0010200F58060834208BFF8
:1046A00042F0010212B9234A934202D121F0800163
:1046B00099604C230121002203FB078787F83D1AEC
:1046C00087F83C2A04B0BDE8F0811B4810405860D0
:1046D000ECE700214FF48053CDE900314C2303FB7C
:1046E000078393F83C2A012ACDE9021188D0D3F838
:1046F000000A022283F83D2A0B4A85682A4082601C
:104700000E4A83F83C1A0121944283F83D1A9AD04C
:104710000B4B9C427FF474AF95E700BFA06D090876
:1047200018250024000001408800CEFF000800404A
:1047300000040040001800408FFF0FFF00040140FC
:10474000000C0040181B00242DE9F04F05460868B6
:1047500089B00C464FEA902CBDF84880ACF5801C1F
:104760009DF84CA0BCF1520F69D8DFF8EC9019F815
:104770000C700D2F63D807EBC706DFF8E0B01946C1
:1047800007EB4606FFF7CEFE23680BEB8606617942
:10479000A279BAF1000F55D194469B0AA3F5801374
:1047A000522B25D819F803000D2821D800EBC0039F
:1047B0000A4601A9CDF8088000EB43004FEA4C03FC
:1047C0004FEACC0C03F002030BEB800003930CF0D8
:1047D00008034FF4807C0493602301934FF400732B
:1047E000CDE906C30023059349F092FE6179A279D1
:1047F0009307304629D543F05BFE154B4C2202FB54
:10480000073797F83D3A012B10D10223D7F8002A39
:1048100087F83D3A0F4B91680B40062B06D0B3F555
:10482000803F03D0136843F001031360216863796C
:1048300001F1340269600021D0182860D15009B01C
:10484000BDE8F08F82F0010CA7E743F087FCD4E7C6
:10485000181B002407000100A06D0908182500247A
:1048600070B504460068830AA3F58013522B03D861
:104870002B4DEE5C0D2E00D970BDFFF753FE294B7A
:104880004C2202FB063696F83D3A012B13D02168E4
:104890000023254A254801E050F8332091421CD0DE
:1048A0000133112BF8D1012100204AF0F9FA204BF5
:1048B00001221A6070BD0223D6F8002A86F83D3A1C
:1048C0001C4B91680B40062BE1D0B3F5803FDED046
:1048D000136843F001031360D9E705EBC30301211B
:1048E000134D93F80A4D20464AF0DAFA04F01F03FC
:1048F000012162091B2C01FA03F345F8223006D18D
:1049000019204AF0CDFA4FF000732B6070BD2E2CA9
:10491000B2D12C204AF0C4FA4FF480536B6070BDC2
:10492000A06D0908181B002400000140A47A0908A2
:1049300000E100E00700010038B5264C94F8203F64
:10494000012B12D1042894BF002301236BB904EB7F
:1049500040000D4694F8381FC4F84C3FB4F83A2F85
:10496000B0F8423FB4F83E0F01B138BD07EE902ACF
:10497000D4F8302F9FED180AB8EEE77ADFED177AFA
:1049800027EE277A07EE902A6422F8EE676A02FB88
:1049900003F307EE903A02FB003366EE806AB8EE4E
:1049A000E76A07EE903AF8EEE77A27EE067A87EEA6
:1049B000270A20EE260A51F081FAD4F8282FB4F8FD
:1049C0003C3F1060D4F8381319442944C4F8501FF0
:1049D00038BD00BF181B0024CA269B3E0AD7233CC3
:1049E0002DE9F043BDB0BFF35F8FA34A0020516AA9
:1049F0000346044621F4803151620146C2F8940016
:104A0000C2F898300133C2F89C10112BC2F8A010E4
:104A1000F6D10523C2F89430536A43F480335362CD
:104A2000BFF34F8FBFF36F8F9448954A9549121A81
:104A300051F0C2FF9448954A9549121A51F0BCFFB3
:104A4000944AD368042B00F0FD8005D8012B00F0B8
:104A50008183022B00F07783874A00238E4C01204C
:104A6000D2F888108D4E41F470018D4DC2F8881037
:104A700020602361216841F08001216021680143A9
:104A80002160216841F480312160216841F4805126
:104A90002160A361E3612362A362E3622363636332
:104AA000A363E36323646364216821F480212160AC
:104AB0007C492366C1F808014FF000614FF6FF0002
:104AC000794B9160D16801400B43D36043F0A6F865
:104AD000A36902460F20C3F30323A169334493F86B
:104AE000883203F01F0322FA03F3C5F8EC343EF0DA
:104AF00005FB6E4AD36813F0040FD36840F0A4801E
:104B00006B4B0021694A0391D96A21F00101D962F6
:104B1000DB6A03F001030393936943F44043936119
:104B2000936903F440430393039B93699B04FCD56F
:104B30004C2200210DA85F4C51F0B2FF5E4A42F2B8
:104B400003031268B3EB124F4FF00003079304F115
:104B5000140318BF1C46E268002A4FD0544B534937
:104B6000D86A20F00100D862DB6A03F001030793E2
:104B70008B6923F4404313438B618B6903F44043F7
:104B80000793079B494A93699F04FCD5424B4FF416
:104B900040314A484FF00108D3F8E020002742F0A6
:104BA0008002C3F8E020D3F8E03003F080030693DE
:104BB000069B0323816108A908930B93CDE909871C
:104BC00042F072FB02230DA8CDF834801E97CDE988
:104BD0001633A3781893A3881993A3791A93E379CA
:104BE0001B93237A1C9323691D934FF480330E93F8
:104BF00042F056FD03283BD098B1FEE72B4A2C4BE0
:104C0000916941F440419161926902F440420792F6
:104C1000DA6A42F00102DA62DB6A03F00103079309
:104C2000AFE7274B1A6812F00E0F4DD11A6822F029
:104C30000F0242F002021A601B6803F00F03022BFE
:104C400042D0FEE7D46007E723F007031D4C43F092
:104C50000203D360D4F8541F06E0D4F8543F5B1A23
:104C6000B3F57A7F3FF64CAF53689804F5D547E724
:104C700072B6FEF7E5FA00BF00ED00E000000000AC
:104C8000483C00000C790A080000002004000020C5
:104C9000B5DA0A085040005800440258A06D0908CF
:104CA00000000024008000510003FA05004802586B
:104CB00000040058C40400240010005C001C0258CA
:104CC00000200052181B00246E4A936903F0700301
:104CD0003F2B05D8936923F0700343F040039361A1
:104CE000684AD36903F070033F2B05D8D36923F0DA
:104CF000700343F04003D361624AD36903F4E06375
:104D0000B3F5806F05D2D36923F4E06343F4806385
:104D1000D3615C4A136A03F070033F2B05D8136A12
:104D200023F0700343F040031362564B9A69140753
:104D300005D49A6922F00F0242F008029A61514AA2
:104D4000936923F470639361136898017FF579AFD9
:104D5000136941F288304C4C23F0070343F00303FE
:104D60001361D4F8541F05E0D4F8543F5B1A834212
:104D700000F2A181136903F03803182BF4D1936971
:104D800003F00F03082B05D9936923F00F0343F0B9
:104D9000080393613D4A136803F00F03022B0BD9FC
:104DA000136823F00F0343F002031360136803F04A
:104DB0000F03022B7FF445AF324A936903F070036F
:104DC000402B05D9936923F0700343F040039361AE
:104DD0002C4AD36903F07003402B05D9D36923F023
:104DE000700343F04003D361264AD36903F4E063C0
:104DF000B3F5806F05D9D36923F4E06343F480638E
:104E0000D361204A136A03F07003402B00F24B81F8
:104E10001C4F42F003FF0346D5F8F004BA69B969A4
:104E2000C2F30322164496F8882202F01F02D340F0
:104E3000C5F8EC343EF062F9002840F03D811023C3
:104E4000149016900DA80D9342F02AFC002840F013
:104E500029813B680E4943F080033B60D7F8F4306A
:104E600043F00203C7F8F430D7F8F43003F002033C
:104E70000293029B0A6A074B42F001020A62D4F8CD
:104E8000541F0CE000440258181B0024002000525C
:104E90000004005800E20400013B3FF4E9AED4F8FE
:104EA000542F9142F8D0D4F8542FD4F8543F9B1A81
:104EB0000A2BFAD94FF48023B14C0DA84FF000080B
:104EC0000D934FF44013032602272E934DF088FED6
:104ED000D4F8EC300DA843F00203C4F8EC30D4F859
:104EE000EC3003F002030193019BD4F8943043F0BB
:104EF0000203C4F89430D4F8943023F00203C4F8C9
:104F00009430A04B1A6841F20303B3EB124F9E4B4F
:104F10009E4A38BF1A469E4B5A601A6822F47C5249
:104F200042F400521A601A6842F060021A600D964C
:104F3000CDE92A884DF054FE4FF4E0430DA8CDF89A
:104F4000E0800D93CDE924884DF04AFE18230DA88A
:104F5000CDF8B4800D93CDF8C8804DF041FE4FF4EC
:104F600000230DA80D934FF4003335934DF038FE18
:104F7000D4F8E03008A9874843F00103C4F8E030D2
:104F8000D4F8E030CDF8308003F001030593059BA1
:104F90004FF48073CDE90A86CDE9083742F084F9F1
:104FA000236908A97C4823F0FE7343F088732361CA
:104FB000D4F8E03043F00403C4F8E030D4F8E03033
:104FC000099703F004030B96CDF8288004934FF45F
:104FD0000073049A0893CDF8308042F065F9236994
:104FE00023F07E4343F0FC43236142F017FE6B4BFA
:104FF0006B4A4146C5F8EC041846D21A51F050FDF0
:105000006848694A6949121A51F0D6FCBFF35F8FAC
:10501000674D4646674C01276B6A23F480336B6209
:10502000C5F8948023E0002A44D0D4F80080637A45
:10503000103414F8061C1B0643EA017343EA4203CA
:1050400014F8052C43EA824314F8042C43EA424343
:1050500014F8032CC5F89860013643EA0243C5F8FA
:105060009C80032E43F00103C5F8A03025D063686F
:10507000227A002BD7D0D4F80080002AD7D128F08C
:105080001F09A3EB0903202B38BF2023184699469C
:1050900051F08CFC431E07FA03F2914518BF0346FA
:1050A000DAB2C4E7FEE7136A23F0700343F040036B
:1050B0001362ADE6FEE7C4E5C3E50523C5F8943009
:1050C0006B6A43F480336B62BFF34F8FBFF36F8F14
:1050D000BFF34F8FBFF36F8F0022C5F85022BFF38D
:1050E0004F8FBFF36F8F6B6943F400336B61BFF376
:1050F0004F8FBFF36F8FC5F88420BFF34F8FD5F864
:10510000805043F6E0762A49C5F34E34C5F3C9050D
:10511000640104EA06002B4640EA8372013BC1F8B1
:105120006022F9D2203C14F1200FF2D1BFF34F8F4F
:105130004B6943F480334B61BFF34F8FBFF36F8FE5
:105140003DB0BDE8F08304210320FDF757FA72B6A5
:10515000FEF776F802200A4B1749D060D3F8F42006
:105160000243C3F8F420D3F8F43003400D930D9AB2
:10517000D1F8003883F30888D1F804389847FEE75F
:10518000004402580010005C7FBB22307FBB22002D
:10519000008400400000025800080258C0E10024CA
:1051A00060E20024E0DC0024C0E10024B9DA0A084F
:1051B00000ED00E0F40400240090F01F0548D0F852
:1051C000043323B1DB6A13B100F54170184702487C
:1051D000704700BF181B0024447C090830B5114CEF
:1051E0004FF0000C234693F800E00633864515D0B7
:1051F0000CF1010CBCF1060FF5D10B4DD5F87C3F3D
:10520000052B0AD00CFB034C0133C5F87C3F8CF80E
:105210000000ACF80210ACF8042030BD062303FBFC
:105220000C4CF4E7702A0024181B002410B5174C0E
:10523000D4F8803F1B883BB9002384F8883F84F86A
:10524000FC32C4F8F83210BDD4F87C2F002AF3DD0C
:10525000012A08D0D4F8843F59880123A4F88A1F72
:1052600084F88C3FE8E7D4F8841F8A8849880132A3
:10527000521A9A42F1D10022D4F8043304F5417055
:105280001B69C4F830239847D6E700BF181B0024D9
:105290000748D0F8003313B190F88C3F0BB10020D1
:1052A0007047D0F8043300F541705B68184700BFC1
:1052B000181B0024174B10B4174C93F8FC222244FF
:1052C000C0E9002493F8FC0293F8882F824217D893
:1052D00093F8FC02824206D300235DF8044B184683
:1052E000C1E90033704793F8FC32002A5DF8044BA3
:1052F000C3F180030CBF012002204A600B6070479D
:1053000093F8FC4200230120121B5DF8044BC1E915
:1053100000237047181B0024C0E100240F4B93F8B2
:10532000FC2293F8880F93F8FC22904293F8FC2219
:105330000FD8904204D3D3F8F832002018447047B5
:1053400093F8FC22D3F8F832C2F1800210441844DA
:105350007047801AD3F8F83218447047181B00249D
:1053600010B51B4C84B01B4B94F8FC2203931344E0
:1053700094F8881F029394F8FC32994294F8FC3216
:1053800014D899420AD294F8FC320191C3F18003F7
:105390000093C9B901223F2B0ED868B994F8FC02DA
:1053A000401AB0FA80F0400904B010BD0022CB1AB8
:1053B000019201220093EEE76946002302A84EF015
:1053C00043FF94F8881FE9E70B440222E3E700BF9C
:1053D000181B0024C0E100242DE9F043164685B0D7
:1053E00000293BD0451E284CDFF8A4804FF000096F
:1053F0006F180DE094F8FC3208468B4294F8FC32AA
:105400001CD9C3F1800318443F281AD8AF4225D0D5
:1054100094F8880F15F8013F411C08F80030C9B214
:105420000B0684F8881FE5D5002094F8FC3284F838
:10543000889F01468B4294F8FC32E2D8C01A3F287C
:10544000E4D994F8FC328B42E0D0104B1B78002B4F
:10545000DCD00020FFF784FFAF42D9D1694602A813
:10546000FFF728FFDDE9003213443F2B00D910B9C4
:1054700005B0BDE8F0830246334602A84EF0E4FED4
:1054800005B0BDE8F08300BF181B00240000002415
:10549000C0E1002430B585B0694602A8FFF70AFFD5
:1054A00058B9094C04F54175D4F8043328465B68B3
:1054B00098470028F8D005B030BD0246012302A865
:1054C0004EF0C2FEEDE700BF181B002470B5114C72
:1054D00016460A4682B0D4F800338119054699422F
:1054E00094F8881F88BF1E1A94F8FC32994203D0A2
:1054F0000192FFF7CFFF019A002033462946C4F8F6
:105500003003D4F80403846A0348A44602B0BDE81B
:1055100070406047181B00241C1E00248C46134654
:10552000014662461846D1E738B5244C002204F6FD
:1055300058701346C4F80023024611780632022937
:105540002BD00133062BF8D10022D4F80433C4F851
:10555000842FF3B1DA6AE2B119489047D4F8843F56
:10556000C4F8800FA3B159889A884368521A02FB85
:105570000333C4F80033FAF761FF94F8FC320546B0
:1055800094F8882F9A4201D0FFF784FFC4F8F852AC
:1055900038BD0C4BC4F8803F38BD03EB4303D4F84F
:1055A000042300EB4303C4F8843F12B1D26A002AFB
:1055B000D2D1044A1046C4F8802FD4E7181B002427
:1055C0001C1E0024447C090810B50A4CD4F804338E
:1055D0005B6A13B104F541709847D4F8F832D4F8F7
:1055E000802F013B5288134452421340C4F8F832D2
:1055F00010BD00BF181B00242DE9F043384E93B0B6
:10560000FFF714FEFFF790FF96F8FC3296F8882F0C
:105610009A4201D0FFF73EFF0025D6F80073C6F886
:10562000F85297B16C46DFF8BC802A4641462046C6
:10563000203501F0FDFE20464EF046FF01220146D6
:105640002046FFF7C9FEAF42EFD896F8FC3296F835
:10565000882F9A4201D0FFF71DFFD6F8803F9B7B31
:10566000012B36D096F8FC3296F8882F9A4201D05A
:10567000FFF710FF0020C6F8F8026FB380466C46B3
:10568000DFF86090054601E0AF421CD92A46494642
:1056900009A801F0CDFE21220021204651F000FA98
:1056A000202221462846FFF711FF2022064609A99D
:1056B0002046203551F021FB08B9202EE4D0AF421E
:1056C00008F10108E2D8B8FA88F0400913B0BDE843
:1056D000F083FFF779FFC5E7012013B0BDE8F08341
:1056E000181B00241CEC0908F0B583B044F0E0FF5F
:1056F000214B292203F58054A3F8DE26A3F8E626E1
:10570000D4F8482212B10022C4F84822D4F850221A
:1057100012B10022C4F85022184E0027012506F2CB
:10572000245283F8907F84F82C52C4F844224BF022
:10573000ABFC06F5A8630DF10600ADF80670C4F8E1
:105740004832D6F86C3598470D4BC4F8500293F8A0
:105750007D31AB4202D0284603B0F0BD06F5AF66FE
:10576000D4F86C02C4F868624DF01AFF054B384655
:1057700083F82370F0E700BF181B0024000000240A
:10578000102C002400ED00E00A4B93F8980518B99E
:10579000094B93F880017047084AD1680329F7D173
:1057A00005494FF0010C81F880C10021D16083F8D8
:1057B0009815704700000024102C00245040005819
:1057C0000321044608B50846FCF718FF72B6104BD3
:1057D000D3E9620350EA03020AD1002211460420F1
:1057E000FCF70CFF11460520FCF708FFFDF728FD2C
:1057F000084A21B24EF66024D2F8382304FB01F1A6
:10580000121843F100038A1843EBE171E7E700BF88
:10581000102C0024181B00240021032008B5FCF7DD
:10582000EDFE72B6FDF70CFD184CD4F8902194F8FB
:10583000960108B54AB11168938809690B40F8B917
:10584000003B18BF0123002BF4D114200CF0F6FC10
:1058500000BFD4F8903163B1196894F896219B8801
:1058600009690B4042B9003B18BF01230BB1FFF798
:10587000D3FFFAF715FEEBE7B3FA83F35B09F5E71D
:10588000B3FA83F35B09002BD4D1DEE7102C00249C
:105890002DE9F04F00218BB041F69462BD4851F0E4
:1058A000FFF80420FCF7A4FE01460520FCF7A0FE4B
:1058B00051EA000340F05E81B74B03934C22002174
:1058C000B448012451F0ECF800214C22B14851F0C9
:1058D000E7F8039BAF4AD3F8CC35B04D147115608F
:1058E0005362C2E907334BF099FAFFF71DFE00211E
:1058F00008460AF029F9FAF7A1FDB0F1000B40F3D0
:105900000981A44B0024A64D03F14C0AA54B274660
:10591000A04605F5CC79A44ECDE9013404E008F5A4
:105920000068C34540F3AC80019AD2F83833C2F81E
:105930003C33FAF7B5FD202249464046FFF7C6FD45
:1059400012229A49484651F0D8F90028E7D1474534
:1059500021D0029B5A1C03EB4301954B029203EBAF
:10596000810394491846049301F062FD5246049B5A
:1059700042F84C3BDAF81C30CAF80C70A8EB070769
:10598000CAE908330123CAF808308B4BCAE9047707
:10599000CAF828309246039B47461222D3F8CC35EA
:1059A000CAF81C30A918335D013291F89811994258
:1059B0000BD00024202AF5D120374946BB45384674
:1059C00054DBFFF783FD0022ECE70134152CF1D105
:1059D000D0197A492022FFF779FD00230A2209A96C
:1059E0007648CDF8249001F0BDFE074609980023C3
:1059F0000A22013009A9099001F0B4FE07900023A2
:105A000009980A2209A90130099001F0ABFE06901D
:105A1000002309980A2209A90130099001F0A2FE89
:105A2000059009A9099800230A220130099001F084
:105A300099FE0490002309980A2219460130099022
:105A400001F090FE97B1DDE9063243EA4211049B72
:105A50005A01059B42EAC32242EA6003A7F2BC72E4
:105A600041EA422243EA0243CAF81C30029B642BFB
:105A700000F0F380474608F50068C3453FF754AF90
:105A8000029A642A00F0E280B84500F0DF800C231F
:105A9000474DA8EB070602F1010803FB02554549F3
:105AA0004246454C284601F0C3FC029ADAF81C3005
:105AB000CAF80050951CCAF80C70CDF80880CAF8D6
:105AC0002840CAE908330123CAE90466CAF8083045
:105AD0004C22304B00213A4F02FB05F501262B44A6
:105AE000184650F0DDFF4C22002150F0D9FF294A22
:105AF0005751039A8462029CD2F8CC250234866006
:105B00004262C0E904BBC0E907224FEA4B03B3F18C
:105B1000805F1EDA4C221F4B00212A4F02FB04F447
:105B2000012502262344184650F0BAFF4C220021DA
:105B300050F0B6FF174A03991751CBF10062D1F824
:105B4000CC15AA40467185604162C0E90711C0E9E1
:105B50000422104B9D6835B91A461B791BB1136896
:105B6000002B40F08380002108460BB0BDE8F04FC9
:105B700009F0EABF4FF47A7200234FF069F9124B33
:105B800040F26D11022440F2B2720D46B0FBF3F305
:105B900024E000BF2033002400000024ACEC0908FE
:105BA000102C0024181B002460EC09083CEC0908A8
:105BB000C82D002450EC09081D550408A82D002408
:105BC00078EC090888EC09088051010001325B1A61
:105BD00012F003040CBF4FF4B77129469942F5DD6A
:105BE0007449002C3CD003910399D1F89C1599423B
:105BF0006FDC714D01245B1A55F8041F0134994282
:105C0000F9DD0133A2F2BC72039D43EA44133C2444
:105C100043EA4223694AB0FBF2F102FB11024FF45E
:105C20006160B2FBF0F100FB11221C20C5F8A00559
:105C3000B2FBF4F004FB1022521042EA401242EA96
:105C4000C12242EA0343C5F8CC3537E6029B012462
:105C50005D1C002B3FF459AF00E06525584C37E739
:105C60000C4603911D21C4F8A015BDE729462E4618
:105C70001564D563C2E91155D46C02F14C0354B3D9
:105C80009C68481E1E648442DE63C3E9116612D01C
:105C9000481C844216D08C427FF465AF0846002829
:105CA0003FF461AF116CCC6B0134CC631964936425
:105CB00001461A46E0E700293FF455AF884253F801
:105CC0000C2CECD1117900293FF44DAF53641A64C8
:105CD000EEE7012495E73B490222264611E0CB6B13
:105CE0000A635B01C1E9046657D003F6FF77531ED0
:105CF00003EB17335A1C0135C1E90D3351F84C0F32
:105D0000C8B10B79002BEAD108690A63002848D191
:105D1000531E10464F694863002F40D007F6FF77A7
:105D200003EB1733201A8B635A1C0135C41851F842
:105D30004C0F0028E5D124483E22013BC0F88043A7
:105D40003F24C0F868234022990F0190C0F88C537B
:105D5000C0F87C33C0E9DB421C4AC0F864239A00D7
:105D60002BB340F2FF10121841F10001520A42EA2F
:105D7000C15202F140010198124C0A44C0F8741358
:105D800002EBC303C0F878235902C0F86033DA0D80
:105D9000C0E9E144C0E9D612E5E61346AAE7134696
:105DA000C0E700F6FF70531E03EB1030B2E701228C
:105DB000DFE700BF000000249C05002480510100A3
:105DC0001D55040820330024181B002494EC0908F6
:105DD000012243F2013C40F2011100230273A0F8BA
:105DE00000C043F2012C418040F6011102720A22E8
:105DF000A0F806C0C381038243828182827500B508
:105E000040F2351EA0F804E05DF804FBFF220346D3
:105E100000F11E01F0B5DA70053303F8012C8B4256
:105E2000F9D1124B4FF0FF3C1726162503F11E0740
:105E300064464FF0150E00220AE093F9062006335F
:105E400093F801E09D78DE7893F9044093F905C05A
:105E500002EB82029F4200EB020100F802E04D706B
:105E60008E70CC7081F804C0E7D1F0BDC87C090801
:105E70004FF0000C01210222032380F805C081713C
:105E8000C2710372704700BF002302220370437087
:105E90008370C370027170474FF4F07140F22E4C62
:105EA0000023072201804FF47A71A0F81EC04FF43E
:105EB000FA6C41844FF4F5614371A0F820C040F2C0
:105EC000012C8371438242F22453818442F22011D7
:105ED000A0F814C040F2034C018144F64C514381B8
:105EE00043F63813A0F816C040F2056C81810E21EC
:105EF000C38102238270A0F818C080F82610827631
:105F0000437400B540F2262EA0F81CE05DF804FBB7
:105F10008388C3F30B039342A8BF134670B51D4695
:105F20000C461A460646806850F046FD6219084B3A
:105F30009442B56908D0074814F8011B00FB03F32D
:105F4000A24283EA0103F7D101202B6070BD00BF9C
:105F5000C59D1C8193010001002303704370837071
:105F6000C37070470023037043708370C370704721
:105F700000220123027042708270C270037143716B
:105F80008371C371704700BFFF2303704370837038
:105F9000C3707047002306214FF47A7201700373B7
:105FA000C0E90123704700BF0023FF22411C10B548
:105FB00000F8132001F8132001330B2BF8D10C4B00
:105FC0004FF0FF31002203F11B048C4605E013F96A
:105FD00002CC13F9011C13F8032C033300EB420E1F
:105FE00000F812C09C428EF80110F0D110BD00BF25
:105FF000EF7C09084FF0180C00210123022280F8E1
:1060000000C04FF00E0C417180F802C04FF0130C2D
:10601000017221214370037180F803C04FF0240CFA
:1060200041720421C37243730374C37483750723DD
:1060300080F80CC04FF0250C81730521C3753823FF
:1060400080F80FC04FF04C0C4174062103760323F7
:1060500080F812C04FF04D0C017539214377202391
:10606000C271827280F815C042768276C17602775C
:10607000837170474FF0FF320023026042608260FC
:10608000C260027403708370C3700371C371704780
:1060900003230370704700BF0A4491421AD001F1F4
:1060A000FF3C41F2210100B502F1FF3E1CF8012F37
:1060B000082380EA022010F4004F4FEA400281EAF0
:1060C00040000CBF90B280B2013BF4D1E645EDD167
:1060D0005DF804FB704700BF704700BFDFED277A13
:1060E000B4EEE70AF1EE10FA0CDDDFED256A9FED64
:1060F000257AF0EE407A30EE660AF4EEC77AF1EED9
:1061000010FAF6DCDFED207AB4EEE70AF1EE10FAD1
:106110000CD5DFED1B6A9FED1D7AF0EE407A30EE74
:10612000260AF4EEC77AF1EE10FAF6D4DFED187A0B
:10613000B4EEE70AF1EE10FA14DDDFED107A37EE77
:10614000C00A60EE006A9FED136A9FED137ADFEDDF
:10615000137AA6EE867A20EE266AE6EE877AA6EE17
:10616000270A7047DFED0E7AB4EEE70AF1EE10FA77
:10617000E7D5DFED057A37EEC00AE2E7DB0F4940ED
:10618000DB0FC940E4CB1641DB0F49C0E4CB16C19D
:10619000DB0FC93F92E741B99730083C15A82ABEEA
:1061A000DB0FC9BF2DE9F047089F002B0E460546BF
:1061B0003C4614BF4FF030094FF0200914F8011B82
:1061C00041B3002A2CDD234600E0B2B113F8010BE5
:1061D0009046013A0028F8D1A8F102086AB1C246F7
:1061E00049462846B04753460AF1FF3A002BF7DCF0
:1061F00028EAE8723978013249B1D71B2846B047FE
:10620000E01914F8011B0029F8D1BDE8F087104609
:10621000BDE8F087002A02F1FF38E0DC0846F4E729
:106220000022EAE703685A1C02601970704700BF39
:10623000024B186803681B68184700BFB851002458
:10624000884230B54FF001043AD301FB04F4B0FBAF
:10625000F4FC8C45F9D2BCB102BB06E0A14203F8C4
:10626000015B11D81446B0FBF2FCBCF1090F0CF134
:1062700057050CF1300E04FB1C00B4FBF1F2EDDC11
:10628000A14203F801EBEDD900221A7030BDA14202
:1062900003F8015BF8D81446B0FBF2FCBCF1090F1F
:1062A0000CF137050CF1300E04FB1C00B4FBF1F2CD
:1062B000EDDCA14203F801EBEDD900221A7030BDEC
:1062C0008446002AEAD1D0E7002870B503DA2D23EE
:1062D000404201F8013B092886464FF0010307DDE3
:1062E00003EB83035B00B0FBF3F2092AF8D8A3B1F8
:1062F0000F4CA4FB0320BEFBF3FCBCF1090F4FEADB
:10630000D0000CF130060CF1570503FB1CEE07D84A
:10631000092B01F8016B0346EBD800230B7070BD0D
:10632000092B01F8015B0346E3D800230B7070BD15
:10633000CDCCCCCC0378092B01D0202B05D110F883
:10634000013F202BFBD0092BF9D02D2B00F0A98089
:106350002B2B75D0B7EE000AA3F13002D1B2092978
:1063600077D8F2EE046ADFED5F7A07EE102A10F8B4
:10637000013FB8EEC77AA3F13002D1B2A7EEA67AF8
:106380000929F0EE477AF0D92E2B66D003F0DF030F
:10639000452B40F0838010B442782D2A00F096807F
:1063A0002B2A00F08380A2F130030130092B00F288
:1063B00084800024002303EB830302EB430310F8E3
:1063C000012FA2F13001303B0929F4D9B3F59A7FAE
:1063D0001A46B7EE007A28BF4FF49A72072B09D9F4
:1063E0001346DFED416A083B27EE267A072BFAD8E1
:1063F00002F00702DAB1F2EE046A012A27EE267AE9
:1064000015D0022A27EE267A11D0032A27EE267A03
:106410000DD0042A27EE267A09D0053A27EE267AEF
:1064200005D027EE267A012A18BF27EE267A002CFF
:1064300045D0C7EE877A5DF8044B20EE270A7047F7
:106440004378B7EE000A0130A3F13002D1B2092936
:1064500087D92E2BDFED237A98D143780130A3F131
:106460003002D1B2092991D8B2EE047AF0EE475A3F
:1064700006EE902A10F8013FB8EEE66AA3F130026A
:10648000D1B2C6EE076A092927EE257A77EEA67AF9
:10649000EED903F0DF03452B3FF47DAF20EE270A52
:1064A00070474378BFEE000A013055E7827802302A
:1064B000A2F13003092B7FF67CAFB7EE007A67EECE
:1064C000877A5DF8044B20EE270A70478278023005
:1064D000A2F13003092B01D801246BE7B7EE007A53
:1064E000A7E700BF0000000020BCBE4CF8B5164D69
:1064F0006B78BE2B25D1AC1C144F022229464FF6D7
:10650000FF70FFF7C9FD22884AB1A618BE4218D213
:10651000052A16D921463446FFF7BEFDF3E721468A
:106520000222FFF7B9FD0222A1180634FFF7B4FDDD
:10653000074B641B9C8041F60F53C31A58425841C5
:10654000F8BD0020FCE700BF0000020800000408BE
:10655000B8510024F0B5067906F0E003402B03D1D2
:1065600045794FF0FF3406E0602B4FF00105F8D17C
:10657000447905FA04F40023012006F00706AB4233
:1065800000D1F0BD052E0FD8DFE806F00308101D7E
:10659000242448B1C85CD75C78400FE020B1C856CD
:1065A000D756C71B784278410133E8E70028FBD073
:1065B00031F8130032F81370784080B220420CBFDB
:1065C00001200020F0E70028EED031F9130032F965
:1065D0001370E6E70028E7D051F8230052F8237043
:1065E000DAE7037903F01803102B1DD004D82BB180
:1065F000082B06D000207047182BFBD1B0F80B00F9
:106600007047114BB0F80B0093F90030591C09D1B9
:106610000E4B1B7A03EB830203EBC20300EB8300F8
:1066200080B27047DBB2F5E7074BB0F80B0093F987
:1066300001305A1C06D1054B5B7AC3EB031300EB08
:106640004300EDE7DBB2F8E7D0050024B8510024A1
:10665000114A00234FF0280C0360838030B54FF4BB
:1066600048744FF0290E02F1120503EB4303AA42CE
:1066700000EB430100F813C081F801E0D3788C806F
:106680008B7008D092F90630063292F801C092F869
:1066900002E09488E9E730BD087D0908092917D090
:1066A000B1FA81F35B0999B1013903604B0001F044
:1066B000030103F00802C1EB01119300C1EB0111CA
:1066C000A3EB92038900C3EB031381809B004380FB
:1066D000704700BF1F22032302704370704700BF42
:1066E00041F201424FF4007100234FF4A07C42803C
:1066F00040F20122018042F60241C2814FF4A472AD
:10670000A0F806C00381438183810182C382828213
:1067100003834383704700BF4FF0010C54210422D0
:10672000002380F800C041708270C370704700BFC2
:10673000144B1522144910B5044618681B792062C1
:1067400004F1250084F8243050F0EBFA0F4B4FF0A1
:10675000010E1A7E84F83AE012B984F83B2010BD8D
:1067600003F11C0CBCE80F0020606160A260E360D4
:10677000BCE80F0084F83BE020616161A261E36145
:1067800010BD00BFCCEC0908D4EC0908B8510024B6
:1067900010B500213822044650F082F90C4A092134
:1067A0000C480123226141F61E6C0B4A21720B49F1
:1067B000A373E161214684F82130A4F826C0C4E91E
:1067C0000502074A0748A262BDE8104027F04CB90D
:1067D0006400DC051A046C070019750343080E00F9
:1067E0001E7D0101E8EC0908B5EEC00ADFED357A3F
:1067F0000023F1EE10FA70B5C8BF30EE270A86B05C
:10680000D8BF30EE670ADFED307A054603A9029360
:106810006E4620EE270ACDE90033FDEEC07A17EE72
:10682000904A84EAE470A0EBE47045F067FA002C2B
:1068300003A8ACBF20232D238DF800304DF044FE7B
:10684000012829D0022833D003281DD003A93046BF
:1068500050F01EFA30464DF037FE044631462846C9
:10686000033CE4B2224650F0A7F8002328462B55FB
:106870004DF02AFE2E22431C31192A54E81850F0FC
:1068800023FA284606B070BD302303A930468DF8A0
:10689000013050F0FDF9DDE743F23002302303A967
:1068A0003046ADF801208DF8033050F0F1F9D1E712
:1068B00043F2300303A93046ADF8013050F0E8F957
:1068C000C8E700BF6F12033A00007A4408F0C6BA66
:1068D00013B568B14C1E14F8011F21B902B0BDE810
:1068E000104008F0CFBA019008F0B8FA0198F2E72A
:1068F00002B010BD202108B550F0D9F9034618B1F7
:106900001A780130202AF9D0184608BD10B50C4677
:1069100028B1C943013801F0010109F05BF9E3072F
:1069200001D4FCF7D9FC10BD2DE9F3410023124D31
:10693000044600EB8106114F05F83C3FB44203D1F9
:106940000F4802B0BDE8F081394628464FF00008F4
:1069500050F09EF92146684650F0B6F9202168466D
:1069600050F0A5F928B969462846043450F090F94A
:10697000E4E780F80080F1E7B851002413320A08F8
:10698000F4510024014B186E34F0C8BCB8510024F7
:106990002DE9FF471E46C368044689469246BDF866
:1069A0003070DDF834804BB3CBB20D2B24D81A4AAB
:1069B000D556BAF1FF3F23D023683146174A3846EF
:1069C000CDE9005AC04752465FFA89F12079FBF7BA
:1069D00041F9024600B10288D3B2314638460393EA
:1069E000C2F30323120B02932368CDE900520C4A31
:1069F000C04704B0BDE8F0870025DAE74D1CD8E7B2
:106A00007B06F6D423683146064A3846C4460C95C0
:106A100004B0BDE8F0476047B0EC090840310A080F
:106A20004D310A0871310A082DE9F041154686B04A
:106A3000884619466A1CBDF830600D9F26D00309B0
:106A400000F00F04184A30464033CDE90045059365
:106A5000B847C0B1EAB2D8F8000098F805100F2A7C
:106A600011D82A46FBF748F968B102880178304608
:106A7000059B0391C2F30321120B02910021CDE982
:106A800000420A4AB84706B0BDE8F0817306FAD45E
:106A9000030900F00F00064ABC460C904033304614
:106AA00006B0BDE8F041604780310A0892310A081B
:106AB000BB310A08084B024608498B420AD21846E5
:106AC00002E01C30884205D20388C3F30B039A42CC
:106AD000F7D17047002070475CB50A0890BD0A08DE
:106AE00070B50546B0F80900FFF7E4FF064B044611
:106AF000284693F86460FFF774FD16B1E368184404
:106B000070BDA368FBE700BFB851002438B5054647
:106B10000C46FFF7E5FF2B7903F0E00203F00703D3
:106B2000602A2AD1052B0CD8DFE803F0030B0F0BEA
:106B30001B1B6A79012393400278DBB214B1134323
:106B4000037038BD22EA0303FAE76A790123934010
:106B500002889BB214B113430380F2E722EA0303D5
:106B6000FAE701236A7903FA02F2036814B11343C6
:106B70000360E6E723EA0203FAE7052BE1D8DFE842
:106B800003F00303050507070470DAE70480D8E77C
:106B90000460D6E770B585880B4604460021C5F32E
:106BA0000B0518462A464FF07BFF6169084A0346E9
:106BB000914202D3074A914205D319B11846BDE864
:106BC0007040084770BD2A46BDE870404FF0F4BEE3
:106BD00090BD0A089DBF0A0838B5064C064DAC4268
:106BE00006D2A16820461C34FFF7D4FFAC42F8D38C
:106BF00038BD00BF5CB50A0890BD0A0808234840AC
:106C000010F0800F4FEA400182EA40000CBFC8B28A
:106C1000C0B2013BF4D1704730B505688D421AD936
:106C200001F1FF3E6C1E00231EF801CF082183EA0C
:106C30000C0313F0800F4FEA430C82EA43030CBFAE
:106C40005FFA8CF3DBB20139F3D17445ECD16A1CE5
:106C500002602B7030BD00236A1C02602B7030BDB7
:106C60009FED067AF7EE007A60EE870A20EE800A42
:106C700070EE277A80EE270A704700BFDB0FC9400D
:106C800007EE101ADFED7E7AB8EE477A27EE000A9B
:106C900060EE277ABDEEE77A17EE103A2033402BEC
:106CA00000F2DC809FED777AB4EEC70AB0EE677A27
:106CB000F1EE10FA0CDDDFED745A9FED746AF0EE20
:106CC000476A37EE657AF4EEC66AF1EE10FAF6DC42
:106CD000DFED6F6AB4EEE67AF1EE10FA0CD5DFED77
:106CE0006A5A9FED6C6AF0EE476A37EE257AF4EE49
:106CF000C66AF1EE10FAF6D4DFED676AB4EEE67A12
:106D0000F1EE10FA40F39680DFED646A36EEC77A52
:106D100027EE075A9FED624A9FED626AF7EE005A2E
:106D2000DFED616AA5EE046ADFED604A27EE054AF1
:106D3000E5EE066AA4EE267AF0EE656AE7EE245ADE
:106D4000E7EE646A86EEA54A9FED537A77EE877A7E
:106D5000BDEEE77A17EE103A2033402B77D89FED3F
:106D6000547AB4EEC70AF1EE10FA0CDD9FED466AD4
:106D7000DFED466AB0EE677A77EEC67AB4EEE67A71
:106D8000F1EE10FAF6DC9FED427AF4EEC77AF1EEFE
:106D900010FA0CD59FED3C6ADFED3E6AB0EE677AE3
:106DA00077EE867AB4EEE67AF1EE10FAF6D49FED3D
:106DB0003A7AF4EEC77AF1EE10FA54DD9FED377AA5
:106DC00077EE677A67EEA74ADFED353A9FED355AE1
:106DD000B7EE006ADFED346AB6EE007AA4EEA35A8D
:106DE00027EEA43AF8EE003AE4EE856AE3EE267A5E
:106DF00036EE676A67EEA37A26EE077AB7EE005A98
:106E0000002380ED044A8361C5EE256A436180ED6D
:106E1000095A0362C36126EE877A26EE866A66EE19
:106E2000A77A80ED007A80ED016A80ED027AC0EDEC
:106E3000037A7047DFED1F6AB4EEE67AF1EE10FADE
:106E40007FF566AFDFED126A36EEC77A60E7B6EE21
:106E5000007ADFED197AB7EE006ACFE7B7EE004AA5
:106E6000F0EE445A70E79FED137AF4EEC77AF1EE34
:106E700010FAA7D59FED067A77EE677AA2E700BFF2
:106E800027D4D2360024F448DB0FC940E4CB1641A6
:106E9000DB0F49C0E4CB16C1DB0FC93FDB0F494014
:106EA00092E741B99730083C15A82ABEF304353F54
:106EB00000247448DB0FC9BF000000009FED2E7A4C
:106EC00070EE077AFDEEE76A16EE903A2033402B1B
:106ED0004FD8B4EEC70AF1EE10FA0CDD9FED276A29
:106EE000DFED276AB0EE677A77EEC67AB4EEE67A1F
:106EF000F1EE10FAF6DC9FED237AF4EEC77AF1EEAC
:106F000010FA0CD59FED1D6ADFED1F6AB0EE677AAF
:106F100077EE867AB4EEE67AF1EE10FAF6D49FEDCB
:106F2000167AF4EEC77AF1EE10FA16DD9FED177AB5
:106F300077EE677A27EEA76ADFED155ADFED156A5F
:106F40009FED157AE6EE256A67EE865AA6EE267A5A
:106F5000E5EE877AB0EE670A70479FED107AF4EE9F
:106F6000C77AF1EE10FAE5D59FED067A77EE677AEB
:106F7000E0E79FED0B0A7047DB0FC93FDB0FC9400D
:106F8000E4CB1641DB0F49C0E4CB16C1DB0F49400F
:106F900092E741B99730083C15A82ABEDB0FC9BF5C
:106FA00000000000B0EEC07AF0EEE06A86FE876A6C
:106FB000B5EE406AF1EE10FA3DD0C6FEC75AC5EEF6
:106FC000867ADFED1E2ADFED1E3ADFED1E4A9FEDC9
:106FD0001E5A9FED1E3AB7EE006A9FED1D4ADFED87
:106FE0001D5AE7EEE23AA7EE834AE7EEA34AA7EE80
:106FF000846AA7EEA45AE7EE855AC5EE867AF4EEC7
:10700000C76AF1EE10FA03D59FED137A77EE677A2F
:10701000F5EEC00AF1EE10FA03D59FED107A77EE87
:10702000677AB5EEC00AF1EE10FA48BFF1EE677A62
:10703000B0EE670A7047DFED077AE0E739094E3DA9
:10704000E3B59E3E88FA163E45FE7F3F99FB243FFE
:1070500069A2163EA7DFA834DB0FC93FDB0F49400A
:107060009FED4D0A90ED005A35EE000A08B5FDEE91
:10707000C07A17EE903A2033402B7BD8FFF72EF8DA
:10708000F0EE403AFDEEC57A17EE903A2033402BF1
:107090007FD8B0EE450AFFF721F8B0EE405AD0EDA8
:1070A000014A9FED3D0A34EE800AFDEEC07A17EEEC
:1070B000903A2033402B69D8FFF710F8F0EE405A91
:1070C000FDEEE47A17EE903A2033402B5BD8B0EE19
:1070D000640AFFF703F8F0EE404A90ED023A9FEDA4
:1070E0002E0A33EE000AFDEEC07A17EE903A2033F6
:1070F000402B45D8FEF7F2FFB0EE404AFDEEC37AD2
:1071000017EE903A2033402B37D8B0EE430AFEF703
:10711000E5FFF0EE407A27EEA36AC1ED024A24EEC5
:10712000233A24EE057A67EE856A24EE254A65EE59
:10713000E77A25EE655AF0EE462A81ED004A65EEC3
:10714000A35AC1ED017AF0EE433A81ED055AE7EE1C
:10715000242AA6EE247AC1ED085AE6EEE43AE3EEDC
:10716000646AC1ED032A81ED077AC1ED043AC1EDED
:10717000066A08BDDFED093A84E7DFED087ACAE761
:107180009FED064ABAE7DFED054AA6E7DFED035AB1
:1071900096E79FED025A82E7DB0FC93F000000002F
:1071A0002DE9F0431D4689B0531C0F460393117817
:1071B000002900F00D8100240646A04608E0304674
:1071C0000134B847039A531C0393117800293CD02B
:1071D0002529F4D1931CCDE903385078302800F0EC
:1071E0008980A0F130034FF00009DBB2092B40F297
:1071F0008C806C282DD0782800F29180572817D9E0
:10720000A0F15803202B00F28A80DFE803F0BB884E
:1072100088888888888888888896B58888888888B3
:10722000888888889E888888888A88A38888BB0000
:1072300058B1252873D125213046B847039A013427
:10724000531C039311780029C2D1204609B0BDE830
:10725000F083039B5A1C03921B78782BB3D8572BCF
:1072600058D9A3F158012029ADD801A050F821F038
:107270009D730408C7710408C7710408C771040826
:10728000C7710408C7710408C7710408C7710408EE
:10729000C7710408C7710408C77104083B73040868
:1072A000C5730408C7710408C7710408C7710408CE
:1072B000C7710408C7710408C7710408C7710408BE
:1072C000C7710408C77104084D730408C771040826
:1072D000C7710408C7710408C77104082373040840
:1072E000C7710408B5730408C7710408C77104089E
:1072F0009D730408D31C4FF0010903939078A0F10B
:107300003003DBB2092B3FF674AF04AA03A946F0A1
:10731000BFFA6EE7002B98D0252B8CD053E7039A49
:1073200051E755F8040B0023049A39460090304683
:10733000FEF738FF039A044445E755F8041B30462E
:107340000134C9B2B847039A3DE7039A55F8043BA4
:107350001C6038E705AB00220A2155F8040BFEF744
:107360006FFF05AA4B46394630460092049AFEF755
:1073700019FF039A044426E705A955F8040BFEF704
:10738000A3FFEEE7A0F1580205AB102155F8040B5E
:10739000B2FA82F25209FEF753FFE2E7A3F1580274
:1073A000102105AB55F8040BB2FA82F25209FEF730
:1073B00047FFD6E705AB00220A2155F8040BFEF77C
:1073C0003FFFCEE705A955F8040BFEF77DFFC8E7A0
:1073D0000C463AE773B5114C06460D460192A06E75
:1073E000A0B10F49FFF774FA3146A06EFFF770FAAB
:1073F0000C49A06EFFF76CFA0B49019B2A46A06E60
:10740000FFF7CEFE0949A06EFFF762FA94F86C30E0
:1074100013B1012384F86D3002B070BDB85100245F
:10742000CF310A08D2350A08CD680408DC310A08D1
:107430000EB400B584B0084905AB019001A853F81B
:10744000042B0393FFF7ACFE019B00221A7004B0DB
:107450005DF804EB03B070472562040800232DE9B2
:10746000F0411C4682B0074603802146013438466D
:1074700031F036F9082CF8D1002307F1FC06DFF8CB
:10748000608087F8EA301D46C7F8EC30C7F8F03066
:10749000C7F8F430C7F8F8301F462A46414601A81D
:1074A0003446FFF7C5FF032201A911F8013B5BB188
:1074B000013A04F8013BF8D1013504362770082D54
:1074C000EBD102B0BDE8F081013520462021144403
:1074D0004FF0E6FA082D06F104062770DDD1F0E73B
:1074E000F4EC0908F7B5114E074600230C46304668
:1074F00015460F496E3600F86E3F04EB45050D4BFF
:10750000002F08BF19460C4F4FF0C2FBAC4202D10E
:107510000A4803B0F0BD394634F8022B6846FFF73D
:1075200087FF694630464FF0B3FBEFE7B8510024C0
:10753000E0310A08E9310A08F2310A08265200242B
:10754000F7B500230B4E044600EB41050A4F06F841
:107550009F3FAC4202D1094803B0F0BD394634F830
:10756000022B6846FFF764FF694630464FF090FBF8
:10757000EFE700BFB851002485320A0857520024B3
:10758000F8B54E1E054601F11F04054F16F8012FF0
:10759000284639460235FFF74BFFA642F6D1F8BD23
:1075A000F7310A0802460846531C05D1034B1A68F6
:1075B0001B790A600B717047014939E77B310A0872
:1075C00086320A0803685A1C02601970090A0368A7
:1075D0005A1C02601970704702681146531C036000
:1075E000D31C11F802CB01605178036093781B041F
:1075F00043EA0123111D43EA0C030160D07843EAFA
:1076000000607047A0F13003092B07D920F020005B
:10761000413819288CBF0020012070470120704795
:10762000303809288CBF00200120704741381928C4
:107630008CBF002001207047613819288CBF0020C2
:107640000120704720280BD0092809D00A2807D02C
:107650000D2805D00B3801288CBF00200120704771
:1076600001207047A0F14103192B98BF20307047CB
:10767000A0F16103192B98BF2038704710B56FF047
:1076800000440246044404E0B3EB0E0015D1A242CC
:1076900014D012F8013BA3F14100192811F8010B95
:1076A000A0F1410C98BF203300F1200EBCF1190F5E
:1076B000EAD91B1A04D10028E9D110BD002010BD61
:1076C000184610BD02B3844610B5841804E0B3EB2D
:1076D0000E0014D1A44513D01CF8013B11F8010B86
:1076E000A3F1410200F1200E192AA0F1410298BF36
:1076F0002033192AEBD91B1A04D10028EAD110BD76
:10770000002010BD184610BD1046704770B50446E5
:1077100008460D464CF0D8FE064602E014F8013F3C
:1077200043B1204632462946FFF7CCFF0028F5D169
:10773000204670BD1C46204670BD38B50749054639
:10774000FFF7E4FF041E0649284618BF0124FFF78F
:10775000DDFF08B144F00204204638BDFC310A08C0
:10776000E9480A082DE9F041064686469EF800C021
:1077700070460EF1010EBCF1200FF7D0BCF1090FDD
:10778000F4D0BCF10A0FACF10B05EFD0ACF10D0455
:10779000B4FA84F46409002CE8D1012DE6D9BCF1D7
:1077A0002B0F3DD0BCF12D0F39D0102A86463DD08D
:1077B0004FF0FF359046B5FBF2F502FB05F7FF43AE
:1077C000FFB20EF1010E002010E0ACF1300C5FFAB8
:1077D0008CFC944512DA8542764602D334D1674553
:1077E00032D21C404FF0FF301EF801CBBCF1390FF4
:1077F000EBD94CF0200CBCF1600F0BD801B10E603E
:107800002CB3B0F1004F2BD9DB0729D54FF0004046
:10781000BDE8F081ACF1570C5FFA8CFCD9E701248C
:10782000102A00F1010E90F801C0C1D1BCF1300F57
:1078300019D04FF0FF354FF01008B5FBF2F502FB01
:1078400005F7FF43FFB2BCE708FB00C0CCE7002808
:10785000DEDA13F0010F18BF6FF00040BDE8F081D1
:107860004042BDE8F0819EF801C00EF10106ACF186
:1078700041056046192D01D80CF1200078280BD065
:107880004FF0FF354FF01008B646B5FBF2F502FB9E
:1078900005F7FF43FFB294E710229EF802C06FF095
:1078A00070450EF1020E0F2790468AE701230A2247
:1078B000002157E770B50D461446FFF71BF8064642
:1078C000A0B1FFF7F3FF40F634039842A8BF184673
:1078D000B0F5617FB8BF4FF46170A0F561731920F6
:1078E000B3FBF0F32B702378013323703046FFF79E
:1078F00001F80646A0B1FFF7D9FF40F634039842DD
:10790000A8BF1846B0F5617FB8BF4FF46170A0F50D
:1079100061731920B3FBF0F36B702378013323708C
:10792000304670BD2DE9F04117461E4605464FF41E
:107930007A72002338463146454C4DF089FA454964
:10794000454A0144454882FB01C34FEAE17C0B44B0
:10795000CCEB631382FB03C24FEAE37C1A44CCEB0B
:10796000621284FB02C44FEAE27CCCEBA40C80FBE5
:107970000C404FEAEC74C4EBE010C3EB0314A1EB32
:107980008401A971C2EB0211A3EB81036B710CEBB3
:107990004C03A2EBC30240F2B55303FB10CC8000B2
:1079A0002A71BCF5896F45DA40F2DA239C4548DC40
:1079B000BCF5B77F2A4BB4BF0022012202EB420183
:1079C0004FEA420803EBC10391B2B3F86E3008EB03
:1079D000020E244C04EBCE044FF00B0E163401E0E3
:1079E00034F8023D634520DDBEF1010EF8D11C4B99
:1079F00042444FF0010E03EBC202B2F8583000F5DA
:107A0000FA600CF1010C4FF47A7285F802E0084438
:107A1000ACEB030C314600232880384685F803C0C0
:107A20004DF016FA2A81BDE8F0810EF1010E5FFAE1
:107A30008EFEE4E7032140F296534FF006080A4613
:107A4000C5E7022140F229434FF004080A46BEE789
:107A5000ABAAAA2A80BC92C78988888873B06D16A1
:107A6000C87C0908207D090808B50D4BD3E900231F
:107A700052EA030C0AD10146002340F201121846D3
:107A80000B804A808B808B710B8108BD054909688A
:107A90008A1843F10003FFF745FF012008BD00BF2E
:107AA000982D0024501E002490420B462DE9F041F1
:107AB000B0FBF2F60446154608D2124A05FB1644FE
:107AC0001846135D00F8013BBDE8F0819642B6FB15
:107AD000F2F706D20B4A05FB1767D15D03F8011BCD
:107AE000ECE7BA42B7FBF2F807D905FB1878054A6C
:107AF00012F8081003F8011BEDE74046FFF7D4FF2A
:107B00000346F2E7FCEC090830B5684C83B0B4F8E2
:107B1000D433B3F57A7F03D94FF47A73A4F8D4330E
:107B2000B4F8D633B3F57A7F03D94FF47A73A4F857
:107B3000D633B4F8D803B0F57A7F04D94FF47A730A
:107B40001846A4F8D833B4F8DA13B1F57A7F03D91C
:107B500000231946A4F8DA33B4F8DC23B2F57A7FAF
:107B600004D94FF47A731A46A4F8DC33B4F8DE3340
:107B7000B3F57A7F02D90023A4F8DE33884202D815
:107B80000021A4F8D813934202D30023A4F8DC33D5
:107B9000B4F8EA23B4F8EC339A4202D90023A4F8EB
:107BA000EA33434B1B8803B3424DAA78062A43D8D5
:107BB000414901EB820191ED2E0A2979002940D13A
:107BC00094F8F41307EE903AAB7907EE101AF8EE3A
:107BD000E77AF8EEC76A86EEA77A0BB130EE000AB4
:107BE000B4EEC70AF1EE10FA30DC637A032B14D836
:107BF000C3EB0313314A02EB4302237A032BC4F88D
:107C0000FC2312D803EB83012D4A03EBC10302EBE3
:107C10008303C4F8003403B030BD0023274A6372E5
:107C2000237AC4F8FC23032BECD90022244B2272C4
:107C3000C4F8003403B030BD29799FED220A002931
:107C4000BED0042A21D8002ACFD021E067EE807A66
:107C5000BCEEE77A8DED017A9DF8042007EE102A3C
:107C6000B8EEC77AF4EEC77AF1EE10FA01DD013210
:107C7000D2B2CAB1102AA8BF1022D2B28A42134689
:107C800038BF0B4684F8F433AFE7053A032AACD982
:107C9000F7EE007A87EE800A4EF010F92B889842B2
:107CA00028BF18462880A0E70122E6E7B851002443
:107CB000241D00208C290024C87C0908805200243F
:107CC000F85200246F1203382DE9F04FDFF8F882E4
:107CD00083B098F8043400AFA3F11702022A00F22F
:107CE0004E82AF4B7B6044F09DFF002800F01E8366
:107CF0000024022088F8A0440FF0DEFC98F8A43499
:107D0000022B00F0C682002800F04083A54B4FF400
:107D10007A7498F895C5002003F524754FF0640E29
:107D20005A88B2F57A7FB3F8462088BF5C80B2F5F6
:107D30007A7F9A8888BFA3F84640B2F57A7FDA88BE
:107D400088BF9C80B2F57A7F01D90022D8809988BB
:107D500003269142B3F85A10B3F85C2098BF98807C
:107D6000914293F86B2003F1660102F1FF3288BF64
:107D7000A3F85A00632A93F86C2002F1010288BF2D
:107D800083F86BE0D2B2092A1A4688BF83F86C00E8
:107D900092F80AB0063211F801ABD34538BF01F8AA
:107DA000010C013EF4D1BCF1010F03F1A40318BF93
:107DB00003F81F6CAB42B3D17B4B9B78042B00F0D4
:107DC000C2822BB9784A1388B3F5F07F00F2E981BB
:107DD000FFF79AFE754898F8AF15FEF75FFC98F824
:107DE000BD150E30FEF75AFCB8F8CA25B8F8C835EC
:107DF0001343B8F8CC2513431BB213B10123A8F8E1
:107E0000CE35D8F884356A4A1A40002A00F0CD826F
:107E1000DA0700F124825D0440F1C7816549D8F892
:107E200088250B400A40C8F88435C8F8882513F423
:107E3000004200F0F781002288F8E32588F8F32556
:107E4000D90440F1F98198F81336022B02D10123AD
:107E500088F81336DFF860A153460AF1780402E08F
:107E60000633A3420CD01A78072AF9D19978DA7828
:107E7000914202D35A79002AF2D0072020F0F0FF75
:107E800000234FF4806088F8A0340FF015FC002820
:107E900000F06F82484DA94699F8050080B199F825
:107EA000001051B1534602E00633A34208D01A78BD
:107EB0008242F9D15A79002AF6D0084620F0D0FF44
:107EC00009F106094C45E7D1374B93F802A0BAF106
:107ED000080F00F0D28198F8953598F8D123A3F1D6
:107EE0000103032AB3FA83F34FEA531388F8903659
:107EF00098F89635A3F10103B3FA83F34FEA5313CD
:107F000088F89636D8F88835C3F3C03188F89316C8
:107F100002D9002288F8D123284A03EA0201D8F8BE
:107F20008435134098F81620C8F88815C8F88435A9
:107F3000002A00F0F381B8F8AC36002B40F0C58180
:107F4000D8F8B03613F07F4F02D00023C8F8B0360F
:107F5000D8F8B8361A4A1A401AB140F20223C8F8C3
:107F6000B83698F8B436013B042B02D9012388F8BF
:107F7000B436AAF1050A134BBAF1030F93F890A592
:107F800040F24681BAF1000F35D000233B60064B2A
:107F90006FF0070103F10809A1EB030B1BE000BF21
:107FA000C87C0908F85200248C2900246857002452
:107FB00009600002F6DFFFFDD0570024DEDDCDFDB5
:107FC000FDFDFFFF241D0020B85100240BEB09002C
:107FD000504580F0EE8019F8010B0028F6D00AF029
:107FE000DBFF0028F2D080798307EFD53B680122C0
:107FF000002B40F0E380BA4B9B7913B10023B84AC1
:108000009371B8F8C23613F00C0F03D1C3F3031306
:10801000022B03D94FF42063A8F8C236B8F8C4364F
:1080200013F00C0F03D1C3F30313022B03D940F653
:108030000123A8F8C43698F8312798F83D379A42BA
:1080400000F2DB8098F8303798F83C279A4204D247
:10805000002388F83037A8F8343798F8322798F892
:1080600026389A4202D9002388F83237DFF8A4C2B2
:108070001CF8012C63467968002002EB42020A4496
:1080800092F8B4B192F8B5A192F8B6E11A7801303D
:108090005A45A8BF5A4603F8012B59799A78514599
:1080A000A8BF51467245A8BF7246032859719A70FD
:1080B000ECD10CF11E0C8B4B6345D9D1D8F80426BA
:1080C000002A00F037810020012102E00635AC4291
:1080D0000ED02B78282BF9D16B78043301FA03F3F7
:1080E0001342F3D0063522EA03020120AC42F0D15C
:1080F00008B1C8F804267C4D05F108042B4613F896
:10810000012B072A67D89C42F9D1EA4688B0202281
:10811000FF21E94648464EF0C3FC734A12F8013B82
:1081200059F8231001315DD1944249F82330F5D13B
:10813000B8F88E25D546B8F88C359A4202D36B4BE9
:10814000C8F88C356A4BFF226A4C03F1900088F81E
:10815000582893F90420142A04D0196834EA01013C
:1081600000F0EE800C338342F3D1634B5A79022A3C
:1081700001D100225A710C37BD46BDE8F08F5F4A2D
:1081800002EBC3037A6093F8D420002A3FF4ABAD2E
:10819000D3F8D830002B7FF4A6AD172388F8043429
:1081A000A1E54FF4F073138012E61C0760D5544923
:1081B00035E63B680022002B3FF41DAF48494B7C5D
:1081C000002B7FF41EAF4B79012B3FF414AF002A34
:1081D0007FF411AF15E7EA4688B02022FF216846F8
:1081E0004EF05EFC05F8016B0136082EA0D005F8B4
:1081F000016B0136082EF5D19AE7002298F8303746
:1082000088F83127002B3FF428AFA8F834271BE764
:108210000023334A1371BAF1000F00F0C480012328
:108220003B60B4E698F8E31500293FF409AED904A1
:1082300088F8F3253FF507AE1A067FF504AE98F8E7
:108240000434182B06D801229A402E4B1340002BE1
:108250007FF4F9ADDFF8C0A00AF1780410E62A49EE
:10826000D8F888250B400A40C8F88435C8F8882516
:1082700098047FF5DCAD2549D1E51A469B79002BA2
:108280003FF429AE537C012B7FF425AE02235374B7
:1082900021E600283FF43AAD1D4BFF2690F904502B
:1082A00098F8F11403F1900093F90820AA4203D141
:1082B000013901241E72C9B20C338342F4D1002C5F
:1082C0003FF424AD88F8F11420E598F8A8060AF0E8
:1082D00063FE00287FF434AEA8F8AC0630E600BF99
:1082E0008C290024FB5200249F290024AE014A015E
:1082F000C455002401000200882D0024C87C090810
:10830000FE9FFFFD00410001F79FFFFDF6BFFFFD4F
:10831000AC56002483520024D0570024284A13432B
:108320001143C8F88435C8F8881504E625480CF0D0
:10833000A7F8DDE4282020F093FDD8F80426C2E653
:1083400088F8582811E7D8F88425D8F8883522F419
:10835000805223F48053C8F884251B4AC8F8883516
:10836000538CB3F57A7FBFF433AD4FF47A735384F3
:108370002EE5D8F8843523F00063C8F88435D8F8A2
:10838000883523F00063C8F8883583E5D8F884255C
:10839000D8F8883522F0800223F08003C8F88425BD
:1083A000C8F88835B2E4524608E7D8F8882543F083
:1083B000080342F00802C8F88435C8F8882527E584
:1083C00000040500C45500248C2900242DE9F04F39
:1083D000784E83B0784B4FF0010AD6F86828DFF862
:1083E000F88102F2DC524345C6F868284CD29B461D
:1083F000724B734D9F1C714B5988002900F0BE8051
:108400007A18AA4234BF00200120052998BF40F005
:108410000100002840F0B280BBF800003C46C0F3E9
:108420000B000BE0118814460A44002900F0A680D6
:10843000AA4280F0A380052940F2A0806188814291
:10844000F0D161798B07EDD123885846DBF808100D
:1084500094F804900193FEF79DFBBBF80010B9EB74
:10846000113F00F093804FF0000ABBF804100BF1AD
:108470001C0B5BF8140CC1F30B0144F0BBFB5BF865
:10848000042CC3451060B6D3D6F884354D4DC6F8DC
:108490008835FFF719FC337AA5F178014A4C03EBD4
:1084A000830203EBC203727AC2EB021205EB830371
:1084B00001EB4202C6F80034C6F8FC231FF0F4FEBC
:1084C0004FF0FF33D6F80004636024F06DFA20F01B
:1084D00019FD05F59B6305F5AA6102E00633994293
:1084E0005ED01A78002AF9D19D78D878854202D3D7
:1084F00058790028F2D096F810366421227203EBE6
:10850000830303EB83039B00632BD8BF6423C6F86C
:108510006038B6F8143601FB03F3632B45DD1A46C9
:10852000C6F8643800232949C6F87C28C6F868389C
:10853000C6F86C38C6F87038C6F87438C6F878389B
:10854000A6F8803886F88238214BC1F8143728F015
:1085500023FCB6F8840896F8861821F007FD32F05F
:108560007DFF15F009FD1B4B012250461B6886F864
:108570008128C6F8683803B0BDE8F08FDBF8081032
:1085800058464FF0000AFEF705FB6EE7019BA11D60
:1085900058469A1FFDF7BCFC00287FF466AF62E7DF
:1085A000F27D003A18BF0122A5E70A46C6F8641812
:1085B000B8E700BFB85100245CB50A080000020803
:1085C00000000408F8520024D0050024241D0020D7
:1085D00080570024501E002490BD0A0838B501229F
:1085E0001C4B032805461C4C83F81C2720D96A1C09
:1085F00000231A490220D2B24FF0140E5200402A32
:1086000028BF4022C854023301EB030C9A420CF8F5
:1086100001ECF7D8FF2D4FF0FF034FF00E0008BF1D
:108620000222224482F88838BDE8384014F022BB88
:1086300000EB800004F5A073257205EBC00003EB8E
:108640008000C4F8000424F0AFF921F0A3FF22F069
:1086500077F8CCE7241D0020B8510024405A0024AC
:10866000054B0121D3F8CC2883F8C91842F4001235
:10867000C3F8CC28704700BFB85100240368C3F387
:10868000100230B5044687B00D463ABB2021039254
:10869000CDE901220122CDE9042103F17841B1F5B0
:1086A000801F0DD2029203F17843694601A85B0C4A
:1086B00003933EF0DFFC88B14FF0FF3007B030BDD0
:1086C000A3F10162B2F5801F04D20222A3F5801348
:1086D0000292E8E7052009F0C1FEFBE72946206881
:1086E00044F02AFA18B9236820332360E6E76FF0D4
:1086F0000100E3E72DE9F041694F92B03B78B12BDF
:108700007AD1FDF7F3FE80F00104E4B2654B04F08A
:108710000104654DB3F8C331644EADF80030B54285
:108720006CD3002C00F0B9803022002106A84EF056
:10873000B7F95F4B0497DB1B05935E4BDA68D407F0
:108740006BD45C4BD3F80C21D0076FD401230025E8
:108750000222694604A88DF840300F954BF064FB67
:10876000022269464FF6FF704F4FFDF795FC044615
:10877000B74265D30025022201A904A8ADF8045030
:108780004BF052FB022201A92046FDF785FC40BABE
:10879000022202A9C043ADF8080004A84BF044FB34
:1087A0000E9878B106ABC0F12002294618444EF06D
:1087B00077F90F9818B906A904A8FFF75FFF0023FF
:1087C0000F900E939DF840300F987BB1394BDA68CB
:1087D00042F00102DA60DA68D20707D5D3F80C213B
:1087E00042F00102C3F80C21D3F80C31B0FA80F04A
:1087F000400912B0BDE8F081012487E7A9881C3543
:1088000055F8140CC1F30B0144F0F4F955F8043C8D
:108810001B68834218BF012481E7274A5A6002F18E
:1088200088325A60DB68D9078BD58FE7224AC3F8B4
:10883000042102F18832C3F80421D3F80C3185E712
:10884000B7F8048002A904A88DF80D50C8F30B08EE
:108850001C3708F10603ADF8083037F81C3CC3F3A9
:108860000B021B0BADF80A2006228DF80C304BF0E2
:10887000DBFA062202A92046FDF70EFC044657F853
:10888000141C424604A84BF0CFFA204657F8141C9B
:108890004246FDF701FC04466AE70120A9E700BF54
:1088A00000000208C87C09085CB50A0890BD0A08E7
:1088B00000000408002000522301674570B5154CE4
:1088C000FFF702FA0122144ED4F86838154684F8EE
:1088D000D02803F2DC53C4F86838FFF70BFF28B147
:1088E0003378B12B02D1FDF701FE30B9032D01D051
:1088F0000135F2E7052009F0B1FD084A0023012106
:10890000126884F8D03884F8811884F8D138C4F813
:10891000682870BDB851002400000208501E0024D1
:1089200001230B4A10B50B4C82F81C37A375FFF7D7
:10893000C5FFFFF74BFD41F20242FF230E20A4F8D2
:10894000882884F88A38BDE8104014F093B900BF35
:10895000241D0020B851002490F88730F7EE002A3B
:10896000DFED695A002103EE903A90F88B3006EE65
:10897000103A90F88930F8EEE33A04EE103A90F8A5
:108980008A30B8EEC66A04EE903A90F88D3063EE05
:10899000A57A03EE903A26EE256AB8EEC44AF8EEC0
:1089A000E44AF8EEE33A26EE276A24EE254A64EE1E
:1089B000A54A63EEA53A24EE064A64EEA74A63EEA2
:1089C000A73AF0B5514D062600F1660EA5F10C0C44
:1089D000B7EE005A06FB01F290F88670AC1802441C
:1089E000F0EE456A15E0012904F1060402F10602E1
:1089F000EED190F8883007EE903A90F8903006EE7D
:108A0000903AF8EEE77AF8EEE66A27EEA55A66EEB7
:108A1000A56A237866EE867A07EE103AB8EEC77A32
:108A200027EE277AFDEEC77A17EE903A66EE847A43
:108A3000FA2BA8BFFA2323EAE3731372637807EED5
:108A4000103AB8EEC77A27EE277AFDEEC77A17EE0E
:108A5000903AFA2BA8BFFA2323EAE37353725CF827
:108A6000213007EE903A002BF8EEE77A49DDA37843
:108A700007EE103A90F88C30B8EE477A03EE103AD1
:108A8000B8EEC33A37EE677A23EE253A87EE272A07
:108A9000B0EE627AA2EE037A64EEA77A66EEA36A7B
:108AA00067EE857A27EE877AFDEEE77ABDEEC77A24
:108AB00017EE103AFA2BA8BFFA2323EAE373937256
:108AC00017EE903AFA2BA8BFFA2323EAE3730EF8C5
:108AD00001300131A38807EE903AF8EEE77A67EEAD
:108AE000A67AFDEEE77A17EE903AB3F57A7FA8BF43
:108AF0004FF47A738F4223EAE3739381BFF673AF27
:108B0000F0BDB7EE007AC7E70AD7233CB882090860
:108B100090F88E306BB3B0F85A308BB190F88F204C
:108B2000642102EB8203C3EB0313B3FBF1F3A0F860
:108B30005A30962312FB03F3B3FBF1F3A0F85C3039
:108B400043884BB190F88F30642203EB8303C3EB6F
:108B50000313B3FBF2F34380B0F846304BB19622D7
:108B600090F88F3013FB02F36422B3FBF2F3A0F80A
:108B70004630704790F821304BB3438B83B190F867
:108B80002230FA22642113FB02F203EB8303B2FBCF
:108B9000F1F2B3F57A7F4283A8BF4FF47A738383EF
:108BA000838843B1FA2290F8223013FB02F3642247
:108BB000B3FBF2F38380C3884BB190F8223003EB10
:108BC0008303B3F57A7FA8BF4FF47A73C3807047ED
:108BD00070B50B4C002504F5247694F8863013B15B
:108BE0002046FFF7B9FE20460135FFF791FF3046DA
:108BF000FFF7C0FF042D04F1A404EED170BD00BF47
:108C0000F8520024034BD3F8280E08B106F03AB905
:108C1000704700BFB851002408B50B46054902460D
:108C2000D1F8280E28B10449FEF7BAFABDE8084089
:108C3000E8E708BDB8510024CD680408024B01469E
:108C4000D3F8280EFDF744BEB851002408B50446F9
:108C50000848FFF7F3FFFFF7D5FF074B186E13F037
:108C600087FF09F087FA012C01D145F007FCFAF7DC
:108C700033FB00BF04320A08B85100240048DDE786
:108C8000BF3D0A080CB4C30607B500D561B905A9F4
:108C900004980191FFF7C0FFFFF7F0FF012003B038
:108CA0005DF804EB02B070470020F8E708B5FFF765
:108CB000C5FFBDE80840E1E710B504460348FFF7EB
:108CC000BDFF2046BDE81040F0E700BF10320A08A3
:108CD0000948002408B5FFF7EFFFFFF793FF074BA4
:108CE00083F82C4EC3F82C4F83F8304F21F0F8FD59
:108CF0002046FFF7ABFF00BF15320A08B851002429
:108D0000034B0146D3F8280E08B106F0A7B8704708
:108D1000B85100240CB407B510F020000BD079B97D
:108D20002320FFF7EDFF05A904980191FFF774FFD9
:108D3000FFF7A4FF012003B05DF804EB02B0704719
:108D40000020F8E70FB407B504A951F8040B01910E
:108D5000FFF762FF03B05DF804EB04B07047154BFA
:108D60001B6870B52BB30025134E1448FFF79EFF08
:108D7000FFF748FFFCF75AFAFCF78AFA044640B1BD
:108D8000132013F077FFFFF779FF0D48BDE870401F
:108D90008CE73046FFF7D6FF782D06D80135FFF770
:108DA00031FF642009F04AFAE6E72546FFF766FF3F
:108DB000F5E770BD181E0024795E0A083C320A08E7
:108DC00056320A080FB407B504A951F8040B0191F3
:108DD000FFF722FFFFF752FF03B05DF804EB04B08A
:108DE00070472DE9F041037903F0E002402A50D0AA
:108DF00004D85AB1202A29D0BDE8F081602A4BD08E
:108E0000802AF9D182794179254812E003F00703DD
:108E1000052B16D8DFE803F0101510150309D0F85C
:108E200005102048BDE8F041CCE7D0F805205142BC
:108E30001D48BDE8F041C5E7B0F80720B0F80510BF
:108E4000F6E7B0F90720B0F90510F1E746790024FC
:108E5000164D174805EBC605FFF7F0FE012395F800
:108E60000876A74202D8BDE8F04107E7D5F80466C6
:108E70004FEA840856F824204AB113B90D48FFF789
:108E8000DDFE56F808100C48FFF75CFF00230134A4
:108E9000E7E741790948C5E70948BDE8F04191E7AE
:108EA000AB320A085C320A0872320A08C87C090828
:108EB00089320A081B360A08DF460A089A320A086D
:108EC000C2320A082DE9F04387B0224EFCF776F94A
:108ED0000269838900250188044602928268DFF8CE
:108EE0008880019242881C4FDFF88090009242688F
:108EF0001A48FFF767FF15B94046FFF7D7FE3B68F2
:108F00009D4212DA3378052B21D809EB8303D3F87D
:108F1000AC27B3882946013511480093063636F848
:108F2000043CFFF74FFF062DE5D144F0D9FC8188C2
:108F30004388CB1A616803FB01110591FCF7EEF938
:108F400005990246074807B0BDE8F0433AE700221A
:108F5000DFE700BF702A0024942A0024DA320A08CE
:108F600044330A0853330A0838330A08C87C09080E
:108F70000249034801F500610EC923E700E0F11F33
:108F800070330A0810B57521044628F0E1F901464E
:108F90000948FFF717FF1A21204628F0D9F90146A2
:108FA0000648FFF70FFF1B21204628F0D1F90146A4
:108FB0000348BDE8104005E784330A0897330A08E0
:108FC000AA330A0838B50C4D95F8D30310F0FD0408
:108FD00005D10A48FFF7F6FE2046FFF7D3FF95F8C4
:108FE000D333013B012B06D80548FFF7EBFE0120E8
:108FF000BDE83840C6E738BDB8510024BD330A0883
:10900000C8330A086F4B42F201011A68B1EB124FE4
:109010004FEA12432DE9F04F93B000F0CF8042F2B7
:109020000302934200F0CC8041F20302934214BF4A
:1090300009230A23644A654D116805EB8303644ADA
:10904000644C6548654FDFF8BC81B1FBF2F2D3F8A0
:10905000C417FFF777FEB4F8322F4FF47A730A2063
:10906000B2FBF3F103FB1122B4F9343F92B2B2FB2D
:10907000F0F25B48FFF7A6FE5A4A5B495B48FFF7F0
:1090800061FEFFF7FBFDA17D594A05EB8101594BBC
:109090005948D31AD1F80C18A288FFF793FE574805
:1090A000FFF7CCFD94F8361F5548FFF74BFE5548A7
:1090B000FFF7C4FD94F8371F5348FFF743FEFFF74F
:1090C000DDFD5248FFF7BAFD00210A4694F8EF3360
:1090D0004E1C0B4113F0010F08D012B14046FFF7B0
:1090E000ADFD31463846FFF72DFE0122072E3146F1
:1090F000ECD1474E96F86A1506F5EC7306F13C0282
:10910000012918BF134693F8DC30032B02D04148E5
:10911000FFF718FE404B96F86A15A3F5CE720129A9
:1091200018BF134693F8DC30012B02D13B48FFF700
:1091300009FE394B96F86A15A3F5CE72012918BFBE
:1091400013461B695B7B012B02D93548FFF7FAFDFB
:10915000DFF8DC80FFF792FD0027D4F8383F08F1F4
:109160002009DFF8D0B0039358F8041B002963D01E
:10917000012303FA07FA039B1AEA030F1CD01AF023
:109180001F0F19D0274B59F82720D85D52F82020FF
:1091900037B12548CDE90412FFF750FDDDE904128F
:1091A0005846FFF7CFFDBAF1020F05D196F84117E7
:1091B00011B11E48FFF7C6FD0137D5E70B2339E78C
:1091C0000C2337E70010005CEC040024C87C09087D
:1091D00040420F00B8510024DB330A0896340A08D5
:1091E000EE330A08F8FF0120000800000F340A08D7
:1091F000000004080000020833340A0862340A0838
:1092000074340A087C340A087E340A0886340A0852
:10921000241D00209F340A08FC1E0020A7340A08E1
:10922000AC340A08F00500241B360A08BA340A08D0
:10923000DC840908B4340A08FFF720FD94F8821D85
:10924000D4F8842D05EB81017D48137AD1F84818B4
:10925000527AFFF7B7FD7B497B48FFF773FD7B49E7
:109260007B48FFF76FFDFFF709FD7A4B7A481968D5
:109270004FF47A73B1FBF3F1FFF764FD07A8FEF733
:10928000F3FB38B107A90AA84AF0FAFE0AA9734805
:10929000FFF758FDFFF7F2FCD4F8C42F002A00F0C6
:1092A0008A8007EE902ADFED6E6AB8EEE77AC6EEA6
:1092B000877AFDEEE77A17EE903A6A4FB7F88405A1
:1092C00058B107EE900ADFED666AF8EEE77A86EEAF
:1092D000A77AFDEEC77A17EE900AD4F8441F59B169
:1092E00007EE901ADFED5E6AF8EEE77A86EEA77A6F
:1092F000FDEEC77A17EE901AB6F87C67642ECDE9BA
:10930000000131465848A8BF6421FFF75BFD97F87C
:10931000863597F8872505EB8303B7F888155348FA
:10932000D3F85C38FFF74EFDB7F89815504889B26E
:10933000FFF748FDFBF742FF016921B182684D4804
:10934000120DFFF73FFD4C48FFF778FCD4F8883545
:109350001B0660D597F8B835032B8CBF47484848A3
:10936000FFF76CFC94F8A434022B26D14548FFF794
:1093700065FC97F8B835042B44D84348FFF75EFCEA
:1093800097F8C835002B44D005EBC303D3F8B418C5
:109390003E48FFF7D7FCFFF771FC3D48FFF74EFC56
:1093A0000126D4F8CC483B4F002C38D1FFF766FC9F
:1093B00013B0BDE8F08F13467FE702200EF09CF952
:1093C000064608B93448D2E732F02EF896F9041070
:1093D00005EB80000131D0F870283048FFF7B2FC6F
:1093E00094F8A734012B04D12D48FFF727FC2D4812
:1093F000BDE7B3792C4805EB8303D3F87018FFF76A
:10940000A1FCF4E794F8A6340BB92848B6E728483D
:10941000B4E72849BCE72848FFF710FCBBE794FAFB
:10942000A4F33846B3FA83F306FA03F205EB830399
:10943000D3F8E81824EA0204FFF784FCB4E700BF7D
:10944000BE340A08D0340A08F1340A08FF340A0886
:1094500005350A08501E00240B350A0825350A0870
:1094600000247449B062002438350A087E350A08A1
:10947000A5350A08B4350A08CF350A08D5350A08D3
:10948000E1350A08F1350A084F5F0A0839360A083B
:1094900055360A0845360A08F7350A0801360A081B
:1094A00015360A081A360A0846400A081E360A08FF
:1094B0002E360A08D3330A0849360A082DE9F04F38
:1094C000DFF8748199B098F80B30002B00F097808A
:1094D00050480025504EDFF864B1FFF7E7FB2F46F8
:1094E000DFF85C91DFF85CA10BA9E8B214F096FFFD
:1094F0009DF83430002B53D0139C54B107EE904AA2
:109500009FED460AF8EE677A80EE270A4CF0D6FC0B
:1095100004460B9A29465846FFF714FC109A002A75
:109520006FD002FB04F04FF47A73B0FBF3F30993AE
:10953000DDF848C0BCF1000F65D00CFB04F142F22D
:109540001073B1FBF3F1082D98F80B3018BF7F189A
:10955000002B5AD017984FF47A7E0A23079015985B
:109560000690169805901198B0FBFEFECDF810E01D
:109570000998B1FBF3FE03FB1E11CDE902E1099945
:10958000B1FBF3F103FB1100BCFBF3F3CDE90010D9
:1095900021465046FFF716FC0023B362C6E90D339F
:1095A000013540361D2D9FD198F80B3023B31C4C4C
:1095B0004FF47A731B48D4F8CC15D4F8D025B1FBFE
:1095C000F3F3D208D4F8D415FFF7FCFB0A221648AF
:1095D000B7FBF2F102FB1172FFF7F4FB134B1B78A0
:1095E000432B06D1D4F8D825D4F8DC151048FFF762
:1095F000E9FB0023C4F8D43519B0BDE8F08F0D485D
:1096000067E7099294E761469DE721464846FFF7E0
:10961000D9FBC1E76B360A08F46000248096184B2A
:10962000B062002412370A0832370A08A81E002444
:1096300056370A08C9360A08B8510024D3360A0832
:109640007B460A08E2360A0813B52948FFF7F6FAFE
:10965000284B93F8F535002B48D02748FFF726FB19
:109660001EF088FB80B1254B254893ED280A8DED2F
:10967000010AFFF7E3FA234B9DED010AB3F88435A5
:109680003BBB2148FFF712FB204C2148B4F81818C7
:10969000FFF758FB94F8143813B31E48FFF706FB86
:1096A000B4F81C181C48FFF74DFB94F81638CBB1E2
:1096B0001848FFF7FBFAB4F81A181848FFF742FBEE
:1096C00094F8153883B1134802B0BDE81040FFF795
:1096D000EDBA4CF0F3FB81B21148FFF773FBD3E70F
:1096E0001048DBE70F48E4E70E48EDE70E48EBE7EC
:1096F00080370A08B851002496370A08A4240020AD
:109700009D370A08B0620024B7370A08241D0020DC
:10971000C6370A08E6370A08F6370A0810380A0872
:10972000C1370A08EF370A08FD770A080EB403B5F7
:1097300003AA52F8041B0192FDF74CFE064BD3F826
:10974000282E1AB90549986EFDF7C2F802B05DF8E7
:1097500004EB03B0704700BFB8510024BF3D0A08B6
:109760002DE9F04798460B7981460F4603F0E00457
:109770001646402C31D10024674DDFF8A081DFF878
:10978000C09122E03B7903F00703013B042B04D88E
:10979000DFE803F006080B0E2000315D28460AE0E2
:1097A0003157FBE736F81410F8E736F91410F5E7EF
:1097B00056F824104046FFF7C5FA7B79013BA342D7
:1097C00002DD4846FFF73AFA01347B79A342D9DC3F
:1097D000BDE8F08756F82410E0E703F00703052BF7
:1097E00058D8DFE803F0030C141619313578602CD3
:1097F0005ED045D8002C66D0202C7CD0E8E796F9C6
:109800000050602C54D03BD8002CF5D148E035886E
:10981000EDE7B6F90050F4E7D6F800A0202C554645
:1098200069D02BD8002CD3D151463C48FFF78AFA97
:10983000D7F805108A4518D8B8F1000FC8D03848B5
:10984000BDE8F047FFF77EBA202C356853D015D815
:10985000002CBDD129463048FFF774FAD7F805101F
:10986000A94202DB4B42AB42E6DDFFF707FA2B468B
:109870003A6848462B49BDE8F04757E7602C17D0B7
:10988000802CA5D13178284B2848002914BF3146B7
:109890001946D5E7202C2DD007D8002C98D1254685
:1098A000B7F90540B7F9076011E0602CE8D1002551
:1098B0007B7945FA03F3DB07BDE8F0474CBF1C4852
:1098C0001C48FFF73FBAB7F80540B7F807602946CC
:1098D0001148FFF737FAAC42C7DCAE42C5DBB8F13E
:1098E000000F3FF475AF324621461348BDE8F047FC
:1098F000FFF728BA00257A79104B03EBC20393F8DF
:1099000008269542B1DAD3F8043653F82500BDE8AD
:10991000F047FFF793B900BF86320A086F320A0892
:1099200030380A0836380A08F55E0A08DF460A08A1
:10993000D7320A08FD770A0846310A08C87C0908A8
:109940007C340A0813B50446084601920091FDF7DD
:10995000C7F802462046DDE9001302B0BDE810401A
:10996000FEE60EB403B503AA52F8041B0192FDF7FC
:1099700031FD054B0549986EFCF7AAFF02B05DF872
:1099800004EB03B0704700BFB8510024BF3D0A0884
:1099900002460149E5E700BF50380A08F8B50C4611
:1099A00006460846FDF782FF2021054620464DF079
:1099B0007EF9044618B93046BDE8F840E8E7114F93
:1099C000114E3B7832789A4201D0FBF763FD0F4B82
:1099D00020461D604AF078FD012201462046FBF733
:1099E000FBFC3B7832789A4201D0FBF753FD2046CE
:1099F0004AF06AFD2A4601460548BDE8F840FFF7EF
:109A0000E1B900BF141E0024A02A0024101E002467
:109A100067380A082DE9F0410D4688B00646084629
:109A2000FDF744FF2021044628464DF040F920B9B7
:109A3000304608B0BDE8F041AAE7FDF737FF2246FF
:109A4000054601460F48FFF7BDF985B1202D2A468E
:109A50006946204628BF2022E846FBF737FD00274D
:109A60000646B74208DBAD1B3444002EEDD1FFF7AC
:109A700005F908B0BDE8F08118F8010B0137FFF7D0
:109A80003FF9EEE77D380A0810B504460748FFF7AE
:109A90000DF9FBF7B1FD20B10548BDE81040FFF717
:109AA00005B920460349BDE810405AE795380A0831
:109AB0009F380A08A7380A08154BD3F86C3A2DE9E5
:109AC000F041044688B0F3B11A6804A91846D56A73
:109AD0006A46A847064688B104AC6D460027DFF801
:109AE0003C80013735F8022B34F8021B4046FFF763
:109AF00069F9BE42F5DC08B0BDE8F08105492046B1
:109B0000FFF72FFFF7E7044908B0BDE8F04128E769
:109B1000B8510024C8380A08E0380A08AE380A08E4
:109B200013B50446084601914AF0CEFC024670B1D6
:109B3000132804D1019909484DF0DFF838B1074BDB
:109B40002046074A074902B0BDE8104009E703492B
:109B5000054802B0BDE81040FFF734B9D4EC09085D
:109B6000E7380A08F2380A081C390A0813B504460F
:109B7000084601914AF0A8FC0199024668B1042800
:109B800003D109484DF0B9F838B1074B2046074AD0
:109B9000074902B0BDE81040E3E60349054802B0BA
:109BA000BDE81040FFF70EB9CCEC09082A390A08C5
:109BB000F2380A083A390A082DE9F04300279BB029
:109BC000064608460C464AF07FFC05461C223946EC
:109BD00002A801974CF064FF25B3402D07D0402325
:109BE0002A46384930461BB0BDE8F043B9E60DF1CE
:109BF000040804F140090222214668464DF091F81C
:109C00000023102209A968468DF80270FDF7AAFD0D
:109C1000099B0DF10202934222D1023408F8010B94
:109C2000A145E8D100213D220AA809914CF038FF56
:109C3000002D3AD0244C257ED5B1202204F11C0100
:109C400001A84CF003FF98B104F11C0109A8FDF72D
:109C500097FC09AB1D4A30461D49FFF782FE04E020
:109C60001A7830461B49FFF77CFE1BB0BDE8F08335
:109C700094F86430CBB9C5B901AD174C0FCD0FC402
:109C800095E80F0084E80F00144B012209A8A4F105
:109C9000100183F8E025FDF773FC1148FFF70CF87D
:109CA00009A91048FFF78EF8DFE70C4B93F8E03571
:109CB0001BB9054B1B7E002BF2D0074909A8FDF705
:109CC0005FFCEDE74D390A08B85100248B390A08CA
:109CD000F2380A086F390A08D4510024B06200240F
:109CE00095390A08A4390A082DE9F74F3D4F8346F4
:109CF00008460D464AF0E8FBD7F884950446B8B903
:109D0000394D0126394F3A48FEF798FF55F8041BA4
:109D100049B106FA04F313EA090F02D03846FFF7F7
:109D200011F80134F2E703B0BDE8F04FFEF7A6BF2B
:109D3000024630492846FDF7C5FC78B92A4C2E4D1D
:109D40002E48FEF77BFF54F8041B0029EBD00B785C
:109D5000002BF8D02846FEF7F5FFF4E72B782D2BE3
:109D600011D10135013C4FF0010A1F4B002653F879
:109D7000048BB8F1000F09D12A462149584603B097
:109D8000BDE8F04FEDE54FF0000AEEE72246414610
:109D900028460193FDF796FC019B00BB0123B340CD
:109DA0009A0505D5174803B0BDE8F04FFEF77EBF12
:109DB000BAF1000F0DD029EA03031348C7F8843520
:109DC000FEF73CFF41460C4803B0BDE8F04FFEF7FC
:109DD000F9BF49EA03030D48C7F88435F0E70136B7
:109DE000C5E700BFB851002418860908BB390A0826
:109DF000B1390A08CE360A0845360A08BF390A08BA
:109E0000CA390A08DB390A08E7390A08F0390A08AA
:109E10002DE9F74F814608460E46174698464AF008
:109E200053FB0446E8B9404D4048FEF78BFF2046FF
:109E30000DF04EFA3B68184206D020460DF05AFA53
:109E400001462846FEF77EFF0134182CEFD13B680F
:109E500013B93748FEF7F2FE03B0BDE8F04FFEF746
:109E60000DBF024633493046FDF72CFC0546A8B924
:109E70002C46314D3148FEF7E1FE20460DF028FA20
:109E800010EA080F06D020460DF034FA01462846A5
:109E9000FEF758FF0134192CEFD1DDE733782D2B75
:109EA0002AD10136013C012548F080734FF0000AA9
:109EB000019350460DF01EFA224683460146304675
:109EC000FDF700FC18BB50460DF002FA019B03425F
:109ED0001DD09DB1BAF1180F02D03B6840EA0308CB
:109EE0001748C7F80080FEF7A9FE5946124803B08C
:109EF000BDE8F04FFEF766BF0025D5E7BAF1180FB1
:109F000002D03D6825EA00050E483D60EBE70AF106
:109F1000010ABAF1190FCCD132460B49484603B0B9
:109F2000BDE8F04F1DE500BF44360A08F8390A08BD
:109F3000023A0A08CE360A0845360A08BF390A0826
:109F4000E7390A08F0390A08CA390A0840F2022338
:109F5000004A5DE7705800246FF07F43004A57E7DE
:109F60006858002408B50A4B93F8E425032A0AD15F
:109F700093F8E535092B06D126F0DAFE0548BDE851
:109F80000840FEF71FBF0449BDE80840E9E400BFF0
:109F9000B0620024093A0A08143A0A0870B5054666
:109FA00008461646FDF782FC0D4B044693F89025B3
:109FB000904205D201460B48FEF704FF204670BDD3
:109FC0002EB1FF2803D10848FEF7FCFEF6E7013A60
:109FD000064928464FF0FF34FFF7C3FCEEE700BF09
:109FE000241D0020233A0A08343A0A08473A0A088E
:109FF0002DE9F04F074691B082480E46824DFEF79C
:10A00000E1FE002381494024062285F808363046C7
:10A01000012391F89015C5F804D685F8094608F093
:10A020006BF80A2008F00AF995F808360C2BDAB21A
:10A0300040F2E4809DF80C50FE2D30D0FF2D0BBF78
:10A0400015240F2401260026944240F0D780611E7B
:10A050006846C9B237F06AFB04F140030DEB030414
:10A0600014F8413C834240F0C48006F1FF389DF86B
:10A070000D305FFA88F8B8F1010F12D903F01F070D
:10A080005C0961376248FEF7D9FD022E6AD0013CB7
:10A09000042C65D8DFE804F00B5E606462000226E1
:10A0A000D2E79DF80E701D469DF80F40EAE759482B
:10A0B0006C464FF0000ADFF8B891FEF7F7FDDFF8C5
:10A0C000B4B15548FEF7BAFD0AF1010A14F8011BB4
:10A0D0004846FEF737FEBAF10C0F49D1FEF7CEFD28
:10A0E000022E4FD064223B464C48B5FBF2F102FBF6
:10A0F0001152C9B2D2B2FEF765FEB8F1010F71D8A4
:10A10000474A484B9DF810104748002914BF114694
:10A110001946464DFEF756FE9DF81110444B454832
:10A12000002914BF19462946FEF74CFE022E59D1CC
:10A130009DF812404048FEF781FD4CB3FF2C37D00C
:10A140000A223E48B4FBF2F102FB1142D2B2FEF702
:10A1500039FE20E03A48ABE73A48A9E73A48A7E792
:10A160003A48A5E700230DF11F008DF83F309FE727
:10A17000374B03FB0AF2B2F1553FA5D85846FEF71C
:10A180005DFDA1E73A4629463248FEF71BFEB7E7D8
:10A190002846FEF78BFD9DF813402F48FEF74EFD35
:10A1A00044B1FF2C21D021462C48FEF70BFE04E0E1
:10A1B0002B48EEE71D48FEF779FD0DF1130500244D
:10A1C0001A4E274FDFF8688015F8013F7BB1FF2B4F
:10A1D0000CBF3A464246214601342248FEF7F2FDC2
:10A1E000042CF1D111B0BDE8F08F1D48E3E73246F1
:10A1F000F1E71D493846FFF7B4FBF3E71B48FEF7CC
:10A2000055FDEFE78D3A0A08B0620024241D0020B6
:10A210009E3A0A08A93A0A08CF3A0A08E13A0A0817
:10A220006D3A0A08763A0A08183B0A087D3A0A0885
:10A23000BC480A082F3B0A08363B0A084A3B0A0872
:10A24000B03A0A08B83A0A08C03A0A08D3330A08EA
:10A25000ABAAAAAAFD3A0A08523B0A0886320A08A3
:10A26000813A0A08623B0A086D3B0A087D3B0A08EE
:10A27000F7310A08F55E0A082DE9F84F07460C4643
:10A28000DFF8A480DFF88490DFF8A0A020464AF031
:10A290001BF9064660B91D4B1D4893F804241D4B5D
:10A2A00003EB8203D3F8C819BDE8F84FFEF78ABD67
:10A2B000024641462046FDF705FA60B1DFF85CB082
:10A2C00000255BF8041BB1B9224638461249BDE8A7
:10A2D000F84FFFF746BB114C114D1248FEF7AEFC8C
:10A2E00054F8041B19B12846FEF72CFDF8E7BDE829
:10A2F000F84FFEF7C3BC324620460135FDF7E2F9C0
:10A300000028DED1544689F80454BFE7B851002430
:10A31000863B0A08C87C0908CA390A0894860908D5
:10A3200045360A08BF390A08CE360A08C13D0A0870
:10A3300038B50D460446052219492846FDF7C2F9ED
:10A3400068B9184B93F86C2022B9012183F86D206D
:10A3500083F86C101448BDE83840FEF7A7BC032210
:10A3600012492846FDF7AEF9A0B90E4D95F86C30AC
:10A3700063B195F86D304BB10D492046FFF7F1FA06
:10A38000002385F86C3085F86D3038BD0948FEF73C
:10A390008DFCF5E720460849BDE83840FFF7E1BAF3
:10A3A00001480A08B8510024903B0A0865490A0888
:10A3B000A63B0A08DD3B0A08F13B0A08F8B5174C32
:10A3C000054694F86C307BB194F86D3063B1144954
:10A3D000FFF7C7FA28461349FFF7C3FA002084F8AD
:10A3E0006C0084F86D00F8BD0F4E96F8E07597B1DB
:10A3F000207E0028F7D10D4D06F20C640FCD0FC45E
:10A4000095E80F0084E80F00012386F8473608F02E
:10A4100055FF3846E7E70120E5E700BFB8510024C3
:10A42000A63B0A08003C0A08B0620024D45100246C
:10A4300008B5FFF7C3FF50B1054B01229A75FEF72F
:10A440003DFA0448FEF738FC0020FEF7FFFB08BD8C
:10A45000B85100241E3C0A0808B5034610462AB12C
:10A46000DB0600D511B1FEF727FC002008BDF8B5CA
:10A470000D4E054696F8643093B9F8BD25B1238892
:10A48000C3F30B039D4204D0A288D4E902014CF02F
:10A4900093FA1C34BC42F1D3002386F86430ECE715
:10A4A000024C034FF6E700BFB85100245CB50A0820
:10A4B00090BD0A082DE9F04F164685B01A4682462F
:10A4C000019130460021334CFFF7C6FF4FF00009E1
:10A4D00006F0100305460293FEF794FB2379019AD8
:10A4E00003F01803934203D0002A48D1182B46D119
:10A4F0004FF00D0B274B0BFB0933B3F80900FCF7AA
:10A50000D9FA80462046FCF76CF80746D8E90221C4
:10A51000024401442046FCF71DF880F001012A4660
:10A520000390C9B23046FFF797FF0546DDE90223E5
:10A5300002B123BB174A0BFB09FB52F80BB0B20662
:10A540000FD573B9594614480393FEF7FBFBD8F8AF
:10A5500008202146039B50463A44FFF701F9FEF7D5
:10A560008DFB59460D48FEF7EDFBD8F80C20002373
:10A5700021463A445046FFF7F3F8FEF77FFB09F116
:10A58000010940F24F230D349945A5D105B0BDE82E
:10A59000F08F00BF98960908253C0A08263C0A0857
:10A5A0000149FFF7DEB900BF303C0A0838B50C4658
:10A5B000054615492046FDF761F830B9FEF708FB5E
:10A5C0001248BDE83840FEF771BB11492046FDF73F
:10A5D00055F8A0B90F4A82F8C60182F8CE0182F878
:10A5E0006A0282F8720282F80E0382F8160382F879
:10A5F000B20382F8BA0382F8F1030748E1E728467C
:10A60000BDE83840CCE700BF3F3C0A08453C0A089B
:10A61000603C0A08B8510024683C0A082DE9F04360
:10A62000064687B008460C4649F04EFF082844D13C
:10A63000671E03AD073429463A46A84612F8010FB3
:10A64000FDF716F801F8010BA242F7D10023DFF85D
:10A6500080908DF8143017F8010FFDF709F805F810
:10A66000010BC1B2484601914CF021FB20B1019988
:10A6700028464CF01CFB28B13046FFF791FF07B08D
:10A68000BDE8F083A742E6D11049404623F0ECF93B
:10A690000E4808230E4910F8012B013B11F8014B1D
:10A6A00002F118026A4402F80C4CF4D103A90948DB
:10A6B0008DF81430FEF786FBE1E70028E8D030463D
:10A6C00007B0BDE8F043FFF763B900BF8C57002423
:10A6D00098000A08843C0A082DE9F74F4FF0000B58
:10A6E000064601AA08462E495D464CF09BF9012713
:10A6F0000446DFF8BC80DFF8BC90DFF8A4A01CBBE8
:10A70000BBF1000F28D1274C002D44D02946264804
:10A71000FEF758FB94F864300BB904F0D1F9FCF75C
:10A720005BFA002384F86D30FEF752FA15B1284623
:10A73000FFF79DFE9FB13046FFF740FE78B1FEF770
:10A74000BDF80020FEF782FABBF1000F0AD02046C8
:10A75000FDF7ACF885B2C5B93046FFF721FF03B06D
:10A76000BDE8F08F41462046FCF7D0FF80B949464E
:10A770002046FCF7CBFF0028EED05F4601AA5146E9
:10A7800000204CF04FF90446B9E74FF0000BF5E715
:10A790004FF0010BF2E70548FEF78EFABFE700BF66
:10A7A00013320A08B8510024943C0A08B73C0A083E
:10A7B0008B3C0A0838480A0807B5009313460A4636
:10A7C0000249FFF7CEF803B05DF804FBCD3C0A0860
:10A7D00020B10078B0FA80F040097047012070473E
:10A7E0002DE9F34106460846FFF7F2FF0D460746FE
:10A7F00070B1002401A92046013441F07FFA0146DE
:10A800003046FFF7EDFF122CF4D102B0BDE8F08125
:10A810000846FDF74BF8C4B2112C72D8681C3D4DA8
:10A82000FCF768F88046E8B93B4B03EB440393F828
:10A8300048168A1E51425141374B03EB440393F8AB
:10A840004826AA5C002955D093F84936192040F2D1
:10A85000EE2100FB03132146304802B0BDE8F04171
:10A86000FEF7B0BA017828464CF021FA78B1032CF3
:10A870002B49A0EB050394BF0022012202EB420208
:10A880000A4452FA83F393F8387A032F04D13046FE
:10A8900002B0BDE8F04183E64046FCF72BF808B370
:10A8A000022FF4D1FDF702F840F6CA0280B21A4B2B
:10A8B000904203EB4403A8BF104640F2EE229042C0
:10A8C000B8BF10461922A0F2EE20B0FBF2F083F8D8
:10A8D0004906BB1E594259410F4B03EB440383F811
:10A8E0004876A9E7022FF4D1304602B0BDE8F04126
:10A8F000FFF74EB821460B4802B0BDE8F041FEF725
:10A9000061BA11233A460849304602B0BDE8F04129
:10A9100052E700BF94020A08B0620024E63C0A082D
:10A92000C87C0908F63C0A08033D0A082DE9F04FE7
:10A93000024691B008460B46FFF74AFF044628B18D
:10A94000104611B0BDE8F04FFFF722B84FF0FF32CC
:10A9500027462646DFF8E082DFF8E092DFF8E0A243
:10A96000CDE90820A24A126E92F83810CDE90E0205
:10A97000CDE90C10CDE90A0007AA9E4918464CF013
:10A9800051F8054604944DB9089A0C9FBA4262D119
:10A990009948FEF717FA11B0BDE8F08F062F12D8CC
:10A9A000DFE807F0041E2328454C51005146284695
:10A9B000FCF7ACFE78B14FF4806001240CF09CFEF3
:10A9C00090F90430089307AA8A49002001374CF017
:10A9D00029F80546D7E72846FCF768FF0890F2E714
:10A9E0002846FCF763FF0990EDE72846FCF7A5FE33
:10A9F0000A90E8E7284649F067FD4146024605907F
:10AA00002846FCF75FFE18B3059A49462846FCF72E
:10AA100059FE06460028D6D02846FCF747FF0428F2
:10AA20000646D0D901467548FEF7CCF9B3E728466B
:10AA3000FCF73CFF00230C900F93C4E72846FCF77B
:10AA400035FF0D90BFE72846FCF777FE0E90BAE77A
:10AA500001230493B7E7DFF8EC8151B2434613F9C1
:10AA6000010B884208D001350C2DF8D100210131AD
:10AA70006348FEF7A7F98EE701216248FEF7A2F9C5
:10AA800000237AB218F9011B8A4200F00C810133CD
:10AA90000C2BF7D13A460121E9E7A7F11402534202
:10AAA0005341059308AD002303F10108EB68A3BBF4
:10AAB00095F900B058460CF0EBFDD5F804A020B194
:10AAC000D0F80090B9F1000F5ED1BAF1000F19D1A2
:10AAD0004FF461434FF0010A6B60AB680BB903237D
:10AAE000AB600023D5F804905846029319462A7AA1
:10AAF000CDE900921A4611F0BDFFE86028B9414641
:10AB0000414891E74FF0000AE7E74A464146BAF16B
:10AB1000000F37D03D48FEF715F9B8F1020F05F1E7
:10AB200010054FF00103BFD1059BDDF83C800B9D64
:10AB300053B13748FEF7BAF8D8F800301B6A1BB19A
:10AB40002A46344940469847049B002B4ED0324950
:10AB5000324B142F18BF19463148FEF733F9142F22
:10AB600009D1049B03B936B12B68DB691BB13246AE
:10AB70002C4928469847002C66D100224146284699
:10AB800041F070F82848C6E7C5F80C90BAF1000FFC
:10AB900025D0414625485246FEF7D4F8514648464E
:10ABA00002F08CFED5F808A0BAF1000F0FD099F88A
:10ABB000042092450BD0534641461D48FEF7C2F88B
:10ABC000D9F800305FFA8AF148469B699847D9F86E
:10ABD0002C30002BA1D00023C9F82C309DE7D9F8E8
:10ABE000082041461348FEF7ADF8DBE70B49B3E711
:10ABF000B851002413320A08413D0A08293D0A08C9
:10AC0000853E0A085A3D0A08663D0A08823D0A0840
:10AC1000393E0A08BDD804080B3D0A08C13D0A08A0
:10AC2000623E0A080D690408A63D0A08C23D0A08EA
:10AC3000143E0A08EF3D0A08233D0A08043A0A08B0
:10AC4000183D0A08D08009081C4F0026DFF87490D0
:10AC50004FF0030A04F09AFF052007F0EFFA99F885
:10AC60009035B34289D917F801BBBBF1000F15D05D
:10AC7000584608F091F9044680B1584604F0D4FED5
:10AC800008B1A0F806A001210490F7F749FCA379C8
:10AC9000049813F0010F03D0F6F7C2FF0136DEE788
:10ACA000F6F7B8FFFAE73A4602210548FEF78AF8B8
:10ACB000099B002B3FF4F1AE0023F2E69429002417
:10ACC0005A3D0A08241D002010B5044608460B46CC
:10ACD000FFF77EFD28B9032208491846FCF7F2FC6D
:10ACE00028B90748FDF7E8FF0120FDF7AFFF204630
:10ACF0000449BDE81040FEF734BE00BF973E0A0885
:10AD00009B3E0A08F13B0A082DE9F74F0546084625
:10AD1000FFF75EFD0B46044618B9334A92F86C768D
:10AD200027B9284603B0BDE8F04F39E42646DFF8DE
:10AD3000C880DFF8C89001AADFF8C4A018462B49E4
:10AD40004BF070FE10B904F02FFF08E056B9012255
:10AD500001462846FFF722F9421C04461BD103B0E6
:10AD6000BDE8F08FFCF7A2FD2F28834636D80FB13F
:10AD700004F00CFFBBF1060F14D01D4901235FFA4C
:10AD80008BF291F89015E0B207F0B6F9002759461A
:10AD90004846FEF717F801AA1449002001364BF087
:10ADA00041FECFE7DAF888351B0113D5FF2C0FD011
:10ADB000E1B22846FFF71CF9E8E701372846FFF71C
:10ADC00017F90B4BF9B293F890258A42F5D8DDE7D5
:10ADD0000027F6E70748FDF769FFD7E72F2241462E
:10ADE0002846FEF7BEFDD6E7B062002413320A08FB
:10ADF000241D0020143A0A08CE3E0A08BD3E0A0867
:10AE0000B85100242DE9F04F064685B008460B46A0
:10AE1000FFF7DEFC044628B1304605B0BDE8F04F30
:10AE2000FEF7B6BD03AA3049184627464BF0FAFD97
:10AE3000A0460546DFF8C090DFF8C0A0DFF8C0B03C
:10AE40005DB92A4B3A46A1B2186E43F0EFF868BBE1
:10AE500027493046FEF785FD28E0B8F1000F06D0FF
:10AE6000B8F1010F25D03046FEF792FD1EE02846CE
:10AE700049F02AFB4946024601902846FCF722FC8D
:10AE800050B3019A51462846FCF71CFC30B3019A96
:10AE900059462846FCF716FC10B3019A2846154976
:10AEA000FCF710FCF0B13046FFF77AFB05B0BDE8C7
:10AEB000F08FBB1E294630465A425A41FFF76EF8C2
:10AEC000421C0446F2D003AA0749002008F10108F9
:10AED0004BF0A8FD0546B3E74746F4E70127F2E744
:10AEE0000227F0E70427EEE713320A08B8510024DE
:10AEF000FA3E0A08F73E0A08EE3E0A08F13E0A0842
:10AF0000F43E0A082DE9F74380460846FFF760FC47
:10AF10000B46054628B14046FEF73AFD03B0BDE8B2
:10AF2000F08301AA2D4918462F464BF07BFD2E4693
:10AF30000446DFF8A8907CB9022DECD1A7F57A730E
:10AF4000B3F57A7F21D94FF4FA634FF47A7224492A
:10AF50004046FFF731FCE1E74DB1012D10D001AAC9
:10AF60004946002001354BF05DFD0446E3E7012230
:10AF700021464046FFF712F8431C0646EFD1CDE7C5
:10AF80002046FCF793FC0746E9E7164DB8B2D5F822
:10AF900020375B689847FF2EBCEEC00A124B0BD1DE
:10AFA000F8EE407A95F89025A24212DC10EE101AC5
:10AFB0000E48FDF707FFB1E7F8EE407A03EB860392
:10AFC00010EE102A31460A48C3ED007AFDF7FAFE6A
:10AFD000A4E70134E3EC017AE6E700BF13320A0884
:10AFE00008400A08241D002020690024253F0A0883
:10AFF000183F0A08F8B507460846FFF7E9FBC8B14D
:10B000001F4B9E6A0136304634460CF073F90546F4
:10B01000F0B90134192CA8BF002420460CF06AF9BD
:10B020000546A8B9B442F4D138461649BDE8F840FF
:10B03000FEF797BC0846FCF739FC04460CF05AF9B9
:10B04000054628B921461048BDE8F840FDF7BABECC
:10B050000B4B9C6211F0D8FD2A4621460B48FDF7A8
:10B06000B1FE182C09D80A480C2101FB040090F805
:10B07000400ABDE8F84011F0FDBD0020F9E700BF2F
:10B08000D0050024343F0A08483F0A085E3F0A08FA
:10B09000C87C090838B50446114D0846FFF798FBEF
:10B0A00068B1104B93F900104B1C06D10E4B197A66
:10B0B0000E48BDE83840FDF785BEC9B2F8E708463E
:10B0C000FCF7F4FB032804D8C0B2FDF787FA294641
:10B0D000E3E7204603220649BDE83840FEF741BCBD
:10B0E000C13D0A08D0050024B8510024773F0A0862
:10B0F000873F0A0838B50446114D0846FFF768FB3C
:10B1000068B1104B93F901104B1C06D10E4B597AC4
:10B110000E48BDE83840FDF755BEC9B2F8E708460D
:10B12000FCF7C4FB032804D8C0B213F08FFB2946F8
:10B13000E3E7204603220649BDE83840FEF711BC8C
:10B14000C13D0A08D0050024B8510024733F0A0805
:10B15000823F0A08444B2DE9F74FDFF824A105464A
:10B160001A7A88468AF800205A7A93F864308AF866
:10B1700001200BB903F0A4FC00263C4CFBF72CFD8E
:10B18000B1460D23394A4146734352F803B058463D
:10B19000FCF7BCFA002841D0B9F1000F01D0FDF74F
:10B1A0006DFD59463248FDF7CDFD00222146284667
:10B1B000FEF7C8FBFDF762FD237903F01803082BA7
:10B1C00045D0102B48D02046FDF70BFE274A0D2313
:10B1D00003FB0623B3F80900FBF76CFC0746D8B164
:10B1E0002046FBF7FEF90090D7E902210244014412
:10B1F0002046FBF7AFF978B9594601901D48FDF795
:10B20000A1FD019AB96828461346009A0A442146CE
:10B21000FEF7A6FAFDF732FD09F10109013640F209
:10B220004F230D349E42ACD10020FFF720F9FF23BD
:10B230008AF800308AF80130B9F1000F11D1424686
:10B240000D49284603B0BDE8F04FFEF78ABB0B4915
:10B250002846FFF71FFFB6E708492846FFF74AFFD1
:10B26000B1E703B0BDE8F08FB85100249896090803
:10B270002A3C0A08A23F0A08CA390A08C13D0A083E
:10B28000D00500242DE9F74F074608460E4649F041
:10B290001BF9044620B1012825D132782A2A22D16F
:10B2A000B24E00254FF00D0BDFF8E092B24640F2AF
:10B2B0004F28AF48FDF7FAFC0BFB05F34846013574
:10B2C0005AF80310FDF73EFD221E3146384618BFDE
:10B2D00001220D36FEF736FBFDF7D0FC4545EBD1DC
:10B2E00003B0BDE8F08F3D2130464BF0E0FC002874
:10B2F00000F0368101460A4611F8014D202CFAD0A3
:10B30000921B0130814610F8011B2029FAD05FFA08
:10B3100082FA4FF00008DFF854B20D23524630464F
:10B3200003FB08F10BEB01045BF801100091FCF743
:10B33000C9F90546002857D10099084649F0C4F8D4
:10B34000824551D1267906F0E001402900F0CB80FA
:10B350000ED8002956D0202900F09D803846854916
:10B36000FEF7FFFA204603B0BDE8F04FFDF739BD08
:10B37000602900F091808029F0D1484649F0A4F876
:10B38000E3790546A679DB070CD52046FBF7A8FB39
:10B390000378014633B12A4648464BF0AEFC0028FC
:10B3A00040F0D880002D00F0D580AE42C0F0D280B1
:10B3B0000D23204603FB08B393F805A0FBF790FB91
:10B3C000324600214BF06CFBAA452CD82A466A492C
:10B3D00048464BF092FC30B32046FBF781FB2A46EF
:10B3E00049464BF0E9FA1EE008F1010840F24F230C
:10B3F000984592D132466149384603B0BDE8F04FD6
:10B40000FEF7AFBA06F00703042B1CD10B460A2245
:10B410004846FCF7A7F9D4F80530014683429DD38E
:10B420002046FBF773FB0D23554803FB08F85BF838
:10B430000810FDF787FC00222146384603B0BDE81E
:10B44000F04FFEF77FBA052B0FD101230A224846A1
:10B45000FCF788F9D4F8053001468342FFF67EAF49
:10B460005B4283423FF77AAFDAE74846FCF71EFAC1
:10B47000B4F80550B4F8071016F0050FAAB28BB255
:10B4800001D02AB20BB29042FFF668AF98423FF764
:10B4900065AF0146C4E765793A4A002602EBC50567
:10B4A000B246334695F808260092009AB24202D975
:10B4B000BAF1000F03D0002B3FF450AFB3E7D5F83B
:10B4C000041651F8260060B149460193FCF7D6F8FE
:10B4D000019B30B94FF0010A31462046FBF716FBBD
:10B4E00053460136E1E706F007066379013E009313
:10B4F000009BAB4297DD4846814610F8013B202B6C
:10B50000FAD02046FBF7ECFA8246042E04D8DFE896
:10B5100006F0031010161F004846FCF7C7F90AF89A
:10B52000050048462C214BF0C2FB013500F1010912
:10B53000DEE74846FCF7BAF92AF81500F1E70023E0
:10B540000A2200214846FCF70DF94AF82500E8E7F1
:10B550000123F5E732460C493846FEF702FAFDE6CC
:10B560003146384603B0BDE8F04FF3E59896090838
:10B57000B23F0A0800400A08F55E0A08CA390A08FC
:10B58000F53F0A08C87C0908C53F0A082A3C0A0892
:10B590002DE9F04F914689B00C461A4600218046AD
:10B5A0004D46FEF759FF00270646DFF8E0B0B9F137
:10B5B000000F69D02946062220464BF047FA0028A2
:10B5C0003246404613BF012100214FF0010A4FF0DF
:10B5D000000AFEF741FF0646287812F0A1FC07900A
:10B5E00010B3687912F09CFC079B4FF461714FF027
:10B5F000190C5B79EA780793AB781CFB021295F87B
:10B6000001E01CFB0313297900B14079CDF804E077
:10B61000CDE90232079B5A46CDE90410009351460A
:10B620003B464046FDF776FB207812F079FC079008
:10B6300010B3607912F074FC079B4FF461714FF006
:10B64000190C5B79E2780793A3781CFB021294F83B
:10B6500001E01CFB0313217900B14079CDF804E02F
:10B66000CDE90232079B5A46CDE9041000935146BA
:10B670003B464046FDF706FB013706340635142FDE
:10B6800095D109B0BDE8F08FCA46CDE70E400A0853
:10B690002DE9F041064686B008460F46FFF798F8B8
:10B6A000054638B100235C4901201A4606B0BDE8C2
:10B6B000F0416DE70846FCF7F9F81328044600F35B
:10B6C000A28006268DF81750544D4643781CFBF790
:10B6D00011F9074670B1FCF7E9F8C0B212F036FC78
:10B6E00040B1AB19027983F818269DF81730013361
:10B6F0008DF817303846FBF7FDF8074668B1FCF7C0
:10B70000D5F80D2809D8062303FB045383F819063E
:10B710009DF8173001338DF81730DFF8FC80B11C2D
:10B720000DF1170238464144FCF7C4F8FBF7E2F884
:10B73000074668B1FCF7BAF8012809D8062303FBCD
:10B74000045383F81C069DF8173001338DF8173029
:10B750003846FBF7CFF880B1FCF7A8F8C0B212F07A
:10B76000F5FB50B10623027903FB045383F81D2631
:10B770009DF8173001338DF817309DF817200623F8
:10B78000042A2FD103FB04530022A3F81C261DF02A
:10B79000B9FB06234FF4617603FB045595F81806B0
:10B7A00012F0BEFB95F81B2695F81A7619238046F1
:10B7B00095F81D0613FB076713FB026612F0B0FB3A
:10B7C0004379214698F80520039395F81C361448D0
:10B7D0000097CDE9016395F81936FDF7F3FA06B045
:10B7E000BDE8F081052A05D103FB0453002283F84C
:10B7F0001D26CCE7062ACAD0002308EB060248F82B
:10B8000006309380C3E713232A460649304606B024
:10B81000BDE8F041FEF7D0BFD0570024B851002456
:10B820000E400A0827400A082DE9F04F174689B054
:10B830001A460C46002181463D46FEF70DFE3A4E63
:10B8400007F190038046DFF8E8B0079394F90410FD
:10B850000023364A92F90800884260D001330C3246
:10B860000C2BF7D10C35079B0C349D42EED109B05F
:10B87000BDE8F08F29460C2220464BF0E7F800285F
:10B880004246484613BF012100214FF0010A4FF004
:10B89000000AFEF7E1FDEA7995F90430804606EBEF
:10B8A000820251464846D2F8702804922A7A06EB62
:10B8B0008202D2F870280392AA7906EB8202D2F8AB
:10B8C000702802926A7906EB8202D2F870280192FF
:10B8D0002A6800925A46FDF71DFAE279514694F91A
:10B8E0000430484606EB8202D2F870280492227A8D
:10B8F00006EB8202D2F870280392A27906EB82024C
:10B90000D2F870280292627906EB8202D2F870288F
:10B910000192226800925A46FDF7B4F9A2E7002F7F
:10B92000A8D1BA46D9E700BFC87C0908AC560024A4
:10B930002D400A082DE9F04707468AB00846FEF771
:10B9400047FF044638B10023544901201A460AB083
:10B95000BDE8F04768E70DF11C0807904E1CC8E9E8
:10B9600001000846FBF7A2FF4C4B40B21A4693F980
:10B970000410814200F08A8001340C330C2CF6D183
:10B98000002425463046FAF7B5FF064638B10135A2
:10B9900000230A22EDB21946FBF7E4FE07904FF0B0
:10B9A0000009DFF800A13046FAF7A4FF064640B3CD
:10B9B000FBF77CFF3A49002251F804CBD3B2604533
:10B9C00003D00132102AF7D100230AEB8302D2F808
:10B9D0007028904215D1B9F1020F1FD0B9F1030FB1
:10B9E00021D05A1EB9F1010FD2B212D00B2A03D8BE
:10B9F0008DF821300135EDB209F10109B9F1040FDB
:10BA0000D1D1052D15D838460AB0BDE8F047FDF76D
:10BA1000BFBF042AF0D88DF82230EBE7052BEBD816
:10BA20008DF82430E6E79A1E0D2AE5D88DF82330EC
:10BA3000E0E798E807001B4B84E807009DF8232007
:10BA4000002103EB82020846D2F8702804929DF888
:10BA5000242003EB8202D2F8702803929DF8222062
:10BA600003EB8202D2F8702802929DF8212003EBAA
:10BA700082030D4AD3F870380193079B00939DF918
:10BA80002030FDF7FFF80AB0BDE8F0870C23012550
:10BA90008DF8200003FB042474E700BFC455002484
:10BAA00038850908C87C09082D400A082DE9F04F9F
:10BAB0008BB00C460021074608921A46FEF7CCFCD4
:10BAC0000026089D4FF019094FF46178DFF8A4B003
:10BAD0000990089B002B49D029460A2220464AF0AB
:10BAE000B5FF0028099A384613BF012100214FF005
:10BAF000010A4FF0000AFEF7AFFC2A89099033468D
:10BB000006925146EA88384605922A790492EA78E4
:10BB10000392AA7819FB028202926A7819FB0282C8
:10BB200001922A7800925A46FDF7F4F822893346AA
:10BB30000136514606923846E2880A350592227946
:10BB40000492E2780392A27819FB02820292627850
:10BB500019FB0282019214F80A2B00925A46FDF753
:10BB600091F81E2EB5D10BB0BDE8F08FDDF820A006
:10BB7000DCE700BF4A400A082DE9F04380468BB05D
:10BB800008460F46FEF724FE044638B100236549F7
:10BB900001201A460BB0BDE8F04387E70846FBF7E3
:10BBA00085FE1D28054600F3B3800A268DF8274040
:10BBB0004643781CFAF79EFE044630B1FBF776FE4A
:10BBC0009DF8273001338DF827302046564CFAF780
:10BBD00091FE074668B1FBF769FE0D2809D80A23D4
:10BBE00003FB054383F890069DF8273001338DF859
:10BBF0002730DFF83091711C0DF127023846494497
:10BC0000FBF758FEFAF776FE074668B1FBF74EFEE3
:10BC1000222809D80A2303FB054383F893069DF8DD
:10BC2000273001338DF827303846FAF763FE074690
:10BC300068B1FBF73BFE0D2809D80A2303FB054337
:10BC400083F894069DF8273001338DF827309DF84E
:10BC50002730062B0CD0002309EB0602404649F89A
:10BC6000063053601381FDF793FE0BB0BDE8F083FF
:10BC70000A260023384606FB0546A6F89636A6F89F
:10BC80009836FAF737FE074640B1FBF70FFE9DF8EE
:10BC90002730A6F8960601338DF827303846FAF794
:10BCA00029FE58B1FBF702FE0A2303FB0543A3F864
:10BCB00098069DF8273001338DF827301B4B4FF045
:10BCC000FF324FF461705A600A2202FB0542B2F85B
:10BCD00098360693B2F89636059392F89436049304
:10BCE00092F893360393192392F8921613FB0101ED
:10BCF000029192F8911613FB01030021019308466B
:10BD000092F890360A4A00932B46FCF7BBFFACE74B
:10BD10001D232246074940460BB0BDE8F043FEF71D
:10BD20004BBD00BF40690024B0620024D005002450
:10BD30004A400A0827400A082DE9F04F80469146FC
:10BD40001F460C4616464FF0000BDFF820A12DEDE4
:10BD5000088B95B094ED008AB5EE408AF1EE10FAAA
:10BD60007DD0D4ED019A94ED029AD4ED038AB9F115
:10BD7000000F49D0D6ED00BA96ED01BAB4EE6B8A49
:10BD8000D6ED02AA96ED03AAF1EE10FA6CD1F4EE0C
:10BD90004B9AF1EE10FA67D1B4EE6A9AF1EE10FA0E
:10BDA00062D1F4EE4A8AF1EE10FA0CBF01210021B3
:10BDB0003A460D46404681F00101FEF74DFBB0EEDC
:10BDC0006B0A074611A8FAF70FFDB0EE4B0A079071
:10BDD0000EA8FAF709FDB0EE6A0A06900BA8FAF76A
:10BDE00003FDB0EE4A0A059008A8FAF7FDFC059994
:10BDF000069A079B039040460291294601925246BB
:10BE000000935B46FCF786FFB0EE480A11A8FAF7EC
:10BE1000EBFCB0EE690A05460EA8FAF7E5FCB0EEB9
:10BE2000490A06900BA8FAF7DFFCB0EE680A059005
:10BE300008A8FAF7D9FC069B059A00210390404612
:10BE40000292524610341036CDE900535B460BF196
:10BE5000010BFCF717FFBBF1080F7FF47BAF15B0A8
:10BE6000BDEC088BBDE8F08F0021A1E76D400A080A
:10BE70002DE9F74F07460D46DFF894A1DFF894B19E
:10BE80002846FEF7A5FC064638B100235949012093
:10BE90001A4603B0BDE8F04F4EE70522514628464A
:10BEA000FBF710FC60B9534B00221A601A611A624A
:10BEB0001A631A641A651A661A6703B0BDE8F08F30
:10BEC00004224D492846FBF7FDFB04462846002C7A
:10BED00044D1FAF70FFD80460028EED048F0F4FA7E
:10BEE000464BC2B253F8049BB9F1000F07D12A4662
:10BEF0004349384603B0BDE8F04FFDF732BD49462F
:10BF000040460134CDE90023FBF7DCFB0646DDE9C2
:10BF100000230028E6D1374A0346002115460133A5
:10BF200042F8101B082BFAD10BEBC404D4F8D8C08C
:10BF3000BCF1000F03D094F8D4E0764505DB494608
:10BF40003048314DFCF73EFF9AE70CEB061305EB4A
:10BF5000061401360FCB84E80F00EEE7FBF7A6FCD2
:10BF6000072804463DD82846FAF7C4FC064658B3CD
:10BF7000FAF7E0F91F4B012503EB041383ED000AE8
:10BF80003046FAF7B7FC064638B1FAF7D3F9194B41
:10BF9000013503EB041383ED010A3046FAF7AAFCDE
:10BFA000064638B1FAF7C6F9124B013503EB041314
:10BFB00083ED020A3046FAF79DFC38B9384603B0E3
:10BFC000BDE8F04FFDF7E4BC0546D9E7FAF7B2F952
:10BFD0000848032D00EB041484ED030A3FF455AF29
:10BFE000ECE7072332460949384603B0BDE8F04F75
:10BFF000FEF7E2BBD45A002481400A08948609085F
:10C00000CA390A0886400A08C13D0A0827400A08BA
:10C01000233D0A08C87C09082DE9F74F92460C46D3
:10C020001A46002181465646FEF716FA002580463C
:10C03000DFF864B0BAF1000F2CD03146042220465C
:10C040004AF004FD00284246484613BF0121002162
:10C0500001270027FEF700FA738880465A460193AD
:10C0600039463AF82530484600932B46FCF752FEF5
:10C0700063885A46394648460193043634F8043BEF
:10C0800000932B460135FCF7FDFD042DD2D103B002
:10C09000BDE8F08F5746EBE790400A082DE9F341E1
:10C0A00005460846FEF794FB0C46074638B10023C8
:10C0B000334901201A4602B0BDE8F041ACE73149EE
:10C0C0002046FBF7DBFA034668B92D4A4FF47A7035
:10C0D0004FF4FA610133108051800432042BF9D1FE
:10C0E00002B0BDE8F0812046FBF7E0FB03280646DE
:10C0F00041D82046FAF7FEFB074670B1FBF7D6FBA6
:10C100004FF0010804463846FAF7F4FB48B92846D0
:10C1100002B0BDE8F041FDF73BBC40F2EE248046A2
:10C12000F1E7FBF7C3FBB8F1000FF0D0A4F2EE2269
:10C1300040F2DC539A4203D8A0F2EE229A420AD986
:10C1400040F6CA0340F2EE220F49284602B0BDE88D
:10C15000F041FEF731BB0D4B00210D4A03EB860386
:10C16000A3F8BC47A3F8BE073346CDE90040084614
:10C17000FCF788FDB4E703233A460649E5E700BF2C
:10C180006C6A0024233D0A08A1400A08B06200241A
:10C1900090400A08033D0A082DE9F04F8FB0894608
:10C1A000174600211A4606460024FEF755F90DF100
:10C1B000240B0546DFF86CA059F82430594602A834
:10C1C00002933FF0FFFC57B357F824303046029AF1
:10C1D000039393422A4613BF012100214FF0010827
:10C1E0004FF00008FEF738F904A9054603A83FF010
:10C1F000E9FC04A923465246009130464146FCF72B
:10C2000089FD23460134524641463046CDF800B000
:10C21000FCF738FD202CCFD10FB0BDE8F08FB84629
:10C22000EFE700BFAF400A08F0B5074689B00846FF
:10C230000E46FEF7CDFA054638B100231949012014
:10C240001A4609B0BDE8F040A6E70846FBF72EFB0A
:10C250001F2804461DD83046FAF74CFB01462046FD
:10C260002FF074FA78B103AE0E48314600EB84002B
:10C270003FF0A8FC23460C4A294628460096FCF7C6
:10C2800001FD09B0F0BD384609B0BDE8F040FEF749
:10C2900087B91F232A460549384609B0BDE8F04052
:10C2A000FEF78ABA7C6A0024AF400A0827400A08D1
:10C2B0002DE9F04F924685B00C461A460021814682
:10C2C0005546FEF7C9F800268046DFF86CB0BAF193
:10C2D000000F2FD02946042220464AF0B7FB002841
:10C2E0004246484613BF0121002101270027FEF7DF
:10C2F000B3F8EB7880465A4602933946AB78484605
:10C3000001932B8800933346FCF704FDE3785A46EB
:10C310003946484602930435A378019334F8043B28
:10C32000009333460136FCF7ADFC102ECFD105B09B
:10C33000BDE8F08F5746E9E7B9400A08F0B507466F
:10C3400085B008460E46FEF743FA054638B100238D
:10C350001C4901201A4605B0BDE8F040A8E7084690
:10C36000FBF7A4FA0F28044623DC3046FAF7C2FA9A
:10C37000014620462FF062F9A8B104F12002124BC9
:10C380002946284603EB820393F8CF27029293F8BD
:10C39000CE270192B3F8CC370C4A00932346FCF722
:10C3A00071FC05B0F0BD384605B0BDE8F040FEF7C1
:10C3B000F7B80F232A460649384605B0BDE8F040D5
:10C3C000FEF7FAB9FC6A0024B0620024B9400A08FA
:10C3D00027400A082DE9F04F87B014461A46054653
:10C3E00003910021FEF738F84FF000080646DFF809
:10C3F00020B106234FF0000903FB08F7C037039B69
:10C40000DB5D0493002C7FD0E35D2846049A0593FE
:10C410009A42324613BF012100214FF0010A4FF02A
:10C42000000AFEF719F8059B06465A46514628466B
:10C43000CDE900934346FCF76DFC049B5A465146F8
:10C4400028460137CDE9009309F101094346FCF77D
:10C4500019FCB9F1060FD2D108F10108B8F1060FA5
:10C46000C7D1E427DFF8A8B0039BA7F1E40913F8CC
:10C4700007A0002C4AD0E35D324628469A45049333
:10C4800013BF012100214FF001084FF00008FDF714
:10C49000E3FF049B06465A4641462846CDE90093F1
:10C4A0000623FCF737FC01370623194A4146284684
:10C4B000CDE9009AFCF7E6FBEF2FD5D1039B93F86B
:10C4C000EF70ACB194F8EF8032462846474513BF71
:10C4D0000121002101240024FDF7BEFF00230C4AA6
:10C4E0002146009328460723CDF80480FCF712FC70
:10C4F0000023074A21462846009307230197FCF7AB
:10C50000C1FB07B0BDE8F08FA24696E7A046CAE798
:10C51000CB400A08F0B5054687B008460B46FEF743
:10C5200057F9044638B100231C4901201A4607B0C8
:10C53000BDE8F0404EE703AE194F02AA184918466D
:10C540004AF070FAB8B1032C04D12846FDF720FA5E
:10C5500007B0F0BDFBF7AAF902AA46F8040B39466A
:10C56000002001344AF05EFAECE7324621460D48DD
:10C57000FCF728FCECE7032CE7D1059BDDE903463B
:10C580001A4601933146E0B22FF0A2F8019B002831
:10C59000EBD12846FEF704F8DAE700BF7C6A0024F6
:10C5A00013320A08CB400A082DE9F04F89B0002663
:10C5B0000C46002107921A460746B246FDF74CFF8B
:10C5C0004FF01909079D4FF46178DFF894B0069099
:10C5D000079B3BB32946062220464AF037FA00283B
:10C5E000069A384613BF012100214FF0010A4FF08F
:10C5F000000AFDF731FF6A790690334619FB028283
:10C600005146384605922A7919FB02820492EA784B
:10C610000392AA7802926A7801922A7800925A4686
:10C62000FCF778FB627933460136514619FB0282EA
:10C63000384606350592227919FB02820492E27887
:10C640000392A27802926278019214F8062B00926B
:10C650005A46FCF717FB0A2EBAD109B0BDE8F08F95
:10C66000DF400A082DE9F04F80468BB00846894626
:10C67000FEF7AEF8074638B10023554901201A46A7
:10C680000BB0BDE8F04F8FE7524C084694F82638BF
:10C6900094F83CB794F83DA70793FBF707F90928EE
:10C6A000054600F38B8006268DF82770464309F176
:10C6B0000100FAF71FF9074658B1FBF7F7F80D2804
:10C6C00007D8A31983F8840A9DF8273001338DF821
:10C6D00027303846FAF70EF9074668B1FBF7E6F857
:10C6E000834509D3062303FB054383F8850A9DF898
:10C6F000273001338DF827303846FAF7FBF8074624
:10C7000068B1FBF7D3F8504509D8062303FB05436E
:10C7100083F8860A9DF8273001338DF82730384694
:10C72000FAF7E8F8074670B1FBF7C0F8079B8342B9
:10C7300009D3062303FB054383F8870A9DF82730B6
:10C7400001338DF82730DFF88890311D0DF1270275
:10C7500038464944FBF7AEF89DF82730062B0BD03E
:10C76000002309EB0602404649F806309380FDF7A6
:10C770000FF90BB0BDE8F08F03FB05444FF4617176
:10C78000192394F8892A13FB0212059294F8882A37
:10C7900013FB02130021104A0493084694F8873AC9
:10C7A000039394F8863A029394F8853A019394F8A7
:10C7B000843A00932B46FCF765FADAE709233A46F8
:10C7C000064940460BB0BDE8F04FFDF7F5BF00BF8E
:10C7D0003C5C0024B8510024DF400A0827400A08C6
:10C7E0002DE9F04F144689B00F461A46002106463F
:10C7F000FDF732FE0546002C00F0D58022783B780C
:10C800009A42024630460DBF4FF001084FF0000833
:10C8100001210021FDF720FE23780546994A414673
:10C820003046FCF777FA3B784146964A3046FCF7AB
:10C8300029FA002C00F0B980627830467B789A4261
:10C840002A460DBF4FF001084FF0000801210021DA
:10C85000FDF702FE637805468B4A41463046FCF7F9
:10C8600059FA7B784146884A3046FCF70BFA07F1C3
:10C87000CA0304F1CA0B4FF0020904934FF0000AF7
:10C88000822305933B78534500F39180002C00F000
:10C89000F28097F8EA30304694F8EA209A422A4625
:10C8A0000DBF4FF001084FF0000801210021FDF7F6
:10C8B000D3FD94F8EA300546744A41463046FCF709
:10C8C00029FA97F8EA304146704A304607F1EC09F8
:10C8D000FCF7D8F9002C00F0D08004F1EC034A46B4
:10C8E00004F1FC014FF001089A4633F802CB32F80C
:10C8F000020B844518BF4FF000088B42F5D188F039
:10C9000001012A463046C9B2FDF7A6FD08210546B9
:10C910005046FAF715FE5E4A034641463046FCF79C
:10C92000F9F997F8EA104846FAF70AFE584A03461A
:10C9300041463046FCF7A6F9002C00F0A0804FF0ED
:10C94000FC094FF0010807EB090104EB0900FAF7B5
:10C9500095FE09F10409002818BF4FF00008B9F549
:10C960008E7FF0D188F001012A463046C9B2FDF72A
:10C9700073FD082104F1FC00F9F7D6FF454A034690
:10C9800041463046FCF7C6F997F8EA1007F1FC007B
:10C99000F9F7CAFF3F4A03464146304609B0BDE8B1
:10C9A000F04FFCF76FB9A0463DE7A04659E7059B5D
:10C9B0003B440693002C5CD0059B06982344194603
:10C9C0000793FAF75BFE049B1A789BF800309A42B3
:10C9D0004CD1B0FA80F84FEA58184B4609F11002D2
:10C9E000F85AE15A0233884218BF4FF000089342C8
:10C9F000F6D188F001012A463046C9B2FDF72CFD78
:10CA0000627804EB090105469BF81800FAF76AFD05
:10CA100002909BF8003041461F4A30460193079B25
:10CA200000930AF10103FCF775F9049B07EB090178
:10CA30007A780AF1010A187E0BF1010B0793FAF7D5
:10CA400051FD079B4146049A09F1100902903046B6
:10CA50001B7801320193069B0492009353460E4AC1
:10CA6000FCF710F9059B093305930BE74FF000081D
:10CA7000B3E7A046D9E7A04623E7A04651E7A04682
:10CA800082E700BFF8400A080A410A0838410A084C
:10CA900050410A0867410A081F410A082DE9F04F72
:10CAA0008FB004460846B04902AA49F0BBFF0646CB
:10CAB00040B903460246AD494120FFF791FE0FB051
:10CAC000BDE8F08FAA49FAF7D9FD074620BB02AAB4
:10CAD000A54949F0A7FFFAF7E9FE0828054606D957
:10CAE00008233A46A3492046FDF766FEE7E7A24C35
:10CAF00094F83C37834202DC84F83C57DFE7064673
:10CB000004F23C77314638462BF0EAFD013694F8C2
:10CB10003C37B342F6DCEFE798493046FAF7AEFD12
:10CB20000546E0B902AA904949F07CFFFAF7BEFE3B
:10CB30000828064603D908232A469149D3E78E4C94
:10CB400094F83D37834202DC84F83D67B7E7284616
:10CB5000013531463FF00EF8082DF8D1F4E7894948
:10CB60003046FAF78BFD074600BB02AA7E4949F022
:10CB700059FF0028A3D0FAF799FE0828054603D9E3
:10CB800008233A468049AEE77B4C94F82638834226
:10CB900009DD014604F23C702BF0ECFD294604F25D
:10CBA0003C702BF0F5FD84F8265888E7774930462D
:10CBB000FAF764FD054618BB06AE6F4BDFF8A89187
:10CBC0000146B0461022304693F8267849F068FFB7
:10CBD000BD4202AA80F20E814946002049F022FFA0
:10CBE00010B93A466A490EE1FAF760FE013528F8B5
:10CBF000020BEDE7674C96E80F0084E80F005EE754
:10CC000065493046FAF73AFD054600283BD15A4BB4
:10CC10000DF11808074693F8269846464F4502AA94
:10CC200051494FF0000080F2F28049F0FBFE0146CE
:10CC300010B94A465949E6E0B2464FF0000B0322CC
:10CC400030464AF06EF8304647F03EFC584502D870
:10CC500001370436E2E79AF800000BF1010BFAF70E
:10CC600007FD0AF8010BEEE74A464D49CBE0414685
:10CC700020460135043408F1040803222BF01AFD84
:10CC8000AF42F4D11BE747493046FAF7F7FC0546B7
:10CC9000002840F0AC80384F02AA334997F83C870F
:10CCA00049F0C0FE00283FF40AAFFAF7FFFD461E28
:10CCB00001D4B04503DC434601223B4913E72A492E
:10CCC00002AA002049F0AEFE014600283FF4F7AE6C
:10CCD0004FF000080DF10C09082203A88DF814800C
:10CCE000CDE903884AF01DF803A847F0EDFB404565
:10CCF0001CD802AA1C49002049F094FE00283FF4E9
:10CD0000DEAE90F800A04FF0000897F83D97DFF8EE
:10CD1000A8B04D4502AA14494FF000007EDA49F050
:10CD200081FE024658B94A4620496CE099F8000055
:10CD300008F10108FAF79CFC09F8010BD4E7002D73
:10CD400040D11378303B092B3CD919490192FAF7AD
:10CD500095FC019A90B310465946FAF78FFC019A58
:10CD6000002838D013494EE013320A08F458002442
:10CD70007E410A0884410A08B85100248F410A08FC
:10CD800098410A08A6410A08B2410A08C4410A08A3
:10CD9000B3420A08E0590024EE410A08D3420A08C7
:10CDA000FA410A0818420A081D420A08F3420A0812
:10CDB000E1310A0830420A0829420A084FF0010806
:10CDC0004FF0FF3510460192FAF770FD0028019AE6
:10CDD00003DA214917E0A846F2E70EAB03EB45035F
:10CDE000013523F8200C94E74A461C490BE03246F3
:10CDF0001B4908E01B49002049F014FE00283FF4BD
:10CE0000F9AE3A4618492046FCF7ABFD57E649F023
:10CE100009FE00287FF428AF144C31E749F002FEE8
:10CE20000028E1D106EBC600114C082203A982308C
:10CE3000374420442BF03EFC5046FAF719FC87F8A3
:10CE4000060804EB061006A96A00023049F0B4FD9A
:10CE500087F81E8833E600BF65420A087A420A084E
:10CE60009D420A0813320A08D0410A08F0590024EA
:10CE7000F45800242DE9F04F0F46914689B0002167
:10CE800087EA09099846139A06460025FDF7E4FA51
:10CE90006FEA09030446DFF88090069328460AF0FB
:10CEA00017FA129B184230D0069BDFF870B003408F
:10CEB00014BF4FF0010A4FF0000A049310EA070371
:10CEC000284614BF4A465A46059307920AF012FABA
:10CED0004346079A5146039000903046FBF71AFFED
:10CEE000049B22463046B3FA83F14909FDF7B4FAB0
:10CEF000039B059A0446009351464346002A14BFFB
:10CF00005A464A463046FBF7BDFE0135182DC5D1BD
:10CF100009B0BDE8F08F00BF7B400A0818430A083B
:10CF200037B504460846019147F0CEFA0199054607
:10CF300002462046FAF7C6FB70B9625D1046FAF762
:10CF400081FB00B932B901352C4420460134037805
:10CF5000202BFAD003B030BD0020FBE70329F0B549
:10CF6000054685B00C46164614D80B4F3970FBF7B2
:10CF700085FE0A492846FEF78DF82246084901A891
:10CF8000FAF756FA01AB324608212846FDF792FA25
:10CF9000FF233B7005B0F0BDD0050024C13D0A0859
:10CFA000773F0A080329F0B5054685B00C461646BA
:10CFB00014D80B4F7970FBF761FE0A492846FEF73B
:10CFC00099F8224608496846FAF732FA6B46324623
:10CFD00010212846FDF76EFAFF237B7005B0F0BDE7
:10CFE000D0050024C13D0A08733F0A0810B5114B53
:10CFF00086B0114904460493104B11480393114B1A
:10D00000114A0293114B0193114B0093114BFBF703
:10D0100099FEFBF733FE10491048FBF7D3FE3CB1F5
:10D020000F4A1049104806B0BDE81040FBF7CABED1
:10D0300006B010BD5F430A0829430A0864430A0882
:10D0400034430A086E430A081F430A0877430A0854
:10D05000FF340A08C751002483430A088B430A0897
:10D06000D4EC0908CCEC09089C430A080120BDE770
:10D070002DE9F04F3E4C87B00A4600210646FDF7E9
:10D08000EBF905903B4A2378608802EB8303D3F8E1
:10D0900074ACF9F70FFD8368C1680493364B93F8BD
:10D0A0006420002A4BD0DDF81080049100272179FC
:10D0B0006279049B07FB012213F80290B8F1000F7C
:10D0C0003FD018F802504D45059A304607F1010748
:10D0D00013BF012100214FF0010B4FF0000BFDF7B2
:10D0E000BBF905907DB305F00F022D095346594653
:10D0F000403502923046214ACDE90075FBF70AFE21
:10D10000B9F1000F2AD009F00F024FEA191953465E
:10D110005946029209F140023046CDE90072174AA1
:10D12000FBF7B0FDA279012A38BF0122BA42BEDC6A
:10D130000834134BA342A5D107B0BDE8F08F904649
:10D14000B4E74546BFE7B8F1000FD9D053460D4AC2
:10D15000594630460097FBF7DDFDD1E77306E1D471
:10D160005346084A594630460097FBF78BFDD9E7EE
:10D1700034880908C87C0908B8510024C9430A0842
:10D180003C890908DF430A0838B50C4B0C4603EB11
:10D19000C0050B4895F86C2B03EB8203D3F8741C85
:10D1A000FBF7D0FD95F8723B33B1611C0548C9B25D
:10D1B000BDE83840FBF7C6BD38BD00BFC87C0908D4
:10D1C000DF460A0885320A0873B50E46114905463E
:10D1D000FAF754FA18B93070012002B070BD2C78FB
:10D1E000602C8CBF613C413C072C10D801350123D9
:10D1F0000A2201A92846FAF7B5FA019B9D4206D0FA
:10D200000F2804D8013440EA04143470E4E7002005
:10D21000E3E700BF7B310A082DE9F04F714D0A4664
:10D220000021824605F1900B2DED028B8BB0FDF7AE
:10D2300013F9814600266C4B93F86440AB7AB342F5
:10D2400000F393801035AB45F4D140F21620F9F786
:10D2500031FCD0E902530CB12C461D460DF1100BE8
:10D26000002715220021584649F01AFC2E78002E7E
:10D2700043D069783046039105F0D8F995F902302A
:10D2800008EE100A5A1C029353425341002C00F03E
:10D29000A6800022039914F802C0A018B44540F0FB
:10D2A0009A8090F90280029A424540F0928042783A
:10D2B0008A4208BF0123012203F001030BF8072073
:10D2C0004A4683F0010150460393FDF7C5F8039BDE
:10D2D00081464CB1454A18EE101A3046CDE900A2FD
:10D2E0004246F9F7A1FB039B414A18EE101A30465B
:10D2F000CDE900A2029AF9F797FB01370335152F04
:10D30000B4D16CB304F13F06384FDFF8E4801BF86A
:10D31000013B02930BBB2078F8B194F90220013253
:10D320001BD0617805F082F905464A460121504636
:10D33000FDF792F894F90220029B29468146207855
:10D34000CDE900A7F9F770FB2078029B4FF0FF3280
:10D350002946CDE900A8F9F767FB0334B442D6D1DA
:10D360000BB0BDEC028BBDE8F08FE888F9F7A2FBAB
:10D37000D0E902230CB114461A46297A6B7A06FBCF
:10D38000013312F903800CB3E756B8454A465046BC
:10D390000DBF01230023012100210293FDF75CF85A
:10D3A000029B814644B1114A31462846CDE900A28C
:10D3B0003A46F9F7EDFA029B0D4A31462846013606
:10D3C000CDE900A24246F9F7E3FA34E74FF0FF3720
:10D3D000DBE700236FE703323F2A7FF45CAF4FF0B7
:10D3E000FF386DE7FC050024B8510024158D0408B2
:10D3F000858C04082DE9F04F80468BB008460D4619
:10D4000047F062F8024670B3A4492846FAF75AF981
:10D41000044640BBFBF732FCA14DA248A24FFBF7EC
:10D4200045FCA24E1420DFF8CC823EF0B7FBE110A1
:10D4300004F0070238460131FBF784FC2B7F6A7F3A
:10D4400006EB8303D3F8741C4AB19948FBF7BAFC86
:10D4500001342435102CEAD10BB0BDE8F08F4046E2
:10D46000FBF7B0FCF4E7284605AA924949F0DAFA3E
:10D47000054620B901464120FFF7CEFEECE78E4974
:10D48000FAF7FCF820B98D494046FCF76AFAE3E761
:10D490008B4E0927002431682846FAF7EFF8002858
:10D4A00008BF3446013F06F11006F4D154B985494E
:10D4B0002846FAF7E3F828B12A4683494046FCF7A4
:10D4C00050FAC9E7002005AA7A498DF8130049F0FF
:10D4D000A9FA0546002C3BD080B1FAF7E7F9461EC1
:10D4E00009D4A37A9E4206DAE2684AB1012303FA1C
:10D4F00000F0104204D12A467449DFE7744DFAE780
:10D50000E0880027F9F7D6FA7249039791F864107A
:10D51000D0E90232002908BF1A46217A637A06FB55
:10D52000013302EB030B12F903A005AA61490020A5
:10D5300049F078FA8146A0BB0123674944B39BF9BF
:10D5400000202046CDE900313146F9F721FA83E782
:10D5500068B10DF11301FFF737FE28B19DF8136094
:10D56000304602F061FA20B92A465C49A6E7584DD8
:10D57000FAE73046A346F4F7A3FB8246304605F0AF
:10D5800041F803903046264605F006FD0746CCE7F5
:10D59000CDE90031524639469DF81300F9F744FAB7
:10D5A0005AE74549FAF76AF8054670BBACB1F6B2DE
:10D5B0004B4F6AB231462079F4F74CFB00283FF418
:10D5C0004BAF028829460378384601350093C2F3F1
:10D5D0000323120BFBF7F6FBEBE7414C102D3868E9
:10D5E00079796AB23FF438AFF4F786FB00283FF44C
:10D5F00033AF028829460378204601350093C2F3F1
:10D600000323120BFBF7DEFBE8E736494846FAF73F
:10D6100035F800283ED04846FAF748F9054642B2A8
:10D620006CB1F1B22079F4F715FBD8B9CDF80090C0
:10D63000731C22682C494046FCF793F90CE7EBB2C7
:10D64000386879790F2B09D99DF8133027491A09C1
:10D65000CDF8009003F00F034032ECE7F4F74CFBF9
:10D660000028F1D006AF28463946F9F79BFF08A9F4
:10D670005046F9F797FF55454AD06DB2002C3BD084
:10D680008BF8005008AB0097721C21681848FBF714
:10D6900099FBE1E64FF0FF35E4E700BFF3430A08EA
:10D6A0005C020024F8430A080E440A08C87C0908F2
:10D6B00094490A0813320A08CE360A081F440A0899
:10D6C000FC05002433440A0837440A0846440A0883
:10D6D000C13D0A08B8510024858C040856440A0844
:10D6E00068440A08043A0A0889440A08AC440A084B
:10D6F000D4440A0845360A089DF81320039B1109F3
:10D700000C489D7002F00F0208AB40310097BEE755
:10D7100034B108AB721C21680748FBF753FB9BE64A
:10D720009DF8132008AB0548110902F00F024031A3
:10D73000F3E700BFF7440A081F450A083A450A08FC
:10D74000224BB0F5FA6F1A680346A8BF4FF4FA638C
:10D75000B3F57A7FB8BF4FF47A73D20416D540F28E
:10D76000DC52904215D040F2DB5207EE903A9042E4
:10D77000F8EE677A1FD8DFED166A9FED167A77EE1E
:10D78000E67A9FED150AA7EE870A7047B0F57A7F13
:10D7900002D89FED120A704707EE903ADFED106A4B
:10D7A0009FED107AF8EE677A9FED0F0A77EEE67A32
:10D7B000A7EE870A7047DFED0D6A9FED0D7A77EED1
:10D7C000E67A9FED0C0AA7EE870A704740570024BF
:10D7D00000007A44D62000C000E08244000000002F
:10D7E00000407A44661000400000404200A0BB4464
:10D7F000D62000400000834410B584464FEA810ED5
:10D80000102312F4004F4FEA420214BF0E240724E3
:10D81000013B92B2CCF80040F444F2D100EB81120B
:10D820008C010351122042F8213010BD10B58446FE
:10D830004FEA810E0424130B013C4FEA021203EB62
:10D84000430392B203F11803CCF80030F444F2D150
:10D8500000EB01130A018450062043F8214010BD5B
:10D86000704700BF704700BF034B00EB400003EB65
:10D87000C000407C704700BFB810002000233D224C
:10D88000437002708370C370704700BF704700BF61
:10D89000704700BF0020704701207047704700BFED
:10D8A000704700BF704700BF704700BF9FED010A7F
:10D8B000704700BF000000000020704703681B692C
:10D8C00018470B4B002130B593F9002001315D78EA
:10D8D0000433092AC8BF1E3A092900EB0204E57285
:10D8E00013F8025C855413F8012CA275ECD130BDFD
:10D8F0009CB40908002383700370C37043707047A1
:10D90000D0F82C3193B1D0F8C82112685368D0F800
:10D9100044219A4210B405D2C0685DF8044B10440B
:10D92000C01A7047D01A5DF8044B7047D0E907233E
:10D930009A4201D3D01A7047C0681044C01A704789
:10D94000D0E90932934212D3A3EB020CD0F8303164
:10D950000169A3B1D0F8C421481E126853689C44E1
:10D96000604502D9A0EB0C007047002070470169A8
:10D970000B44A3EB020CD0F83031002BEAD1481E47
:10D98000A0EB0C00704700BFD0F8303113B190F815
:10D99000E0017047D0E90903181AB0FA80F0400995
:10D9A000704700BFD0F82C21034610B472B1D0F8F4
:10D9B0004421C1685C69881A013A205C08BF0A46A4
:10D9C0005DF8044BC0B2C3F844217047006A5C693B
:10D9D000411C205CDC68C0B2A14238BF0A465DF839
:10D9E000044B1A62704700BFD0F8E43103B1184706
:10D9F000704700BFF8B590F8F931012B1CD0002A10
:10DA0000164619DD05460F460269436AD41AA8690D
:10DA10003946B4421844A8BF34462246361B48F063
:10DA2000CBFF686A2A6927440444002EB4FBF2F352
:10DA300002FB13436B62E9DCF8BD00BF38B5D0F8D8
:10DA4000E43104460D460BB19847B8B1636AA26948
:10DA5000D554636A21690133D4F830218B4228BF41
:10DA60000023636222B12046BDE83840F5F7B8BA1A
:10DA7000D4F85021136843F08003136038BD00BF11
:10DA800070B5094C236873B10546002606E0996815
:10DA90001A681E7321609047236823B15A6818469C
:10DAA000AA1A002AF3DA70BD8078002470B5204CE1
:10DAB0002378012B00D070BD1E4B1B68002BFAD0C1
:10DAC0001D4D2B6828465B6898470028F3D01B4BF8
:10DAD0001B4E1A68338892889A4219D3194900223A
:10DAE000284609684968EA622A6803FB01F1D3689D
:10DAF00098473388144A013352683380002ADAD0B9
:10DB0000116893884A69134218BF1B048B6170BD6A
:10DB10000D4B00225B682270002BCCD00B491A6899
:10DB200009789B88890748BF1B04936170BD00BFBB
:10DB3000A42A0024181E00241C1E00249C2A002451
:10DB4000A22A0024982A0024581E0024641E0024BF
:10DB500008B5294B1B68DB041ED5B5EE400AF1EE73
:10DB600010FA26D0DFED257AB4EEE70AF1EE10FACE
:10DB70001FD49FED237AB4EEC70AF1EE10FA2AD82B
:10DB800070EE677A9FED1F7A9FED1F0AA7EE870A56
:10DB900048F094F980B208BDDFED187AB4EEE70AD8
:10DBA000F1EE10FA0BDA9FED190A48F087F980B20E
:10DBB00008BD9FED170A48F081F980B208BD70EEEC
:10DBC000677A9FED147A9FED140AA7EE870A48F052
:10DBD00075F980B208BDDFED117ADFED116A70EEE4
:10DBE000677A9FED107AA7EEA67AB0EE470A48F062
:10DBF00065F980B208BD00BF4057002400004042D4
:10DC000000E0824466BEFFBE0060BB4400007A4470
:10DC10000080BB4438DFFF3E00407A44000083446C
:10DC200066BEFF3E00A0BB44F8B5C24B1D6815F0B0
:10DC300004072DED048B40F0EA809FEDBF9ABF4CA6
:10DC400015F0200505D094F8D05015F0020540F0ED
:10DC5000908094F80831DFEDBA8A13F0010340F0A8
:10DC60009B8094F80921002A7ED1D4ED437A9FED60
:10DC7000B56ADFEDB56A67EE867A94ED457A39EEDE
:10DC8000477AE9EE267A84ED447AC4ED437A65B1A9
:10DC9000012194F81C21D4F8D4308A4284F80A1166
:10DCA000C4F8183118BFC4F81031A84B1E780E2ED6
:10DCB00000F0FF8000279FEDA08A94ED4B7AD4ED11
:10DCC0004C6A38EE478AD4ED4A7AA6EE887A37EE67
:10DCD000676A84ED4B7AE6EE867AC4ED4A7AC4ED43
:10DCE000497A0FB1C4ED447A94ED4F7AD4ED4D6A80
:10DCF000F0EE475A9FED965A77EEE66AC4ED4D7AFC
:10DD0000F0EE477A94ED506A94ED4E0AD6EE855ABD
:10DD1000E6EE257A37EEC07AC4ED4F7AA6EE070A12
:10DD200084ED4E0A48F0CAF802B282EAE273A3EB2D
:10DD3000E2739BB2092B68D9002AACBF0A380A30BB
:10DD400005B20E2EA4F844514AD0242E09D1DFED9D
:10DD5000817A94ED440A20EE270A48F0AFF87E4B12
:10DD60005880BDEC048BF8BD84F80A3184F8093181
:10DD70007BE7D4ED387AB4F8E430F8EEE77AC4ED16
:10DD8000357A002B64D1DFED6E8A94F808310125D5
:10DD900013F001033FF465AF94F80931002B4FD025
:10DDA000D4ED459A39EE698A002D35D094F80A31C0
:10DDB000012B01D0002F68D1002B40F0B280634AC4
:10DDC00016780E2E00F0B280002F35D094F81C315A
:10DDD000B0EE489A012B7FF670AF94ED498A6CE75C
:10DDE000DFED5B7A5C4C68EEA78A9FED5A0A29EE5C
:10DDF000000AFDEEE88A18EE903A238048F05EF8BB
:10DE0000E5806080BDEC048BF8BD002599E74B4CA4
:10DE1000012794ED319A13E74C4B1E780E2E24D037
:10DE200094F80A51DFED448A002DCDD094F81C31CE
:10DE3000002B4ED0022BC7D1B0EE489A0127CCE779
:10DE4000D4ED439A0123C4ED459A84F80931A9E73A
:10DE500007EE903ADFED3E6A9FED407AF8EEE77A02
:10DE6000C6EEA78AC8FEC78A8FE7D4ED497A94F830
:10DE70000A51DFED318A9FED370A0E2627EE800A20
:10DE800048F01CF8344B9880CEE7D4ED357A012366
:10DE900037EEC90A84F80A3130EE290A84ED460AC1
:10DEA0002A4B77EEC07A1E78C4ED497A0E2EBDD18A
:10DEB000E1E7D4ED357A00279FED297A264B67EE0E
:10DEC000877A9FED1D8AFDEEE77A17EE902A9A80F9
:10DED000F3E6002FB0D094ED496A94F81D3136EE88
:10DEE000499ADFED206A07EE903AB8EEE77A79EECC
:10DEF000297AF0EEE77A67EE877AF4EEE67AF1EEC9
:10DF000010FA03DD68EEA66AC6EEA78AF7EE007A7D
:10DF1000B0EE489A77EEE87A27EE888AA6EE288A4D
:10DF2000CBE6D4ED357A94ED460AB9E7D4ED497ADB
:10DF30001D46A0E7F0600024000000008078002467
:10DF40009A99993ECDCC4C3FCDCC4C3EA81E002496
:10DF50000000C842CDCCCC3DAC1E00246666663FB6
:10DF60000AD7233C00401C466E4B1B782DE9F04F2E
:10DF700087B0002B00F0CF806B4D4FF000086B484E
:10DF8000A968FAF71FFF69686948FAF71BFF694B30
:10DF90006948DFF8DCA1D3E90031C91A674BD3F82F
:10DFA0004821B1FBF2F2FAF70DFFFAF767FE644879
:10DFB000FAF77CFE6348FAF779FE634B5FFA88F460
:10DFC0001B78A34221D8614C0025614FFAF756FE19
:10DFD0002646013556F8041B3846FAF7B3FE162DCF
:10DFE000F7D101255A4EFAF749FE234661680135FB
:10DFF00030461B680434C91AFAF7A4FE162DF4D172
:10E0000007B0BDE8F04FFAF739BE524B14264FF077
:10E010003C0B671C03EB840306FB045693ED000ADC
:10E0200047F04CFF96F81EE081B2B6F80E901EF055
:10E03000010F80B214BF52222D221EF0020F049055
:10E04000504614BF54232D231EF0040F07EE903AC0
:10E0500014BF56232D231EF0080F009317EE903A9D
:10E0600014BF4FF0430C4FF02D0C1EF0800FCDF875
:10E0700004C014BF4FF0530E4FF02D0EB1FBFBF157
:10E080000591642101FB09F1CDE902E13946FAF776
:10E0900059FEB37FDB073AD55C232F4A6343D1187F
:10E0A000D05891ED010A70B1B8EE400ADFED2B7A3D
:10E0B00020EE270A07EE900AF8EE677A80EE270A2C
:10E0C00047F0FCFE00B2642290FBF2F102FB110269
:10E0D0002348FAF737FE1421224808F1010801FB12
:10E0E000075701FB0454F988628A0491218B02F0DE
:10E0F000030392080391E18A0291A18B0191A18A05
:10E10000009119214B43218AFAF75CFE55E7164826
:10E11000FAF794FDDFE7154807B0BDE8F04FFAF7CE
:10E12000C5BD00BF040000205814002056450A0851
:10E1300066450A08701C00207D450A088078002486
:10E14000AA450A0806460A08B42200200415002041
:10E15000B6460A08383700207811002000401C46D7
:10E160007F460A0894460A088B460A08BA460A08F7
:10E1700062460A082DE9F84F06460C461E4D382720
:10E180004FF00008DFF87890DFF878A02046FCF721
:10E190001FFBD5F800B048B921465846F9F7B6FA42
:10E1A00020B921466868F9F7B1FA80B15846FAF704
:10E1B00045FD696811B15046FAF7C4FDA96811B16F
:10E1C0004846FAF7BFFD4FF00108FAF757FD013F47
:10E1D00005F11005DAD12046FCF7FAFA48B9B8F192
:10E1E000000F06D1224630460449BDE8F84FFBF740
:10E1F000B8BBBDE8F88F00BFC0B40908E2460A0802
:10E20000DC460A08D6460A088160F4F7B5BC00BFB0
:10E210000171F4F7B1BC00BFF8B590F8F931012BEA
:10E220006BD0D0F830310446002B67D0EFF3118566
:10E23000502383F31288D0F830311B6803F00103B8
:10E24000002B57D1D0F8D021D0F8D4110A4302F0D6
:10E250002102212A4ED0D0E909218A425AD054D92C
:10E26000531A9BB2A262002284F8E021D4F8D02194
:10E27000202A3FD1A26951183CD0B3FA83F2520947
:10E28000002B37D094F8CC01012833D02120A4F8FA
:10E29000A6314FF0010CC4F8D821C4F8D001D4F84D
:10E2A000C401C4F8A011A4F8A43184F8CCC100289A
:10E2B0003AD0234E90F834E0C663224EE64502651C
:10E2C0000664214EC6640CD090F83560D4F85071C5
:10E2D000664580F834C021D04FF4006380F83420C4
:10E2E0004365102100222023C4F8D81184F8CC21E2
:10E2F000C4F8D031EDB285F31188F8BDD0F85021C3
:10E30000136843F080031360F8BD00691A46431A8E
:10E310009BB2A7E7012380F8E031EBE707F1280281
:10E3200038F0E4FC0028DCD1D4F850310022402140
:10E33000196284F8CC219A6842F080029A60D9E789
:10E34000394A08085D4A0808994A08082DE9F84F33
:10E35000B64C804694F80831DB072DED028B79D559
:10E36000B34B94F84C51B34E1F88012D5FD0022D52
:10E3700038D0002D44D094ED588AF37B33B1B38963
:10E3800023B1AD4B1B78002B40F0EA8094F84D216F
:10E39000AA4238BF2A46337A632B07D8022D00F0F1
:10E3A000FF8094F85811002940F01181A34BB0EE82
:10E3B000487ADFEDA36A1A70B17BD4E95C30C4F807
:10E3C00074311B1A07FB03F307EE903AF8EEE77A75
:10E3D000A7EEA67A84ED587A002970D1BDEC028BA5
:10E3E000BDE8F88FB4F85031BB42C4D2954B01253B
:10E3F00094ED588A1B6884F84C51C4F86431BCE72A
:10E40000B4F85231BB421ED38E4BD4F864111A6853
:10E41000F37D521A03EB830303EB8303B2EB830F09
:10E42000A9DB012594ED588A84F84C51A5E7B4F88E
:10E430005431BB4280F0A080B4F84E31BB4202D2CE
:10E44000002584F84C517F4B94ED588A1B68C4F822
:10E45000643192E794F84C51DFF8D491EB1E012B14
:10E4600039D9B9F80800C0F30B0046F059FD092866
:10E4700040F3C5806F4EB9F80070F3889F4203D314
:10E480003288BA42BFF471AFB7EB430F3FF76DAFBD
:10E490000323DFED6D7A684A84F84C31B0EE678A69
:10E4A00084F84D310023C4ED587A1370A4F84E312E
:10E4B000A4F85031A4F85231A4F8543196E0012A5E
:10E4C00000F09680022A89D10720BDEC028BBDE8BE
:10E4D000F84F0EF0CFBB574EB9F80070F3889F424B
:10E4E00002D33288BA4202D2B7EB430F79DDB9F8D2
:10E4F0000800C0F30B0046F013FD092840F3938099
:10E500000022357D84F84C2184F84D21002D00F047
:10E51000A180494B1D702B46154699B2B28873886D
:10E5200012FB01F213FB01F3717C92B29BB28A429F
:10E53000A4F84E21A4F8503140F2D080521A92B281
:10E540008B42A4F8522140F2C7805B1A9BB2A4F818
:10E550005431642384F859310023C4F85C3104E752
:10E5600010F020F900284ED102232A469D4284F85B
:10E570004D3138BF1A460EE7324BD4F864111A6891
:10E58000337E521A03EB830303EB8303B2EB830F57
:10E59000FFF6F1AE022594ED588A84F84C51ECE672
:10E5A00094F8580198B90121C4F85C81804684F838
:10E5B0005811C3F16403254908FB03F381FB0301F0
:10E5C000DB17A3EBA153643384F85931EEE6D4F89A
:10E5D0005C011F49A8EB00088845EADB84F8593143
:10E5E000E4E6032D40F0818094ED588A0325C4E6CB
:10E5F000BDEC028B0820BDE8F84F0EF03BBBB9F82C
:10E6000000700C4EB1E6337C834207D301232A46C7
:10E610009D4284F84D3138BF1A46BCE600232A4695
:10E6200084F84D31B7E6032DDED0A4E680780024CF
:10E6300038680024445700243768002436680024D2
:10E64000ACC52737501E0024000000006BCA5F6B6A
:10E650008096980032882A4BDFF8B0A01B68B7FB81
:10E66000F2F2013293F96C10082A28BF0822D3B2C3
:10E670008AF8003000293FF450AF91423FF44DAF8B
:10E68000204991F800E00EF1010101F003018E45EF
:10E690003FF443AF4FF0FF3C4FF0A40B09E018B933
:10E6A0003CEA2C0C28BF8C46013101F003018E4559
:10E6B00016D015480BFB010090F96C008242EED198
:10E6C0008C465FFA8CF0F9F789FF9AF80030B9F8B8
:10E6D000007094F84C5120E7002338E700222FE720
:10E6E000BCF1FF3F3FF419AFEBE7B9F80800C0F306
:10E6F0000B0046F015FC09283FF7BDAE3BE600BF16
:10E70000B8550024C0510024F85200243768002472
:10E710002DE9F041CF4CA36820469847002800F02F
:10E720009380B4F90E30A17D06EE903AB4F9103022
:10E73000092907EE103AB4F91230F8EEE66A07EE4E
:10E74000903AB8EEC77A4FF00103F8EEE77AC4EDDD
:10E75000126A84F8543084ED137AC4ED147A75D0BB
:10E76000BD4D04F1480022F0B3FBAA8DAB6A002A2C
:10E7700077D1BA4A1268520700F1AE80B3F900208F
:10E7800094ED126A06EE902AB3F90220B3F9043030
:10E7900007EE102AF8EEE66A07EE903A2B88B8EEFC
:10E7A000C75A94ED137AF8EEE75AD4ED147A76EE60
:10E7B000666A37EE457A77EEE57AC4ED126A84ED43
:10E7C000137AC4ED147AFBB3D5ED024AD5ED085A9D
:10E7D00076EEE46A95ED055A95ED033A77EEE57A23
:10E7E00037EE457AD5ED063AE6EE834A95ED094ACD
:10E7F000F0EE656A95ED016AA7EE235A95ED047A6D
:10E80000E4EE276AD5ED077A34EEC62AC5ED024A52
:10E8100075EE472A85ED055A76EEE75AC5ED086A8A
:10E82000F0EE466AA2EEA37AE4EE257AE3EE026AFF
:10E8300085ED047A84ED137AC5ED016AC4ED126AA0
:10E84000C5ED077AC4ED147ABDE8F081824D04F17C
:10E85000200104F1480022F0D5FAAA8DAB6A002A03
:10E8600087D0B2F5C87F00F0A9807D49002694EDDD
:10E87000127A0020D1ED5E6A012AD4ED137AF8EE07
:10E88000E66A94ED146AA66476EE876A91ED5F7A83
:10E89000B8EEC77AFDEEE66A37EE277AD1ED607AF8
:10E8A000C1ED5E6AF8EEE77A1880BDEEC77AE664DD
:10E8B00077EE867A81ED5F7A5880FDEEE77A2665FD
:10E8C000C1ED607A988000F09A80013AAA85634A87
:10E8D000126852077FF552AF614EB6F88421322A92
:10E8E0002DD0002A40F0868096F8A221002A3FF41D
:10E8F00045AF06F5CA705B4F4FF0000C07C887FBA9
:10E90000028ED21786F8A2C1C2EB2E12A689921BE4
:10E910009A8087FB0062C017C0EB221087FB01279B
:10E92000C91701221880C1EB271159804E4BA3F85B
:10E930000EC0C3F80A20F9F7F3FFAB6A1EE71A68A6
:10E94000DFED4A7AC6F88821B3F90420A6F88C21B5
:10E95000454AD268C6F8902194ED127A0020002131
:10E9600077EE877AA0641980B6F88421FDEEE77A05
:10E97000322AC6ED657A7BD096ED667A012AD4ED0F
:10E98000137AB8EEC77AD4ED146AE064598037EE92
:10E99000277AD6ED677A2065F8EEE77A9980BDEEA2
:10E9A000C77A77EEA67A86ED667AFDEEE77AC6ED4F
:10E9B000677A6ED0013AA6F8842195E7D4ED126A01
:10E9C000002094ED137A0021D4ED147AFDEEE66A6E
:10E9D000BDEEC77A224EFDEEE77AA064C6ED5E6A10
:10E9E000198086ED5F7AE0645980C6ED607A206513
:10E9F00099806AE7D6ED657AF8EEE77AACE717EE2C
:10EA0000907ADFF860C016EE906A17EE101AC837D9
:10EA1000C836C8314FEAE77E8CFB0787CEEBE71795
:10EA2000B4F80CE0A7EB0E079F808CFB06E7F61707
:10EA3000C6EBE7161E808CFB016CC917C1EBEC110D
:10EA40005980094BC3F80A20D881F9F769FFAA8DCC
:10EA5000AB6A3AE7482400201024002040570024E5
:10EA6000807800241F85EB517C57002400000000B3
:10EA700094ED137AD4ED147ABDEEC77AE064FDEE1E
:10EA8000E77A5980206586ED667A9980C6ED677AC7
:10EA900090E70B2086F8A12186F8A0110EF0EAF885
:10EAA000AB6AD6F88821D6F890111A60B6F98C2195
:10EAB0009A80024AD160B6F884217BE77C57002413
:10EAC00038B5074C074DAC4203D3074B01221A70EF
:10EAD00038BDA288D4E9021047F06EFF1C34F2E77B
:10EAE0005CB50A0890BD0A081C520024224B30B5C0
:10EAF00083B09A7901906AB393F82630DFED1F6AEC
:10EB000007EE903A1E4B1F4CF8EEE77A1D7886EE22
:10EB1000A77A84ED187ADDB11B4BDDED017AB3F8ED
:10EB2000AE31F8EE670ADFED197A00EE103A60EECA
:10EB3000A70AB8EE400AF8F793F804F12003002181
:10EB400003EBC5021960083303ED010A9A42F9D1BB
:10EB500003B030BD0E4A12681201F9D593F8263081
:10EB6000DFED066A07EE903A064BF8EEE77A86EE9E
:10EB7000A77A83ED187AEBE78C2900245555554088
:10EB8000B42200203837002080780024BD37863535
:10EB900040570024A54B1B78002B00F0B2802DE9D4
:10EBA000F04FA34E83B096F80491B9F1010F02D053
:10EBB00003B0BDE8F08F9F4B9F4F1B6893F8345014
:10EBC000002D6ED09D4B0022DFED9D6ABE4697ED75
:10EBD000187A904693F800B040F6FF7A67EE266AFE
:10EBE0009FED986A3346984C019200971CE000F420
:10EBF0007061B1F5006F00F0B38000F29380B1F561
:10EC0000806F00F0DB80B1F5C06F7BD1C0B24CF0FB
:10EC1000080C988283F81EC0013214330EF1040EE2
:10EC20000234D2B2AA422AD093F81EC09889BCF10D
:10EC3000010FDCD1504500F0D080C0F30801400A3C
:10EC400001FA00F081B2002900F0BF807F4F80B24E
:10EC5000BBF12D0F07EB5101B1FBF0F000F0D780B5
:10EC60004FF6FF718842D7D007EE900A0199F8EE6F
:10EC7000E77A014480B2019167EEA67AB3E0009F83
:10EC8000B8F1000F0DD0DDED017AB8EE677A07EE2E
:10EC9000908AF8EE677A27EE267AC7EE276AC7EDE4
:10ECA000196A6B4BDFED6B6A1878C7ED1A6A10B3FF
:10ECB000694A97ED185A5E4902EB8000A2F14803B9
:10ECC000CC89083353ED037A143107EE104A53ED23
:10ECD000025AB0EE676AB8EEC77A97EE056AE5EEBB
:10ECE000867AE2EC017A904243ED037AC6FEE76A47
:10ECF000E6D1C7ED1A6A022386F8043103B0BDE8F5
:10ED0000F08F7047B1F5007F31D14CF0020CC1B2E9
:10ED100083F81EC093F81FC019828C45BFF47CAFE6
:10ED2000D87779E7B1F5406F13D0B1F5606F06D1B0
:10ED3000C0B26CF07F0C988383F81EC06CE7B1F50D
:10ED4000206F14D1C0B24CF0200C188383F81EC081
:10ED500062E7C0B24CF0400C588383F81EC05BE7FA
:10ED6000C0B24CF0100CD88283F81EC054E7504556
:10ED700046D0C0F30801400A01FA00F081B221B385
:10ED8000324F80B2BBF12D0F07EB5101B1FBF0F018
:10ED900049D04FF6FF7188423FF43EAF07EE900A2C
:10EDA0000199F8EEE77A014480B2019167EEA67A04
:10EDB0004CF0010CD88183F81EC017E0C0B24CF0B3
:10EDC000040C588283F81EC026E7BBF12D0F7FF498
:10EDD00023AF4FF0FF3121801EE7BBF12D0FF0EE86
:10EDE000467A08D00020D88183F81E9008F10108E7
:10EDF000CEED007A10E74FF0000100202180F2E70D
:10EE0000BBF12D0FF0EE467A08D00020D0E74FF688
:10EE1000FF71208088423FF4FFAE25E74FF00001EC
:10EE200000202180C4E72080B3E700BF0400002059
:10EE3000581400204424002038370020A81E002445
:10EE40000000704200000000AC1E0024C027090032
:10EE5000B4220020FFFF7F7FA437002010B5437B42
:10EE600004468268581C6073D154627B237B9342B2
:10EE700000D802B910BD2368D4E9010198470023E6
:10EE8000637310BD427B42B1036810B50446D0E9FC
:10EE9000010198470023637310BD7047F0B5066801
:10EEA00095B0044617463578012D08D0022D02D1C1
:10EEB000326A002A36D00025284615B0F0BD96F9F2
:10EEC00004000328D4BF00250125B0F1FF3F08BF8F
:10EED00045F00105002DEED1642606FB00F0434EFF
:10EEE00006EB000C18303044DCF81860002EE3D03C
:10EEF000FF29247964D09CF85920202A50D19AB255
:10EF0000002B49D09CF85830012B49D000923B4649
:10EF10000A4661003FF0A6FD002841D101252846A0
:10EF200015B0F0BDCDE90A730DF10F0361F07F015B
:10EF30000592049301238DF81C2006938DF8303040
:10EF40008DF8443000230D92109212928DF80F101C
:10EF5000CDE908220022CDE90E23EFF3118510231D
:10EF600083F3128803681B6A002B37D004A8069B22
:10EF700002461BB1D3691432002BFBD1336ABBB1FB
:10EF8000996839B9934213D0196879B15B68996867
:10EF90000029F7D01433F3E74FF40073CCF85C305A
:10EFA000134A138801339BB2138085E7C3E90040FD
:10EFB000EDB285F311882268136A002BFCD1ADE70E
:10EFC0009CF859102029EBD19CF858100129E7D062
:10EFD00061003FF025FE0028A0D0E1E704ABEDB2D0
:10EFE000336285F3118847F0CBFEE4E7681F002405
:10EFF0004868002430B593B004460DF10705089227
:10F0000000228DF807100993012100238DF81420A8
:10F010000B920E92109204918DF828108DF83C10EE
:10F020000168CDE90252CDE906220022CDE90C2388
:10F03000EFF3118C102383F3128803681B6A0BB360
:10F0400002A8049B02461BB1D3691432002BFBD1EA
:10F050000B6A6BB1996839B9934209D0196829B123
:10F060005B6899680029F7D01433F3E7C3E90040DF
:10F070005FFA8CFC8CF311882268136A002BFCD198
:10F0800013B030BD02AB5FFA8CFC0B628CF31188BD
:10F0900047F076FEF0E700BF30B40568EFF3118C5F
:10F0A000102383F3128803681B6AEBB18B68044654
:10F0B0000A461BB1D3691432002BFBD12B6A6BB10A
:10F0C000986838B9934209D0186828B15B68986885
:10F0D0000028F7D01433F3E7C3E900415FFA8CFC52
:10F0E0008CF3118830BC70475FFA8CFC29628CF37A
:10F0F000118830BC47F044BE30B58BB04FF0010CE6
:10F1000004460568009100218DF80CC08DF820C0E0
:10F110000991CDE90123CDE90411CDE90611EFF301
:10F12000118C102383F3128803681B6A0BB36846A3
:10F13000029B02461BB1D3691432002BFBD12B6A10
:10F140006BB1996839B9934209D0196829B15B68E4
:10F1500099680029F7D01433F3E7C3E900405FFA58
:10F160008CFC8CF311882268136A002BFCD10BB045
:10F1700030BD5FFA8CFCC5F820D08CF3118847F0C5
:10F18000FFFDF0E730B593B0002304468DF807107B
:10F190000DF106018DF8062001220DF107058DF80D
:10F1A00014308DF828208DF83C200B930E9310938B
:10F1B0000295CDE90332CDE90631CDE908320022CE
:10F1C00000230168CDE90C23EFF3118C102383F3A6
:10F1D000128803681B6A0BB302A8049B02461BB18A
:10F1E000D3691432002BFBD10B6A6BB1996839B922
:10F1F000934209D0196829B15B6899680029F7D052
:10F200001433F3E7C3E900405FFA8CFC8CF31188F8
:10F210002268136A002BFCD113B030BD02AB5FFA39
:10F220008CFC0B628CF3118847F0AAFDF0E700BF5D
:10F2300030B5002395B0012204468DF81C300DF145
:10F2400007050D93109312930B928DF830208DF8D3
:10F2500044208DF8071004950168CDE90532CDE909
:10F2600008330DF10F0300220A930023CDE90E238A
:10F27000EFF3118C102383F3128803681B6A1BB30E
:10F2800004A8069B02461BB1D3691432002BFBD1A4
:10F290000B6A6BB1996839B9934209D0196829B1E1
:10F2A0005B6899680029F7D01433F3E7C3E900409D
:10F2B0005FFA8CFC8CF311882268136A002BFCD156
:10F2C0009DF80F0015B030BD04AB5FFA8CFC0B62EB
:10F2D0008CF3118847F054FDEEE700BF0246074B60
:10F2E00002209A4208D801335B0840009A4280B25B
:10F2F00002D2FF28F8D97047704700BF7FF0FA02AA
:10F30000013905292DD81B4B4FF0280C02460CFB68
:10F3100001FC10B403F5D874634464444FF0010C4D
:10F32000046003F5D87480F888C093F8B00102280F
:10F3300019D0C9B2104809014158C3F8B41171B1CC
:10F340000221604683F8B0114FF48071A18102F16F
:10F3500010014C32C3E972125DF8044B7047002073
:10F36000FAE70020704793F8BD216046624483F8B5
:10F37000BD21F1E780780024382100242DE9F04FE9
:10F38000934F85B0DFF858924FF0010B4FF0000813
:10F39000904E0AE008F101080BF1010B283709F142
:10F3A0000509B8F1060F00F0FB803B78022BF1D184
:10F3B00099F90320511C00F0F680D2B294465FFA0E
:10F3C00088F10F2A6BD88448002403E0013403300D
:10F3D0002A2C64D00378002BF8D145788D42F5D1E2
:10F3E0007D4804EB44047D4D044402EB4200A478C4
:10F3F00005F8204005EB8000756884604068A842ED
:10F4000000F04B81B56AA84200F06581F56CA84216
:10F4100000F06981356FA84200F06981D6F89450F8
:10F42000A84200F07281D6F8B850A84200F084815A
:10F43000D6F8DC50A84200F07B81D6F80051A842F3
:10F4400000F08381D6F82451A84200F07981D6F8E3
:10F450004831984200F08E81D6F86C31984200F025
:10F460008381D6F89031984200F0A781D6F8B43164
:10F47000984200F09C81D6F8D831984200F0A981DA
:10F48000D6F8FC31984200F0AA81D6F82032984292
:10F4900000F0998116F8083C002B00F092800132B0
:10F4A000D2B262458DD90023019399F90420531CEF
:10F4B0007DD0D2B296465FFA88F10F2A68D84648C6
:10F4C000002403E0013403302A2C61D00378012B9F
:10F4D000F8D145788D42F5D13F4804EB440404440B
:10F4E00002EB4200A5783D4C04F8205004EB80006C
:10F4F000746885604068A04274D0B46AA04200F08D
:10F50000EE80F46CA04200F0F680346FA04200F070
:10F51000F780D6F89440A04200F0FB80D6F8B840BF
:10F52000A04200F00081D6F8DC40A04200F0F68056
:10F53000D6F80041A04200F01281D6F82441A04242
:10F5400000F00781D6F84841A04200F01F81D6F8AC
:10F550006C31984200F01481D6F89031984200F056
:10F560002081D6F8B431984200F01581D6F8D83110
:10F57000984200F04681D6F8FC31984200F03B8179
:10F58000D6F82032984200F0308116F8083C93B14A
:10F590000132D2B2964590D20023C7E90433F9E68E
:10F5A00005B0BDE8F08F4FF00F0C002207E74FF0D9
:10F5B0000F0E00227FE7132306F807BC06F8083C6D
:10F5C000E6E7142306F807BC06F8083C67E700BF27
:10F5D000307A00245C020024C46E09089C010024D7
:10F5E0006C5B00244FF0000C6346E2460AEBCA0055
:10F5F0000AF1010A06EB8000047F029400F11C046A
:10F600000394029C002CC3D1037206EB0C03039AF3
:10F610007B611323C56080F81DB050461370F2F76C
:10F62000BDFB019B002BB7D07869F2F763FA38690C
:10F63000F2F760FA3B697A68D968BB695962402180
:10F640005C60996002F120019C631960C3E9034486
:10F65000C3E90544C3E90744C3E90A44C3E90C44C8
:10F660007B698BB1D9683032FB6959621C629C633B
:10F67000C3E90024C3E90244C3E90444C3E90644DE
:10F68000C3E90A44C3E90C440023504660491A46C2
:10F69000F2F798FB01233B737CE61D469E460EEB7A
:10F6A000CE0A0EF10100019006EB8A0090F81CA032
:10F6B00000F11C0EBAF1000F7FF4F1AE03721423B7
:10F6C0003544C46080F81DB08EF8003001983D616B
:10F6D000F2F764FBE9E6012324259E46DFE74FF0BD
:10F6E000240C9A4682E7022348259E46D7E7032347
:10F6F0006C259E46D3E702234FF0480C9A4675E7E7
:10F7000003234FF06C0C9A4670E7042390259E4625
:10F71000C5E704234FF0900C9A4667E706234FF0A5
:10F72000D80C9A4662E705234FF0B40C9A465DE781
:10F730000623D8259E46B2E70523B4259E46AEE7AC
:10F740004FF490754FF0080EA9E70723FC259E465D
:10F75000A5E74FF4907C00234FF0080A46E7072303
:10F760004FF0FC0C9A4641E702234FF4B4754FF07A
:10F770000A0E94E74FF4A27501234FF0090E8EE7AD
:10F7800002234FF4B47C4FF00A0A2FE74FF4A27C17
:10F790004FF0090A2AE74FF4D87C04234FF00C0AF3
:10F7A00024E74FF4C67C03234FF00B0A1EE74FF407
:10F7B000D87504234FF00C0E71E74FF4C675032380
:10F7C0004FF00B0E6BE74FF4077507234FF00F0E4A
:10F7D00065E74FF4EA7505234FF00D0E5FE74FF430
:10F7E000FC7506234FF00E0E59E74FF4077C0723F4
:10F7F0004FF00F0AFAE64FF4FC7C06234FF00E0A96
:10F80000F4E64FF4EA7C05234FF00D0AEEE600BF64
:10F81000850E00008B681BB1CB691431002BFBD126
:10F82000C1E90002704700BF036810B59B68044639
:10F8300098470122FF236273A37310BD036810B5BC
:10F8400004461B6898470121236820469B68984717
:10F85000E37B0133E37310BDF0B583B004460D467E
:10F860001646089F0193384644F02EFE216828442E
:10F870003246E672A07220468E692946019BB44644
:10F8800003B0BDE8F040604703689B6A184700BFBB
:10F8900003685B6D03B11847704700BF0368DB6CFA
:10F8A00003B11847704700BF002310B5C373044667
:10F8B00042748A6C016003730AB119469047236849
:10F8C000012120469B689847FF2123680122A173EC
:10F8D000DB6C62731BB12046BDE81040184710BDB9
:10F8E0002DE9F04F4C484FF0010A4C494FF0020906
:10F8F0004B4B4FF0040808271026202540244FF0DA
:10F90000800EDFF820C130F8022F12F0010F03D073
:10F910001960083323F804AC12F0020F03D0196009
:10F92000083323F8049C12F0040F03D01960083345
:10F9300023F8048C12F0080F03D01960083323F861
:10F94000047C12F0100F03D01960083323F8046C04
:10F9500012F0200F03D01960083323F8045C12F072
:10F96000400F03D01960083323F8044C12F0800FC5
:10F9700003D01960083323F804EC12F4807F05D01B
:10F980004FF4807B1960083323F804BC12F4007F25
:10F9900005D04FF4007B1960083323F804BC12F43F
:10F9A000806F05D04FF4806B1960083323F804BCD6
:10F9B00012F4006F05D04FF4006B1960083323F880
:10F9C00004BC12F4805F05D04FF4805B19600833EB
:10F9D00023F804BC12F4005F05D04FF4005B1960FB
:10F9E000083323F804BC12F4804F05D04FF4804B49
:10F9F0001960083323F804BCD20B05D04FF4004241
:10FA00001960083323F8042C01F5806161457FF407
:10FA10007AAFBDE8F08F00BF5670090800000258A9
:10FA200098210024001C025810B50409013C062C42
:10FA300016D80D4A00F00F0332F8141041FA03F201
:10FA400012F001020ED0012098400138084045F024
:10FA500067FA064B064A1B5D184402EBC00010BD56
:10FA6000002010BD104610BD5870090868700908C4
:10FA700098210024F8B50C4F97F8343093B10B4C13
:10FA80000025A66801353079FFF7CEFF20B194F844
:10FA9000DC10F279F2F700FA97F8343004F5B47418
:10FAA000AB42EEDC0120F8BD801C00203C050020AC
:10FAB00038B50C4605460078FFF7B6FF611C0446D2
:10FAC000C9B210B14123C171837120466978F2F740
:10FAD00027FDAB7820461BB1BDE83840F2F79AB855
:10FAE000BDE83840F2F79CB82DE9F041FFF79CFFE4
:10FAF0000C4B054600241F680B4EBC4201DBBDE8E1
:10FB0000F08104EB4403F05C03EB0608FFF78CFF85
:10FB1000854204D121464046BDE8F041C8E70134A2
:10FB2000EBE700BFC85B0024985B0024054B53F84B
:10FB3000203033B11A689B8851690B4218BF1B04EF
:10FB400093617047581E00240E4B012210B40E4CD6
:10FB500093F800C002FA00F354F8200003EA0C0303
:10FB600051B1003B18BF012318B1016882883BB135
:10FB70008A615DF8044B7047B3FA83F35B09F3E7DE
:10FB80001204F5E7641E0024581E002410B5054C2D
:10FB900023681B6998472368002283F836209A63FC
:10FBA00010BD00BF4424002010B5084C236893F812
:10FBB000352012B1DB68984700B910BD044A012115
:10FBC0002368126883F836109A6310BD442400201D
:10FBD000501E00240D4A02EBC00310B593F8A4E2B6
:10FBE00093F8A5428EEA010C644500D110BDD3F80C
:10FBF000A032C0002BB11C688E459B8808BF1B0437
:10FC0000A361104480F8A5C210BD00BF8078002415
:10FC1000F8B5114E0124114D522716F8010BFFF7CC
:10FC200003FF0022202118B1C4718771F2F734F963
:10FC300015F8010BFFF7F8FE4FF0530C002240219E
:10FC400020B1C47180F806C0F2F726F90134E4B29D
:10FC5000052CE2D1F8BD00BF947400248874002400
:10FC600038B50C4614F8011B41B105462B682846EF
:10FC70001B68984714F8011B0029F7D138BD00BF55
:10FC800003681B68184700BF03682DE9F0415F6AED
:10FC90001FB13B46BDE8F041184704460D461646E5
:10FCA00000E023689B6820469847B042F9D3002EB5
:10FCB00008DD2E442368204615F8011B1B68984771
:10FCC000B542F7D1BDE8F08103685B68184700BF13
:10FCD00003689B68184700BF0368DB68184700BFCC
:10FCE00003685B69184700BF03689B6A03B1184744
:10FCF000704700BF0368DB6A03B11847704700BF55
:10FD000003682DE9F04116469A6A04460D460AB189
:10FD1000904723685F6A5FB1324629462046B8475C
:10FD20002368DB6AC3B12046BDE8F0411847236869
:10FD30009B6820469847B042F9D3002EF0DD2E4450
:10FD40002368204615F8011B1B689847B542F7D178
:10FD50002368DB6A002BE6D1BDE8F08170B504466C
:10FD60000E461546236820469B689847A842F9D35B
:10FD70002A4631462046BDE87040C1E72DE9F843E8
:10FD8000D0F8E8510446C24F95F800C017F91CE0BE
:10FD90005FFA8EF30F2B40F2AD80D0F830010028CF
:10FDA00051D0BC4E7368984200F05E81B36A9842AD
:10FDB00000F01981F36C984200F05C81336F984237
:10FDC00000F05C81D6F89430984200F05981D6F862
:10FDD000B830984200F05881D6F8DC30984200F0F4
:10FDE0006581D6F80031984200F06681D6F824315A
:10FDF000984200F06381D6F84831984200F0628161
:10FE0000D6F86C31984200F06181D6F89031984272
:10FE100000F06281D6F8B431984200F05F81D6F8E4
:10FE2000D831984200F06081D6F8FC31984200F059
:10FE30005F81D6F82032834200F05C8116F8083CDE
:10FE4000002B00F0A280D4F82C31002B50D0914E22
:10FE50007268934200F00A81B26A9A4200F0A6806A
:10FE6000F26C934200F00481326F934200F00481FF
:10FE7000D6F89420934200F00581D6F8B82093423A
:10FE800000F00481D6F8DC20934200F01181D6F80E
:10FE90000021934200F00E81D6F82421934200F015
:10FEA0000F81D6F84821934200F00E81D6F86C21DC
:10FEB000934200F00D81D6F89021934200F00A8120
:10FEC000D6F8B421934200F00B81D6F8D8219342A2
:10FED00000F00881D6F8FC21934200F00781D6F8A3
:10FEE0002022934200F0088116F8083C002B54D0E1
:10FEF000BDE8F883684B00211E461A4603E0013135
:10FF000003322A293ED010780428F8D15078604571
:10FF1000F5D101EB4101614A0EEB4E003144897885
:10FF200002F8201002EB800250689160C4F838118A
:10FF3000C4F8300107EB4C0797F9012001323FF478
:10FF40002EAF002204E0013203332A2A3FF427AF08
:10FF500019780529F7D159786145F4D102EB4202AD
:10FF60004E4B0EEB4E0E3244927803F82E2003EBEC
:10FF70008E0EDEF80430CEF80820C4F83421C4F820
:10FF80002C310CE7D4F83001D4E70B230CF1010C31
:10FF900006F8083C06F807CC55E72B780C2201330D
:10FFA00006F8082C06F8073CBDE8F883012303EBAC
:10FFB000C3032A7806EB830101329B00087FD2B28B
:10FFC000002895D1F058364B4A7798420CBFA020B4
:10FFD000A1200C230B773EF0E5FF6B682433C4F8B7
:10FFE0004C31BDE8F883012303EBC3030CF1010C92
:10FFF00006EB83089F0098F81C305FFA8CFC002BFE
:020000040805ED
:100000007FF421AF0B23F059DFF8949088F81DC0DE
:1000100048450CBFA020A12088F81C303EF0C2FF4C
:10002000F05995F8316048450CBFA020A1203EF062
:10003000B9FF1C4BB109B8F91600C8F81030C8F860
:1000400018403EF02DFFB8F91630002B07DB03F007
:100050001F0101225B098A40134941F823206B6884
:100060002833C4F84831EEE60023BDE700239EE7BD
:1000700002239CE70223B7E7032398E70323B3E7B0
:100080000423B1E7042392E70523ADE705238EE7B8
:10009000087400245C020024C46E09089C0100243A
:1000A000000002409D0B040800E100E006239BE7EE
:1000B00006237CE707237AE7072395E7082393E7DE
:1000C000082374E709238FE7092370E70A238BE7E6
:1000D0000A236CE70B236AE70B2385E70C2383E7EE
:1000E0000C2364E70D2362E70D237DE70E235EE713
:1000F0000E2379E70F2377E70F2358E7154B1B886B
:100100005BB9154A154B12781B688AB17BB11A6826
:100110009B8800B91B0493617047114BD3F8D4221C
:100120002AB150B9D3F8C022106083F8D1027047C9
:1001300080F00100002BEAD1F9E7B3F8D8C2012121
:10014000084AD3F8C002B2FBFCF20A41026083F80D
:10015000D1127047625B0024685B0024645B00245A
:100160008078002440420F0038B537F057FD0D4924
:100170000D4DD1F8FC20A5FB00500C4C42F08072D4
:100180000B4B800CC1F8FC204FF060420949C4F8C9
:100190004801C2F8B01F00225A601A6842F00102FA
:1001A0001A6038BD00ED00E083DE1B438078002438
:1001B000001000E055CEACC530B4EFF3118310222F
:1001C00082F312880B4C4FF0E0210B480025226887
:1001D000DBB2013222608A69C0F8DC22C0F8E0524A
:1001E0000A6983F31188054A1368013330BC136030
:1001F000704700BF501E0024807800246C2A002421
:10020000244B5B68C3F3080330B4EBB9EFF31183FD
:10021000D3B9214C4FF0E02C204A1368DCF81800C9
:1002200011688B42F9D1D4F8DC128842F5D8D4F8A1
:1002300048414FF47A7101FB04F2101AB0FBF4F05C
:1002400030BC01FB03007047EFF31183102282F3EF
:1002500012884FF0E022104C95691169C90303D54B
:100260000121C4F8E01295690C4ADBB21268D4F897
:10027000E00283F31188D4F8481110444FF47A72E5
:1002800002FB01F35B1BB3FBF1F330BC02FB00305C
:10029000704700BF00ED00E080780024501E00246D
:1002A0002DE9F04FED4C94F8E4622DED048B022E15
:1002B00091B0019040F0FC8117F090FD94F8083166
:1002C000D80700F1AD8218F0B5FA94F80831DB07D1
:1002D00000F1B98194EDD94AE149BDEEC44AD4EDAB
:1002E000DA4A94EDDF5AFDEEE44AD4EDDB5A14EE1F
:1002F000103ABDEEC55AFDEEE55A94EDDD6AB3F550
:10030000FA6FD4EDDC6ABDEEC66A94EDE07AA8BF60
:100310004FF4FA63FDEEE66ABDEEC77AD4EDDE7AFD
:10032000B3F57A7FD4EDE13AFDEEE77A94EDE24A57
:10033000B8BF4FF47A73A3F57A73C3EBC3135B00B2
:10034000A1FB03239B097F3B8DF8343014EE903AD8
:10035000B3F5FA6FA8BF4FF4FA63B3F57A7FB8BF6D
:100360004FF47A73A3F57A73C3EBC3135B00A1FB5D
:1003700003239B09C3F17F038DF8353015EE103A46
:10038000B3F5FA6FA8BF4FF4FA63B3F57A7FB8BF3D
:100390004FF47A73A3F57A73C3EBC3135B00A1FB2D
:1003A00003239B097F3B8DF8363015EE903AB3F569
:1003B000FA6FA8BF4FF4FA63B3F57A7FB8BF4FF472
:1003C0007A73A3F57A73C3EBC3135B00A1FB03231A
:1003D0009B097F3B8DF8373016EE103AB3F5FA6F74
:1003E000A8BF4FF4FA63B3F57A7FB8BF4FF47A73BE
:1003F000A3F57A73C3EBC3135B00A1FB03239B0933
:100400007F3B8DF8383016EE903AB3F5FA6FA8BFFF
:100410004FF4FA63B3F57A7FB8BF4FF47A73A3F55C
:100420007A73C3EBC3135B00A1FB032317EE102AFF
:10043000B2F5FA6F4FEA9313A8BF4FF4FA627F3B0D
:10044000B2F57A7F8DF83930B8BF4FF47A72A2F5E1
:100450007A72C2EBC2125200A1FB023217EE903A3E
:10046000FDEEE37AB3F5FA6F4FEA9212A8BF4FF4AC
:10047000FA637F3AB3F57A7F8DF83A20B8BF4FF42C
:100480007A73A3F57A73C3EBC3135B00A1FB032359
:1004900017EE902AFDEEC47AB2F5FA6F4FEA931385
:1004A000A8BF4FF4FA627F3BB2F57A7F8DF83B30FC
:1004B000B8BF4FF47A72A2F57A72C2EBC21253003F
:1004C00017EE902AB3F5FA3FB4BF00230123B2F52B
:1004D000FA6FA8BF4FF4FA62B2F57A7FB8BF4FF453
:1004E0007A72A2F57A72C2EBC2125200B2F5FA3FEA
:1004F00001DB43F00203D4EDE37AFDEEE77A17EE79
:10050000902AD4EDE47AB2F5FA6FFDEEE77AA8BF4F
:100510004FF4FA62B2F57A7FB8BF4FF47A72A2F55F
:100520007A72C2EBC2125200B2F5FA3F17EE902A6D
:10053000D4EDE57AA8BF43F00403B2F5FA6FFDEEFF
:10054000E77AA8BF4FF4FA62B2F57A7FB8BF4FF4EA
:100550007A72A2F57A72C2EBC2125200B2F5FA3F79
:1005600017EE902AD4EDE67AA8BF43F00803B2F55F
:10057000FA6FFDEEE77AA8BF4FF4FA62B2F57A7F20
:10058000B8BF4FF47A72A2F57A72C2EBC21252006F
:10059000B2F5FA3F17EE902AD4EDE77AA8BF43F000
:1005A0001003B2F5FA6FFDEEE77AA8BF4FF4FA62D6
:1005B000B2F57A7FB8BF4FF47A72A2F57A72C2EBC5
:1005C000C2125200B2F5FA3F17EE902AD4EDE87A43
:1005D000A8BF43F02003B2F5FA6FFDEEE77AA8BF9B
:1005E0004FF4FA62B2F57A7FB8BF4FF47A72A2F58F
:1005F0007A72C2EBC2125200B2F5FA3F17EE902A9D
:10060000A8BF43F04003B2F5FA6FA8BF4FF4FA62F7
:10061000B2F57A7FB8BF4FF47A72A2F57A72C2EB64
:10062000C2125200B2F5FA3F0E4AA8BF63F07F0330
:10063000D2F8CC128DF83C3092F89C32032B02D1C8
:10064000002940F0BF840023074F1D4684F8E432A0
:10065000064B1B78002B3CD10AE000BF80780024B9
:10066000D34D6210A82A0024A81E00244024002094
:10067000FFF7C6FD019BB200C3F101031844744BA0
:100680001B68D3F81CC004EB8603D3F8B8344FEAD8
:10069000DC114FEAA31EBEEBDC1F01D08B019911C8
:1006A0008842224440F3CF808001C2F8B80410E0B1
:1006B0000123684A9E4282F88C3021D10EF03EFB25
:1006C0000223654F1D4684F8E432644B1B78002BEF
:1006D000CED03B78472B07D104EB8603604AD3F892
:1006E000B8349B1122F8163004EB8503D3F8B834E4
:1006F0009B11C4F8C43411B0BDEC048BBDE8F08F7D
:1007000094F8E532002B40F0838094F8E632002B19
:1007100099D0002394F8E75284F8E632019B002D2B
:1007200040F0AE80002B00F0AF8094F8E832002B50
:1007300000F068854B4A4FF0010903969FED4A8A05
:100740009346DFF834811646484FDFF830A10EE0BB
:10075000736858469847032D3EDD013594F8E8321A
:1007600008F10408AAEC010A9D4280F26882072D74
:100770003B6BD4BF795DE9B2002BE9D07368584672
:100780000291984702997A8B04EB4103B88BB3F836
:1007900034339A4200F24E8207EE900A07EE103A86
:1007A000F8EE677AB8EE477AC7FEC77A09FA01F120
:1007B0003B6B194205D0D4F85C3313F4807F00FE04
:1007C000270ABCEEC00A032D10EE103A9BB200EED1
:1007D000103AB8EE400AC0DCB5EE400AF1EE10FA6D
:1007E000BBD0B8F8003006EE903AB8F80230F8EE18
:1007F000666A07EE103AB8EE477A30EE660A37EED0
:10080000667A60EE087A87EE870A30EE080AA4E777
:10081000144AD36810469847002384F8E53274E7F9
:10082000134B1B68002B3FF40EAF12491A6809786E
:100830009B88C907084F58BF1B04936100231D46BE
:1008400084F8E43204E7013BC2F8B83441E700BF62
:100850005825002038370020A81E002440240020FE
:10086000AC1E00249468002400007A448C570024B5
:10087000581E0024641E00246C6A00246C7B002433
:1008800013B1013D84F8E752C24AC34F1369002BEC
:1008900000F0AC8198470546FFF7B2FCD4F8F82386
:1008A000431BAA1A069300F0A181C4E9FE520199E4
:1008B000D4F80034CB1A06999942B8BF13463A7857
:1008C000DFEDB66A3E2A019AC4F800244FF6DC72C6
:1008D00000F0B2829A4240F2B631A8BF1A468A426C
:1008E000B8BF0A4607EE902A9B1AB8EEE77AB3FA29
:1008F00083F35B09C6EE877A84F80434A84B1A8028
:10090000A84BC3ED007AA84D2B68D80400F1DB8218
:1009100094F80D34022B00F09983042B00F0B98376
:10092000012B00F0C383D4F88024019B9F499B1ABC
:100930008B4239DC0199914239D007EE903A9C4BB9
:100940009FED9C7AB7EE006AF8EE677A93F829304B
:10095000DFED996A9FED995A67EE877A07EE103AB4
:10096000B4F80E24B8EEC77AB4F8103477EEC65A4D
:100970009A4236EEC77A27EE057AA7EE256A67EE29
:10098000277A87EE867A40F0F2828D4BB3F9002009
:10099000B3F90210914240F00083B3F90420B3F997
:1009A0000610914240F0CE82019BC4F88034854B02
:1009B000019A9A4200F27F8217F0FEFEB0F1000821
:1009C00018BF4FF001080EF047F9002894F80831DD
:1009D00094F89DB4B8BF404294F89CA403F001037E
:1009E0005FFA80F9BBF1000F05D0BAF1010F02D018
:1009F000002B40F07D82002284F89E24002B00F022
:100A0000FF80BAF1010F19D0B8F1000F16D16E4B6B
:100A1000187819F077FF88B96C4B01226C491B6874
:100A200081F8D92293F82C30003B18BF012381F8BC
:100A300098300AE094F89E34002BE2D00023644AF8
:100A400082F8D932012382F89830624B5A78002A12
:100A500000F0998094F89F24002A40F0948094F844
:100A60000C24002A40F08F8094F8A024002A40F043
:100A70008A80554A107819F045FF564B002840F0FF
:100A800082802A6882F01002C2F300125BEA02023E
:100A900003D1B8F1000F00F0E9831A79914517D31B
:100AA0004D49DFED4E7A91ED007AB4EEE77AF1EE42
:100AB00010FA15DA91ED017AB4EEE77AF1EE10FA58
:100AC0000EDA91ED027AB4EEE77AF1EE10FA07DA77
:100AD00052004B2AA8BF4B22D2B29145C0F0C68328
:100AE0003F4ADFED407A92ED097AB0EEC77AB4EE74
:100AF000E77AF1EE10FA40F1B98392ED047AB0EEA4
:100B0000C77AB4EEE77AF1EE10FA40F1AF8392EDD6
:100B10000E7AB0EEC77AB4EEE77AF1EE10FA40F151
:100B2000A583D4F8B02412B9019AC4F8B0245A8825
:100B3000B9F14A0FD4F8B014D4F8B43488BF5208CD
:100B400001985B1A03444FF47A7000FB02F293425F
:100B500002D9012284F89F24002900F094833A7876
:100B60001F2A07D14FF47A72B3FBF2F31E4AD380E7
:100B700001239380BAF1010F00F01E8301231D466B
:100B800084F8E432A1E53B781F2BF3D1164B002209
:100B90005A60EFE794680024A81E002400247449DA
:100BA00034680024887C00244057002490D003003F
:100BB0008C570024BD378636000080430000803B00
:100BC0008C060024404B4C00D05A0024B855002419
:100BD00038370020AC550024247D00249A99193E12
:100BE000983B00200000C842AC1E0024D4F8FC232F
:100BF000002A7FF45CAED4F80034019AD31A5EE682
:100C00000122C048C04980F8D9220A6892F82C20F5
:100C1000003A18BF012280F898203A781F2A01D1A3
:100C2000BA4A5360BAF1020F00F0BA82002384F886
:100C30009C34A3E707EE902AF8EE677AB6E5D4F87D
:100C40005813324694F8608311F04001039E08F077
:100C50000108039118BF4FF00008AD4984F8618383
:100C6000089109680491002B00F0DC82A94903F186
:100C7000FF39DFF8B4A200250988B9F1030FDFEDD1
:100C8000A69A09EE101A798AA8BF4FF003099FEDC2
:100C9000A38A08EE901AA249B8EE499A0B9291F8ED
:100CA00003B0F8EE688A0791798B0291B98B0AF14B
:100CB000480705910499CDE9096301F596714B4602
:100CC0004646D94688469B46002E00F08980954BC3
:100CD00003EB8500D0ED007ABCEEE77A17EE103A10
:100CE00098B2029B98427BD3059B984278D8C7F86C
:100CF0000080B9F1000F7CD04E460135C7FEE97A7D
:100D00000437C7FE887A5D45EAEC017ADCDDB0463F
:100D10000A9BCB46099E0B9AAB423DDD8249DFED33
:100D20007E9A01EB850948319FED7C8A01EB8507AE
:100D3000049901F5967ACDE909625646C24698466D
:100D4000BAF1000F00F06181764B03EB8500D0ED26
:100D5000007ABCEEE77A17EE103A98B2029B834213
:100D600000F25381059B8342C0F04F813E60BBF18E
:100D7000000F40F06381039B002B40F05F81013541
:100D8000C7FEE97A0437C7FE887AA845E9EC017AFC
:100D9000D6D1099ED0460A9A089B1968B8F1000F6F
:100DA00000F0DE81079BD9601B69002B00F02282D6
:100DB000CB1A0799096A9942C0F212825B4F3B78BD
:100DC000282B07D1D4EDDC7A504BFDEEE77A17EEF5
:100DD000901AD98094F8F433013384F8F43355E54C
:100DE000B9F1000F10D0032D00F0C981F0EE687A40
:100DF00083E7039B002B80D0E8B21CF0F3FD07EEE5
:100E0000900AF8EE677A78E7039B002BF4D13868F4
:100E1000049B181A002802DADAED007A6DE74FF029
:100E20000003E8B2002684F861331CF0DBFD07EE16
:100E3000900AF8EE677A60E79A4240F2B6313C4891
:100E4000A8BF1A468A42B8BF0A4680FB03C107EE14
:100E5000902A95B29A1ADB17B8EEE77AC3EBA10392
:100E60000699B2FA82F280FB01C10698C6EE877A33
:100E70005209C01784F80424C0EBA1002D49A1FB3E
:100E800005C147F6FF7C63454FEAD101A8BF634621
:100E90006045A8BF6046DFF874C0ACF80030264B50
:100EA000ACF802001D80254BACF80420ACF806100D
:100EB000C3ED007A27E51A4B9A78002A7FF47CADBF
:100EC00001229A7078E5D4F85833D9073FF520AD60
:100ED00094F80831DA077FF51BAD94F80C241AB9A1
:100EE00043F0020384F80831042016F009FE0FE5F0
:100EF000134B5B7E4B453FF69DAD012384F89E343A
:100F00009CE500BF38370020B8550024AC1E0024F3
:100F1000501E0024C457002400A00C4500803B4410
:100F2000145A00246C7B0024E47B0024A81E0024B7
:100F300067666666CDCCCCCC34680024887C0024FF
:100F40008C57002407EE902AB84AF8EEE77AD2EDE3
:100F5000006A82ED017A77EEE67AE7EE276AC2ED63
:100F6000006AFDEEE66A16EE902ADA801CE507EECE
:100F7000903AAF4BF8EE677AD3ED006A83ED017AD1
:100F800077EEE67AE7EE276AC3ED006AFCEEE66AE2
:100F900016EE903AA4F80E34F7E407EE902AA54A2C
:100FA000F8EEE77AD2ED006A82ED017A77EEE67A22
:100FB000E7EE276AC2ED006AFDEEE66A16EE902AB9
:100FC0005A80EAE4087B00287FF43DAB01230B73D1
:100FD0000921D2F8DC32516540F20312C3F8A410A3
:100FE0000DA9A3F890201A69C3F89C1003F1900191
:100FF000012AC3F8A80002D10DA8C3F8A000D2B2FC
:10100000186840F08FFFFFF71EBBBBF1000F05D043
:10101000032D13DC032D49FE287AB0E6039B6BB940
:101020003868049B181A0028C0F29780032D05DC4D
:101030004FF000034FF0000A84F86133E8B21CF06F
:10104000D1FC07EE900AF8EE677A98E67A4B7B4A75
:10105000DB7B04EB8303D3EDD87AFDEEE77A17EE62
:10106000903A1BB2B3F5FA6FA8BF4FF4FA63B3F529
:101070007A7FB8BF4FF47A73A3F57A73C3EB8323F7
:10108000A2FB0323C3F38F13A4F80E34A4F8103487
:1010900049E4FFF7B5F8D4F87C34C01A684B98429D
:1010A0007FF741AC0023A4F80E343CE4D4F81434A8
:1010B000019AD31A002BFFF636AC44F62063134492
:1010C000C4F814345F4BBFF34F8F5F4AC2F85C32F1
:1010D000BFF34F8FBFF36F8F94F8212442B194F880
:1010E000202433F8121004EB420289B2A2F86C14E7
:1010F00094F82D2442B194F82C2433F8121004EB08
:10110000420289B2A2F86C1494F8392442B194F8DE
:10111000382433F8121004EB420289B2A2F86C149E
:1011200094F8452442B194F8442433F8123004EB87
:1011300042029BB2A2F86C3494F8443494F80D2423
:1011400004EB4303012AB3F86C349BB27FF4EBAB9E
:101150009B08A4F81034FFF7E6BBD9ED007A0EE641
:101160003A4D079F2868FB6840F004003961CB1AAC
:10117000286078688342C8BF87F825801EE6DFEDC7
:10118000347AB0469FED337ACB46C9FE677A0A9B24
:10119000C7FE877A099E0B9A0425CAED007ABBE543
:1011A0000B6893F86230002B3FF4E8ACD4F85C3362
:1011B0001D063FF5E3AC39E5274B1B6893F85F301C
:1011C0004B45BFF4DBAC0223002284F89C34234B54
:1011D0005A609A61DA6243F83C2F5A609A60CDE413
:1011E0001A490123079880F825300B6823F004037F
:1011F0000B60E3E5079801611448016841F00401C0
:101200000160D6E5164B174A08931B68D4F858338B
:1012100083F0400894F86033C8F3801808EA0308A4
:1012200084F86183104B0793B6E500BF147D00245A
:10123000047D00240C7D00248C570024D34D6210C3
:1012400060E316006018012400ED00E0845A0024D9
:1012500000A00C4500803B44B8550024983B00207A
:10126000501E002494680024145A0024D4F8B0249A
:1012700032B1D4F8B4349B1A019A1344C4F8B4348C
:101280000023C4F8B0343B781F2B7FF473AC4FF4C9
:101290007A72D4F8B434B3FBF2F3024AD380002359
:1012A000938067E4AC1E0024CC4BDB79022B40F02A
:1012B00040812DE9F047CA4CB4F8A43513F400631B
:1012C0002DED028B00F04C8194F8C874002F00F0D3
:1012D0003982FEF795FFD4F85035DFF83483C31A0E
:1012E0009FEDC07A98F8006007EE903ABE4DD4EDBD
:1012F000498A4A2EF8EEE77AC4F85005C5ED018A0E
:1013000067EE877AC5ED097A00F05E81382E00F02D
:101310005B81492E40F05E81B44BB4F8D824B4F818
:10132000DA141A80B4F8FC20D9805A80B4F9582510
:101330009A80DFF8E0A2062F9AF81C30A3F105038B
:10134000B3FA83F34FEA531384F8E0341BD1A84B6C
:10135000D3ED137AD3ED125AD3ED146A67EEA77A60
:1013600093ED006A9B89E5EEA57A07EE103AB8EE98
:10137000C77A36EEC77AE7EE077AB1EEE77A66EE1D
:10138000077AC5ED057AB4F95A35DFED9A6AD11AB4
:10139000DFED997AA4F8DA3407EE101AB8EEC77ABE
:1013A000B4EEE67A67EE277AF1EE10FA00F23881B1
:1013B0009FED9A7A77EE877AC5ED077AB0EEE78AE5
:1013C0004A2E85ED0E8A02D188490A814B8194F814
:1013D0005C95B9F1000F63D0D4F860354C2E9FEDC9
:1013E000876A07EE903A864AB4F8FA30F8EE677AE0
:1013F000D2ED006AA4F8D834C5ED086A27EE867AE3
:10140000C5ED027A85ED037A92ED017AC2ED017A9B
:1014100077EE677A87EEA60A85ED0B0A00F04B811E
:10142000B4F8721599B307EE903A94F89335F1EE4B
:10143000005A92ED0F7AF8EEE77AB5EEC07A77EEC1
:10144000C07AF1EE10FAF0EEE77A67EE867A06EEF1
:10145000103AB8EEC66AC7EE866A36EEA56AC5EEE1
:10146000867AC5ED1F7A40F37781DFED667AB0EEBC
:10147000006A67EE277AC7FEC67A042F05D1B0EE60
:101480000C7AC6FEC76A76EEA77AC5ED0F7A482EAB
:1014900000F00C814A2E03D144F010FD534B18800C
:1014A000FEF7AEFE9AF81C30052B40F0C78094F88A
:1014B000D03013F0010200F0DD80D4F894255249B9
:1014C000821A8A4240F3F68203F0020394F8FE2067
:1014D000C4F89405002B94F99A350CBF0121002122
:1014E00084F898150CBF00210121042A34BF012281
:1014F0004FF0FF321344022B1A46A8BF0222012BE1
:1015000022EAE27284F89A2500F3DC82002384F850
:10151000993584F84C15092F32D8DFE817F01A02F4
:101520006502F701BF016001500125002700370166
:101530003301364B03F1780102E006338B420ED0C3
:101540001A78072AF9D19878DA789042FFF4B1AE88
:101550005A79002A7FF4ADAE06338B42F0D1704742
:101560001F4684F8C834B4E618F0A8FB95ED057A58
:10157000D5ED1B7AB4EEE77AF1EE10FA00F3EF80C6
:1015800098F800304A2B18D0382B16D0242B09D1CC
:10159000DFED197A95ED100A20EE270A44F08EFC53
:1015A000124B188018F044FA17F088FF0023BDECA6
:1015B000028B84F85C35BDE8F08795ED120A44F0A3
:1015C0007DFC0A4BD880EDE7B0EE680A44F076FC6B
:1015D000064B9880B4F95825ABE600BFC4570024E9
:1015E00080780024BD378635487D0024AC1E002459
:1015F000482400200000E1C4CDCCCC3D0AD7233CD8
:10160000E47D00243EC3AE393F420F00D057002492
:10161000A81E00244C6800240000E1440000B443EC
:101620005FED036AB4EEE67AF1EE10FAC4BF1FED87
:10163000057A77EEC77AC5ED077ABFE6002384F80E
:101640004C35092F9CD801A353F827F053190508EE
:10165000731A05080D1905089D180508DF170508F8
:10166000BF170508691505086D1505088D170508CC
:101670008517050884F84C25092F81D801A353F854
:1016800027F000BF531905089B1A05080D19050816
:101690009D180508DF170508BF1705086915050817
:1016A0006D1505088D1705088517050844F006FC1B
:1016B000C64B9880F4E6FDEEC07AC44817EE901A47
:1016C0000181B4F8721500293FF4EAAE07EE903AB2
:1016D00094F89335B1EE005ADFEDC25AF8EEE77A8E
:1016E00092ED0F7AB5EEC07A77EEC07AF1EE10FA8D
:1016F000F0EEE77A67EE867A06EE103AB8EEC66A42
:10170000C7EE866A76EE854A66EEA57A85EE246A8D
:10171000FDEEE77A17EE903A438185ED1F6A40F3BC
:10172000D881DFEDAB7AB0EE006A67EE277AC7FEAC
:10173000C67A27EEA57ABDEEC77A17EE103A1BB22D
:1017400083819AE6012384F8C83417F0B7FE18F0B5
:101750006FF994F8C874BCE5DFED9E7A8DE69E4A79
:10176000136843F00073136094F80831D90709D562
:1017700094F80C241AB943F0020384F808310720C6
:1017800016F0BEF9002384F8C834F9E6924A1368CB
:1017900043F00073136094F80831DA0709D594F820
:1017A0000C241AB943F0020384F80831012016F022
:1017B000A7F9002384F8283584F8C834E0E6D5ED8D
:1017C000137AF4EEE87AF1EE10FA05DD0622002332
:1017D00084F8C82484F8283518F070FAD0E6B7EEFB
:1017E000007AD5ED1A7AD5ED0A5AB4F87235F4EECE
:1017F000C77A95ED147AF1EE10FA44BF77EEA57A28
:10180000C5ED1A7A07EE903A744BF8EEE77A5B7AF8
:10181000F4EEC77AF1EE10FACCBF012200229A4210
:1018200005D177EEC77AA7EEA57A85ED147AB7EEE3
:10183000007AD5ED207AF6EE006AB0EE006A37EE57
:10184000677A27EE267AE7EE257A36EE677AC5EDD7
:10185000207A85ED1E7AB9F1000F3FF491AEB4F80D
:101860006C35D5ED035A07EE103A95ED176AB8EED0
:10187000477AF4EEC65A67EE266A85ED157AF1EEE0
:1018800010FA66EEA77AC5ED167A3FF679AE052214
:10189000002384F8C82484F8283571E6B7EE007A6E
:1018A000D5ED1A7AF4EEC77AF1EE10FA05D595ED7A
:1018B0000A7A77EE277AC5ED1A7AF3EE0E7AB4EE4D
:1018C000E78AF1EE10FA0DD5B4F86C3507EE903AD0
:1018D0000423F8EE677A84F8C8340023C5ED157A3E
:1018E00084F82835B4F8723595ED0B7A07EE903A06
:1018F0003A4B85ED147AF8EEE77AB4EEE77AF1EE3A
:1019000010FA4CBF012200225A7239E6D5ED117A45
:10191000324BF4EEE87A1A7AF1EE10FACCBF0123DA
:101920000023934200F0D980B4F88235C5ED127AD5
:1019300007EE903A95ED037AF8EEE77AB4EEE77A9F
:10194000F1EE10FA02DD032384F8C834EB6A2B654C
:1019500016E694F80831DE0704D4214B1B7A002BDD
